:020000040000FA
:060000000209E80201B64E
:03002B0002084385
:03003B000205318A
:03004B00021CF1A3
:030053000200E7C1
:03005B00021CF292
:03006300021CF389
:1000830002014B01FF01010F10FEFFFA11FA11FAF1
:1000930011FA11B610B010FA11E41E00000000A806
:1000A3001F000000000C0000000C0001FFFF010214
:1000B30000320A000000A30AE80364006400B801E8
:1000C30002050000000205020701051E02051E02CB
:1000D3000A0A03B80B02803E01020125250A140116
:1000E300E0020206C0E074F21203CFA2AFE433FED3
:1000F300D2AFE5A7FFE5A1F5085F5410600612181B
:10010300BA75A1EFE5085F540860081218C075A11D
:10011300F7802BEFA2E0C0D0E508A2E092F012092D
:1001230032158182F05017906198E0F8900B79E0D6
:10013300C398A2D265D0335002E8F075A1FEEEA2B7
:10014300E092AF7F01020486C0E074F21203CFA2F3
:10015300AFE433FED2AF9061A4E0F8759B00E59164
:1001630058540860087591F7121902802AE59158CE
:10017300541060087591EF121908801BE8A2E0C0C3
:10018300D0E591A2E092F0120932158182F0500776
:10019300E0C2E0F0121A529061A3E0F8E5E9585486
:1001A30004600E121A2875E9FB906193E0A2E64001
:1001B300F2808BC0E074F21203CFA2AFE433FED21D
:1001C300AF9061A5E0F8E5BF585404600675BFFB26
:1001D300121A6A020141C3E498F8E499F912021A67
:1001E3008026C3E49AFAE49BFBE920E7E912021AAA
:1001F300E498F8E499F922C3E498F8E499F912022F
:100203001AE498F8E499F9C3E49AFAE49BFB22EB25
:1002130020E7CFE920E7E0B90010BB0008E88AF047
:1002230084F8AAF022E4FBC8FA22EB70227B10C800
:1002330033C8C933C9335007C39AC3DBF280069A64
:1002430050012ADBEAC833F4C8C933F4C9FA22756A
:10025300F008E4C833C8C933C933C99AC99B5004E9
:10026300C92AC93BD5F0ECFBC833F4C8E4C9FA2268
:10027300080808EAC0E0EBC0E086F0E7A4FA180932
:1002830086F0E7A42AFA180986F0E7A42AFA1809DF
:1002930086F0E7A42AFA1986F0E7A4FBE5F02AFA28
:1002A300190886F0E7A42BFBE5F03AFA190886F063
:1002B300E7A42BFBE5F03AFA18180986F0E7A4C582
:1002C300F02BFBE43AFA1908E7C5F0C6A426F6E5D5
:1002D300F03BFBE43AFA1886F0E7A4F6E5F00826CB
:1002E300F6E43B08F6E43A08F6D0E0FBD0E0FA2265
:1002F300E4CFC0E0E4CEC0E0E4CDC0E0E4CCC0E0B5
:1003030075F020C3E633F608E633F608E633F6085D
:10031300E633F6181818EC33FCED33FDEE33FEEF3D
:1003230033FFC3EC9709ED9709EE9709EF97191976
:1003330019400FFFEC97FC09ED97FD09EE97FE19A5
:100343001906D5F0BEECF709EDF709EEF709EFF75B
:10035300191919D0E0FCD0E0FDD0E0FED0E0FF2277
:100363002518C582C0E0E51934FFC583C0E0E51850
:10037300C3958224F810AF088583198582188008F5
:10038300858319858218D2AFCEF0A3E520F0A37838
:1003930008E608F0A3DEFAEFF0A3E58124FAF8E615
:1003A30008F0A3E608F0A3E608F0A30808E608F0BF
:1003B300A3E608F0A315811581D0E0FED0E0F8157F
:1003C3008115811581E8C0E0EEC0E022C0D0251878
:1003D300C582C0E0E51934FFC583C0E0E518C395C5
:1003E3008224F310AF0885831985821880088583DA
:1003F30019858218D2AFC8F0A3E9F0A3EAF0A3EB02
:10040300F0A37908E709F0A3D8FAECF0A3EDF0A381
:10041300EEF0A3EFF0A3D0E0F0A3D0E0F0A3D0E0A0
:10042300F0A3E520F0A3E5F0F0A322120A4AB900F5
:1004330003020470E49003017848790F8002F0A36B
:10044300D8FCD9FA901148AA82AB839000867862CF
:1004530079018015E493A3AC82AD838A828B83F008
:10046300A3AA82AB838C828D83D8E9D9E77582678F
:100473007583B374031207BB7582EC75831C740018
:100483001207BB851983851882E0C0E0A3E0F9A3B6
:10049300E0FAA3E0FBA37808E0F608A3DFFAE0FCA8
:1004A300A3E0FDA3E0FEA3E0FFA3E0C0E0A3E0C060
:1004B300E0A3E0F5D0A3E0F520A3E0A3F5F010AFAF
:1004C300088583198582188008858319858218D247
:1004D300AFD082D083D0E0F8D0E032FA0675F010C6
:1004E3008E1A8F1B85821F85831E8518828519832B
:1004F300E0CEA3E0CF851F82851E83EBC9EAC8ED5A
:10050300CBECCAC3E833C8E933C9EA33CAEB33CB0C
:10051300C3EA9EF51DEB9FF51CB35004AB1CAA1D4B
:10052300EC33CCED33CDD5F0DAAE1AAF1B22C0E0FD
:10053300C0D0E8C0E0E9C0E0C082C083C2E9900651
:100543000CE0602890060DE0F8A3E0F5838882E0D4
:10055300F5C190060DE0240108A3E03400F99006EC
:100563000DE8F0A3E9F090060CE014F0D083D082FC
:10057300D0E0F9D0E0F8D0D0D0E032D083D082EC14
:10058300C0E0EDC0E0E493A3FCE493A3FDED4C6075
:100593000D120656EC24FFFCED34FFFD80EFE493CF
:1005A300A3FCE493A3FDED4C600D1206C6EC24FFFF
:1005B300FCED34FFFD80EFD0E0FDD0E0FCE493A33D
:1005C300C0E0E493C0E022851983851882E0A3FE8E
:1005D300E0A3F5207808E0A3F608DFFAE0A3FFE044
:1005E300A3C0E0E0A3C0E0E0A3C0E0E0A3C0E0E07C
:1005F300A3C0E010AF08858218858319800885821F
:1006030018858319D2AFD083D0820207C1D083D09B
:1006130082E9C0E0E493A3C386F0C5F095F0F9083E
:10062300E493A386F0C5F095F0700BE493A3C3990C
:100633004005E9048002A3E475F002A42582F58253
:10064300E5F03583F583D0E0F9E493A3C0E0E493C8
:10065300C0E022C0E0C3E493960874019396184067
:100663000FE493667008087401936618700070199C
:10067300A3A3C3E49396087401939618A3A3400D10
:10068300D0E0D0E0D0E00205BAA3A3A3A3A3A3D0F4
:10069300E0227404800474028000CCC0E0EDC0E06A
:1006A300E518C39CCCAD1950011D10AF068C188DF5
:1006B3001980068C188D19D2AF12073DD0E0FDD0FA
:1006C300E0FC22C0E0C0F088F0E493667008087490
:1006D300019366187000A8F0A3A3700BD0F0D0E0CC
:1006E300D0E0D0E00205BAA3A3D0F0D0E022D083BB
:1006F300D082CCC0E0E493A3600612079C1470FA86
:10070300E493A3600612088D1470FAD0E0FCE4931E
:10071300A3C0E0E493C0E022CAC0E0E493A3C5828F
:10072300CCC582C583CDC583F0A3C582CCC582C5A4
:1007330083CDC583DAE5D0E0CA22CAC0E0E0A3C511
:1007430082CCC582C583CDC583F0A3C582CCC582C7
:10075300C583CDC583DAE6D0E0CA22C008C3E096DC
:10076300F50808A3E096420808A3E096420808A308
:10077300E09645087001D3D00822700908080822C2
:100783006016181818C6C333C608C633C608C6335E
:10079300C608C633C6D5E0EA22C0E0E493A3D39CDF
:1007A3005010E493A3C39C400AD0E0D0E0D0E00211
:1007B300070EA3A3A3D0E022C09FF59FE473D09FAD
:1007C30022D083D082C09FE493C0E0740193C0E041
:1007D300740293F59F222518F58210AF08F518408F
:1007E3000215198008F51840021519D2AF8519832F
:1007F300227404800A74038006740280027401C0A8
:10080300E0F4041207D9D0E0120A2522C0D025183B
:1008130010AF08F518500205198008F518500205A5
:1008230019D2AFD0D022BB0102E722C082C0838994
:10083300828A83BB0003E08002E493D083D08222C8
:10084300C0E0C0D0E8C0E0E5A8D2AFC2C7A2E7923B
:10085300AFD0E0F8D0D0D0E0326016080808C6C3A5
:1008630013C618C613C618C613C618C613C6D5E0D2
:10087300EA22C3E0C696F608A3E0C696F608A3E00C
:10088300C696F608A3E0C696F622C0E0E493A36CEE
:100893007009D0E0D0E0D0E002070EA3A3D0E0229D
:1008A300251810AF08F518400215198008F51840EF
:1008B300021519D2AF22E76670100809E766700ABD
:1008C3000809E76670040809E76622C3E09608A3EF
:1008D300E09608A3E09608A3E096A2D265D033225F
:1008E300E066701008A3E066700A08A3E06670046F
:1008F30008A3E06622C3E096F008A3E096F008A3FD
:10090300E096F008A3E096F022E026F608A3E0368E
:10091300F608A3E036F608A3E036F622E627F60843
:1009230009E637F60809E637F60809E637F622C07E
:10093300E0E8C0E0E58124FCF8E6A2E7D0E0F8D0E7
:10094300E022700422600D18C6C333C608C633C63E
:10095300D5E0F41822E657F60809E657F60809E643
:1009630057F60809E657F622E056F608A3E056F6CE
:1009730008A3E056F608A3E056F622E056F008A3D3
:10098300E056F008A3E056F008A3E056F022E6474D
:10099300F60809E647F60809E647F60809E647F6C2
:1009A30022E026F008A3E036F008A3E036F008A31F
:1009B300E036F022E4C396F608E496F608E496F6E9
:1009C30008E496F622C6F4C608C6F4C608C6F4C6FA
:1009D30008C6F4C622C3E09608A3E09608A3E096EF
:1009E30008A3E0962275D00075814075180175192A
:1009F300030002042EE0F608A3E0F608A3E0F608DD
:100A0300A3E0F622600C08C6C313C618C613C6D5E6
:100A1300E0F422E6F008A3E6F008A3E6F008A3E674
:100A2300F022CAC0E0E6F0A308DAFAD0E0FA22E046
:100A3300FAA3E0FBA3E0FCA3E0FD22EAF0A3EBF0C2
:100A4300A3ECF0A3EDF022E5C754F84401F5C77910
:100A530001222518F582E43519F58322C2AF75D634
:100A63009F020000221207C42724001207C4402457
:100A7300001207C46624001207C4A124001207C48D
:100A8300E524001207C40C25001207C45D250012DB
:100A930007C40D26001207C4C526001207C48D27FC
:100AA300001207C44D28001207C49128001207C47E
:100AB300B628001207C4F928001207C446290012F9
:100AC30007C4BC2A001207C4422B001207C4602BC0
:100AD300001207C48A2B001207C4A42B001207C4F8
:100AE300B32B001207C4BE2B001207C47E2C0012C6
:100AF30007C4D72C001207C4992D001207C4A12DD7
:100B0300001207C4352E001207C4A12E001207C419
:100B1300CC2F001207C4F12F001207C47630001245
:100B230007C40531001207C4C931001207C4E831F4
:100B3300001207C4F732001207C40933001207C4B6
:100B43007433001207C48D33001207C4C934001272
:100B530007C45B35001207C49435001207C4E0359F
:100B6300001207C4F336001207C41739001207C472
:100B73002239001207C42D39001207C43839001274
:100B830007C44239001207C44D39001207C467393C
:100B9300001207C47139001207C47B39001207C45D
:100BA3008639001207C4AE39001207C4093A00128D
:100BB30007C4253A001207C4DF3A001207C4C33C36
:100BC300001207C41C3D001207C44C3E001207C4A8
:100BD300723E001207C4EC3F001207C477430012B1
:100BE30007C44945001207C41247001207C4BF4790
:100BF300001207C43349001207C4D249001207C4C4
:100C0300174A001207C4814A001207C4904A00120F
:100C130007C4104D001207C4B94E001207C4264F73
:100C2300001207C40550001207C42851001207C45C
:100C33009052001207C4AF52001207C404530012AB
:100C430007C40954001207C43154001207C489545D
:100C5300001207C46855001207C4AC55001207C43C
:100C6300F755001207C46256001207C4A7570012B3
:100C730007C40B58001207C44559001207C4AC5BE4
:100C8300001207C4DD5B001207C4955D001207C4A0
:100C9300EA5D001207C4EE5E001207C48B5F001208
:100CA30007C4E45F001207C49760001207C43961E8
:100CB300001207C4D961001207C47E62001207C480
:100CC3006A80011207C4A980011207C4F0820112CD
:100CD30007C43A83011207C45584011207C4BD84B3
:100CE300011207C4F284011207C46686011207C405
:100CF300E988011207C4128A011207C4C58A0112C6
:100D030007C42193011207C4B693011207C49D9629
:100D1300011207C49697011207C40498011207C46D
:100D23004A99011207C4299A011207C40E9C0112A1
:100D330007C41F9E011207C4779E011207C4499F6F
:100D4300011207C4779F011207C434A0011207C41C
:100D53000BA1011207C4D2A1011207C476A201128A
:100D630007C49FA2011207C4C1A2011207C417A599
:100D7300011207C4EFA5011207C433A6011207C469
:100D83009BA6011207C453A7011207C485A701122A
:100D930007C4C9A7011207C4FFA7011207C44BA8C0
:100DA300011207C4A0A8011207C4A5A8011207C411
:100DB300F8A8011207C41DA9011207C42CAA011225
:100DC30007C490AA011207C400AB011207C48CAB7D
:100DD300011207C459AE011207C43DAF011207C483
:100DE300C0B0011207C4F6B2011207C4A4B30112C2
:100DF30007C454B4011207C495B6011207C438B727
:100E0300011207C47FB7011207C42BB9011207C42B
:100E13003FB9011207C449B9011207C471B90112DC
:100E230007C47DB9011207C49CB9011207C4BCBB36
:100E3300011207C40BBD011207C44FBD011207C441
:100E4300F7BD011207C4DABE011207C485BF011240
:100E530007C4D1C0011207C4CFC1011207C475C2B0
:100E6300011207C416C3011207C42DC3011207C41C
:100E730064C3011207C46EC3011207C479C301120C
:100E830007C497C3011207C4DBC3011207C438C4E4
:100E9300011207C45DC4011207C477C4011207C459
:100EA30003C5011207C420C6011207C47CC6011280
:100EB30007C463C7011207C48AC7011207C4FEC768
:100EC300011207C479C8011207C47DC9011207C4FE
:100ED30073CA011207C422CB011207C435CC011215
:100EE30007C4D1CC011207C453CD011207C431CEBC
:100EF300011207C469CE011207C4C1CE011207C48F
:100F03008ACF011207C4ABCF011207C432D001123A
:100F130007C456D0011207C478D0011207C4C1D048
:100F2300011207C4D7D2011207C4BAD3011207C4EE
:100F33006BD4011207C4A1D6011207C4F1D6011262
:100F430007C431D7011207C473D7011207C4CFD71F
:100F5300011207C4FDD7011207C421D8011207C427
:100F630074D8011207C4A2D8011207C4DBD8011236
:100F730007C430D9011207C496D9011207C400DB94
:100F8300011207C423DD011207C490DD011207C457
:100F9300B9DD011207C444DE011207C4ABDE01123E
:100FA30007C4F6DE011207C41ADF011207C43EDFCD
:100FB300011207C499DF011207C4B4DF011207C489
:100FC3006DE0011207C434C5031207C473C50312CD
:100FD30007C47880021207C4BE80021207C49E8130
:100FE300021207C4A082021207C4A383021207C419
:100FF3002F85021207C48D85021207C44A86021286
:1010030007C46887021207C4D987021207C4158868
:10101300021207C46388021207C46D88021207C450
:10102300B188021207C40D89021207C4A8890212EB
:1010330007C4258A021207C4F48A021207C48D8BDF
:10104300021207C4AD8B021207C4E38B021207C45A
:10105300148C021207C4D58C021207C4E58C021249
:1010630007C4398D021207C4548D021207C4668D5A
:10107300021207C46F8D021207C4C98D021207C47E
:10108300258E021207C4718E021207C48C8E0212BF
:1010930007C4BD8E021207C4DA8E021207C4E68E9D
:1010A300021207C45A90021207C47390021207C4B3
:1010B300DA90021207C4ED90021207C4FB900212E9
:1010C30007C4AF91021207C49392021207C4999303
:1010D300021207C42394021207C42D94021207C4F8
:1010E3009A94021207C4B194021207C4E394021241
:1010F30007C41C95021207C44695021207C4A7959C
:10110300021207C4C795021207C4E595021207C469
:101113002B96021207C45197021207C49E9702121C
:1011230007C4CD97021207C44398021207C46B98F1
:10113300021207C4A498021207C4B298021207C489
:101143000A99021207C45999021207C49899021204
:1011530007C4C899021207C4F499021207C4FF997D
:10116300021207C41D9A021207C4DF9A021207C4AF
:10117300E99A021207C42A9B021207C47F9B021238
:1011830007C4939B021207C4909C021207C4A39C3A
:10119300021207C4B89C021207C45A9D021207C464
:1011A300DD9D021207C49B9E021207C4A69E021273
:1011B30007C4D29F021207C4EE9F021207C440A0C5
:1011C300021207C47FA0021207C494A0021207C42C
:1011D300F6A0021207C485A1021207C4D0A102120D
:1011E30007C421A4021207C49FA4021207C414A5B2
:1011F300021207C436A7021207C44EA7021207C47D
:1012030051A7021207C45DA7021207C471A70212F5
:1012130007C479A7021207C4ACA7021207C45CA8CB
:10122300021207C4D2A8021207C445A9021207C4B6
:10123300F9A9021207C4AEAA021207C4CDAA021268
:1012430007C473AB021207C49EAB021207C4A1AB5F
:10125300021207C40BAC021207C433AD021207C457
:101263000BAE021207C496AE021207C4AFAF02124E
:1012730007C46CB0021207C4A5B0021207C4D6B0EB
:10128300021207C494B1021207C4C4B1021207C404
:101293009FB2021207C438B3021207C4C3B30212C7
:1012A30007C474B4021207C4F7B4021207C429B501
:1012B300021207C46AB5021207C498F4011207C4E4
:1012C300FDF4011207C435F5011207C484F50112B8
:1012D30007C4A6F7011207C489F9011207C4F6FC73
:1012E300011207C42BFD011207C44DFD011207C4EF
:1012F300B2FD011207C4E8FD011207C40BFE01127F
:1013030007C438FE011207C4C3D8021207C42279E6
:10131300001207C46E79001207C4DC79001207C4F7
:10132300FD79001207C4AD7A001207C4B67A001221
:1013330007C4097B001207C4327B001207C4997BE0
:10134300001207C42A7C001207C46C7C001207C475
:10135300B67C001207C4157D001207C4D323001204
:1013630007C4D27D001207C4117E001207C4507E49
:10137300001207C4857E001207C4977E001207C4BB
:10138300A97E001207C4C87E001207C4D17E0012D2
:1013930007C4877F001207C4C77F001207C48DC02C
:1013A300031207C46AB7031207C4A0B7031207C422
:1013B300D4B7031207C424B9031207C4A7E0011268
:1013C30007C4E6E1011207C422E2011207C4E1E304
:1013D300011207C40AE4011207C49DE6011207C4FF
:1013E300E1E6011207C46AE8011207C402E9011227
:1013F30007C46AE9011207C40BEA011207C44DEAE4
:10140300011207C48DEA011207C418EC011207C4C4
:1014130088ED011207C4ADEF011207C4DBEF01121F
:1014230007C402F0011207C40BF0011207C466F0EF
:10143300011207C4F9F0011207C417F4011207C41B
:1014430012C6031207C428C6031207C4B19E0312AF
:1014530007C4E49E031207C4819F031207C4BD9F00
:10146300031207C4D49F031207C4F99F031207C4CE
:101473003EA0031207C46FA0031207C4A7A0031260
:1014830007C421A2031207C43BA2031207C4E9C481
:10149300031207C460C1031207C4A8C1031207C41F
:1014A300E7C1031207C4FAC1031207C404C203123B
:1014B30007C44487031207C46A87031207C47787E4
:1014C300031207C4A587031207C4E287031207C4E4
:1014D300D788031207C43689031207C45F8903122E
:1014E30007C47889031207C49589031207C41A8AAB
:1014F300031207C4D58A031207C4148B031207C44B
:101503009A8B031207C4AF8B031207C4C48B031255
:1015130007C4D98B031207C4EE8B031207C4128CC2
:10152300031207C42B8C031207C43C8C031207C499
:10153300528C031207C46B8C031207C4AB8C0312C7
:1015430007C48B96031207C4F196031207C4FF96D0
:10155300031207C40D97031207C42097031207C48D
:101563005D98031207C47098031207C48998031285
:1015730007C4FA98031207C43099031207C4499A9F
:10158300031207C4D7E8021207C429E9021207C4E9
:1015930012EA021207C4ABEA021207C4F5EA021206
:1015A30007C452EB021207C484EB021207C425ECF2
:1015B300021207C451EC021207C46CEC021207C4F6
:1015C300BBEC021207C4D1EC021207C4DEEC021218
:1015D30007C412ED021207C464ED021207C4BEED84
:1015E300021207C40CEE021207C42EEE021207C445
:1015F300A7F0021207C4DCF0021207C473F102124F
:1016030007C4E8F1021207C4EDF1021207C429F27C
:10161300021207C488F2021207C428F3021207C495
:101623004DF3021207C457F3021207C45AF302120E
:1016330007C4E3F3021207C4FEF3021207C411F452
:10164300021207C44CF4021207C44FF4021207C477
:101653005AF4021207C496F4021207C49CC403127C
:1016630007C4B4C4031207C40080031207C44F8025
:10167300031207C4F181031207C4AD83031207C425
:10168300F583031207C4DD84031207C40E86031215
:1016930007C43086031207C48C86031207C410875D
:1016A300031207C4CA62001207C4DF62001207C430
:1016B3005C63001207C4E563001207C4616400128F
:1016C30007C4CA64001207C40D65001207C49465F9
:1016D300001207C42866001207C4B466001207C4C8
:1016E300F666001207C4B16B001207C4E06B001268
:1016F30007C4D76D001207C45B70001207C41471CE
:10170300001207C43172001207C47F75001207C4A8
:101713008F75001207C45A77001207C408780012A5
:1017230007C48A78001207C4CBDA021207C485DB28
:10173300021207C427DC021207C497DC021207C493
:1017430050DF021207C427E0021207C494E002121A
:1017530007C411E2021207C4DBE2021207C44BE31F
:10176300021207C411E5021207C424E6021207C4D9
:10177300BDE6021207C483E7021207C474C603124C
:1017830007C476C6031207C45EB9031207C48FB930
:10179300031207C449BA031207C4AFBA031207C43A
:1017A300E6B3031207C472B5031207C4E8B5031204
:1017B30007C41EB6031207C4A8B6031207C4FBB6B8
:1017C300031207C428B7031207C432C6031207C49F
:1017D30016C2031207C424C2031207C47BC6031232
:1017E30007C4C6C3031207C4D6C3031207C4E8C39E
:1017F300031207C430C4031207C48CBE031207C408
:1018030011BF031207C475BF031207C4F07F001290
:1018130007C4DEA5031207C4ECA5031207C466A61A
:10182300031207C43EA7031207C4C9A8031207C4BF
:1018330039C4031207C473C4031207C4E1FD0212BF
:1018430007C4E4FD021207C43BFE021207C47AFE7A
:10185300021207C454FF021207C4388D031207C4CF
:101863008D8D031207C4898F031207C4BB8F031224
:1018730007C4DD8F031207C4F68F031207C40F904A
:10188300031207C41991031207C4B491031207C4C6
:1018930038BB031207C45DBB031207C46DBB03123D
:1018A30007C48CBB031207C4C4BB031207C4F9BB30
:1018B300031207C43BBC031207C44ABC031207C488
:1018C30054BC031207C46BAC031207C491AC0312DC
:1018D30007C4C3AC031207C4D2AC031207C4F1ACF0
:1018E300031207C451AD031207C45AAD031207C450
:1018F300B9AD031207C4DDAD031207C47FAE0312F3
:1019030007C48CAE031207C49DAE031207C47DC582
:10191300031207C49AC5031207C448A2031207C4DB
:10192300A2A3031207C4AFA3031207C4C2A30312E3
:1019330007C4E1A3031207C4F7A3031207C40BA44C
:10194300031207C46EA4031207C4B1A4031207C48D
:1019530061A5031207C4BFA5031207C4CFA50312D1
:1019630007C449C3031207C46DC3031207C49AC350
:10197300031207C4B0C3031207C4C3AE031207C4E0
:10198300EAAE031207C40BAF031207C470AF03120E
:1019930007C422B1031207C43BB1031207C452B1F7
:1019A300031207C45BB1031207C479B1031207C45E
:1019B30083B1031207C48DB1031207C4A0B103128C
:1019C30007C402B2031207C43BB2031207C45EB2D8
:1019D300031207C4A3B2031207C4CAB2031207C493
:1019E300E5B2031207C4EFB2031207C416B303121E
:1019F30007C45CB3031207C4CAC2031207C4E6C216
:101A0300031207C44CC6031207C4CFF4021207C45F
:101A1300FBF4021207C417F5021207C42AF50212D7
:101A230007C440F5021207C4ABF5021207C4E5F57B
:101A3300021207C4F8F9021207C415FB021207C405
:101A430049FB021207C48EFB021207C4E1FC021217
:101A530007C409FD021207C41EFD021207C42EFDAE
:101A6300021207C461FD021207C4B6FD021207C4C5
:101A7300C6FD021207C45EBC031207C46DBC031289
:101A830007C491BC031207C4B1BC031207C4D1BC81
:101A9300031207C4EFBC031207C407BD031207C434
:101AA30035BD031207C44FBD031207C4B2C50312E9
:101AB30007C42EA9031207C435A9031207C41FAA1A
:101AC300031207C44FAA031207C475AA031207C45B
:101AD30098AA031207C4BAAA031207C4E5AA0312F9
:101AE30007C43EAB031207C477AB031207C4C3ABEF
:101AF300031207C4F0AB031207C410AC031207C4EC
:101B030080BD031207C498BD031207C486BE031227
:101B130007C489BE031207C4E0FE011207C452FFC3
:101B2300011207C490FF011207C4D1FF011207C4B9
:101B33008EBF031207C4EABF031207C427C00312F0
:101B430007C4FD9A031207C41C9B031207C46B9BB3
:101B5300031207C4879B031207C4B89B031207C46D
:101B6300C59B031207C4D29B031207C4BE9C031276
:101B730007C4FC9C031207C40C9E031207C4179EE0
:101B8300031207C4299E031207C4329E031207C41B
:101B93003C9E031207C4F391031207C41396031266
:101BA30007C42196031207C4E5C5031207C476D7F9
:101BB300021207C421D5021207C4C1D4021207C4FA
:101BC30079D4021207C4EBD3021207C4DED3021284
:101BD30007C4D8D0021207C43ACE021207C403CDF9
:101BE300021207C457CC021207C49DCA021207C4CB
:101BF3004DC8021207C4D4C7021207C47BC702121E
:101C030007C40BC7021207C4E2C6021207C4D3C437
:101C1300021207C491C4021207C475C4021207C496
:101C2300C1C3021207C479C3021207C42F230012CF
:101C330007C4A522001207C44422001207C4F221DC
:101C4300001207C4E021001207C4C4C1021207C472
:101C530044C1021207C441C1021207C4A4DA02122A
:101C630007C45CC0021207C42AC0021207C467BFBC
:101C7300021207C492BD021207C486DA021207C415
:101C8300417D001207C44BBD021207C41DBD0212E1
:101C930007C41ABD021207C407BD021207C4C7BC9A
:101CA300021207C4B6BC021207C4CDBB021207C49A
:101CB30063BB021207C415BB021207C4DDB70212CD
:101CC30007C49DB7021207C4B9B6021207C48CB683
:101CD300021207C4CFB5021207C466D9021207C4A1
:101CE3009FB5021207C494FE0100000080FB32324C
:101CF30032E4738F0001000D0B870001000C0B24ED
:101D03000002007D11250002007F112600020081E0
:101D13001127000200831128000100851129000109
:101D2300008611840004008711860001008B112AAC
:101D33000001008C112B0001008D112C000100907B
:101D4300112D000800F80A2E00010091112F000147
:101D530000921130000100931131000100941132FF
:101D6300000100000B33000100010B34000100955A
:101D73001136000100020B380001009611390001F1
:101D8300008F1183000200A011630001000B0B649C
:101D9300000100F50A650001008E116D0001009F2E
:101DA300116E000200F60A4300010097114400027D
:101DB300009811450001009A11460002009B11474B
:101DC300000800030B480001009D114B0001009E19
:101DD3001104000100A211A1000100A511370001A7
:101DE30000A41188000100A31100000000000000FE
:101DF3000136360101000102010001030100010463
:101E030001060605020000070100340801000F095E
:101E13000401010D0100FF0E080000170200001964
:101E23000100FF1A0100011B0100FE1C0100081D37
:101E33000200001F01000120010001210200002314
:101E430001000F24020000260100012701000828D9
:101E53000200FF2A0100072B0102402C0100002D84
:101E63000100012E0100012F0100FF30010B1C3185
:101E73000800003A0100083B01000F2F0100000396
:101E830002710230016002110270020102020202B9
:101E9300028002100261023A00410063027302727F
:101EA300026202430200021302380000020002042D
:101EB30002120200020002000200020402040237BE
:101EC3000037003C024402000239000002000265B0
:101ED300020002350281020002050282028302002F
:101EE3000203007100300160001100700031022014
:101EF30003500480001000610000001400630073AD
:101F0300007200620043000000130006000000009E
:101F130000040012000000000000000000040004A0
:101F230000370037003C02440000000000000000BE
:101F330000650000003500810000000500000083FB
:101F4300000000030471040204600411047004021D
:101F53000402040104020410046104000414046371
:101F630004730472046204430400041304060400AB
:101F730004000404041204000400040004000451D7
:101F8300046400000400040004440400040004008A
:101F9300040004650400043504810464000504009E
:101FA300048304000401037103010301030103011A
:101FB30003010322030203010310030003000300D0
:101FC300030003000300030003420300032403068A
:101FD3000300030003040312032503230325032340
:101FE300030403040300030003000344030003008A
:101FF3000323030003650321003503810300030565
:102003000300030003000301017101010101011138
:102013000101013101010101018001100161013B55
:102023000014006301730172016201430100011393
:102033000106013D01350004011201000100010008
:1020430001000104010401330133013C0144013265
:102053000136000001000165010001350081010026
:102063000105018201830100013600010006000021
:10207300000F00000000000000000000000000034B
:10208300FFFF00000403FFFF0000FFFF0FF4010048
:1020930005C4040320000100130B0000000000002E
:1020A300000003010F00003A171300EC1601003A79
:1020B300170200C2160300C8160400CE160500D48A
:1020C300160600E016FFFF000001080D06380D0894
:1020D300320D0B440D10840C020E0D05260D071452
:1020E3000D0CEA0C0DFC0CFF000010114011161131
:1020F3001C113A112E11281146114C1152115E1167
:1021030022110A11041100160F00000B150B020017
:1021130002220F32000006FA110C121212DA101802
:1021230012D410E010140AE5D5C5B5A5A59585858B
:10213300756514100E104A1050104410FC0F541201
:10214300721278125A12661260120C0E020B040BF2
:102153000A0708000F303016181920231A1C1E30E6
:10216300303017181921301B1D1F300001191618A4
:1021730016161523030000034948424D1817250579
:102183000200383C3E363B3B352B432C48121E1293
:10219300241230122A12341158116C1264116A116C
:1021A300020402010101010902201026101A10562F
:1021B3001000BE040A2C103E101900E8037F000C27
:1021C30000280028210000000009030C0508080C62
:1021D3000A03080900040013FF1E1E1001C082C079
:1021E300838A828B83E0D2E7F0121626023355C02E
:1021F30082C08379001226AC125106C082C083903C
:102203000330124351D083D082C3E09CA3E09D509E
:102213000C125923FAA3E012222360010902335559
:10222300FBEA75F00BA4FAA8F075F00BEBA428FBFE
:10223300900332E02AF8A3E03B8882F583E0540F51
:102243002274F712036389081226AC122752ACF0EA
:1022530075F00BE9A42CF9900332E028FEA3E039D2
:10226300FF7401650860067402650870208A828B1A
:102273008312273E12355574026508701B1225FD23
:1022830012278570138E828F83E4F0800BEA240378
:10229300FCEB12272012272CEEFAEFFB121C440250
:1022A300338874F412036312625179008E828F8330
:1022B300E06076890A890B8065E50A75F00BA4FA5C
:1022C300A8F075F00BE50B1222307046E50A75F0A5
:1022D3000BA4F8AAF075F00BE50B1227648E828F1E
:1022E30083E085088285098312284685088285094B
:1022F30083A3123555EE2403FCEF1227291230670E
:10230300124CF1AA08AB09121C4479019003301254
:102313004700E50A2401F50AE50B3400F50B122604
:1023230005E50A9AE50B9B409002492E74F51203CA
:1023330063EAFEEBFF740B120A55123365750A014B
:10234300EC4D602BEC12626DED12510612354C7997
:1023530001121C38E5084509606F850882850983E9
:10236300A312625B7902AA08AB09121C38805AE5F2
:10237300084509602B12526E123A1B12306812275D
:102383006F700CEEFAEFFB121C32E9F50A80CBEE0C
:102393002403FA1226A770317903EEFAEFFB80CA01
:1023A3008E828F83A3E064FE7003A3E0F4700BEED0
:1023B30024030A0A0A1226A7700CEEFAEFFB121C7A
:1023C30032E9F50A8003750A00A90A7F030205CAE8
:1023D30074F71203639003301234BBEA4B602FEAA5
:1023E30075F00BA4FAA8F075F00BEBA428FBEAFE3A
:1023F300EBFF1213B09003321234BB900332124539
:10240300456012EEFCEFFD790012131A800790036A
:1024130032E4F0A3F0023388900330123CAFC3EEF2
:1024230098EF9922C082C083EC4D6005121B2A806D
:10243300097C087D00790012131A02335574F612D1
:1024430003637900EA4B6018780088081255A6EBFD
:1024530012591F60047901780808E8C3940840EA18
:10246300022E2874F712036374F31208A3ECFEED33
:10247300FF851882851983E4F004120A55EAF0A354
:10248300EB124A7A7403120A55AC82AD83EEFAEF6B
:10249300FB120A68EEFAEFFB120A6E02338374F73B
:1024A30012036374F31208A3ECFEEDFF8518828513
:1024B3001983E4F0EAFCEBFD7403120A5512283F7A
:1024C3007401120A551235488E828F831235557462
:1024D300FE68700374FF6960047901800279000269
:1024E300338374F7120363EAFEEBFF122543701480
:1024F30012254E8E828F83E0F4F88A828B83E05814
:10250300F0121C44A90802338874F7120363EAFE2D
:10251300EBFF7508008E828F83E0602212254370E3
:102523001D12254E8A828B83E08F838E82F8E058BA
:10253300700CE0F88A828B83E048F0121C4480C45C
:10254300121C3EE9F508740165082212626612271F
:1025530056122698FAA3E039FB2274F41203638A15
:10256300088B097C007D001225FD12272C1226BD45
:102573001262587900850882850983A3E064FE709E
:1025830003A3E0F460717E007F008062EEFAEF1235
:1025930022236057EEFAEFFBEA75F00BA4FAA8F0DA
:1025A30075F00BEBA428FB900332E02AF50AA3E0B5
:1025B3003BF50B850882850983A31249C8850A82E6
:1025C300850B83A3E06A7003A3E06B701EE50A2406
:1025D30003FAE50B1226A8700AE50A2403FCE50BAF
:1025E3001227291226B17901125275122F8A122647
:1025F30005EE9AEF9B409502492EEA24030A0A0A44
:10260300EB22900330124E57C32274F31203638AF2
:10261300088B098A828B83A312625B1226AC126237
:1026230058750C001225FD1226A870547E007F00F9
:10263300804912268AFAA3E0398A82F583E0540F8F
:10264300603612268AF50AA3E039F50BE50A24035E
:10265300FCE50B1227333400FB121B24E9640170E1
:1026630017850A82850B83A3124F18A312355512BF
:1026730026B1750C01125275122F8A12241B40B217
:10268300A90C7F050205CAEEF8EFF9E875F00BA473
:10269300F812269822AAF075F00BE9A42AF9900300
:1026A30032E02822EF12277F2212626CEB221226DD
:1026B300BD123071EEF0A3EFF022E50812626DE572
:1026C300092274F5120363EAFEEBFF8E828F83A364
:1026D30012625B7C007D00EE24030A0A0AEF1227D4
:1026E3002CEEFAEFFB121C3EE9F50A7401650A7041
:1026F30029126266122752AAF075F00BE9122764B9
:10270300850882F58312273E12276F700DE5082492
:1027130003FCE50912272012272C0223CC3400FDE9
:10272300EE2403FAEF221227333400FB120A682245
:102733003400FDE5082403FAE50922A31227432206
:1027430012274722E0F8A3E0F98E828F83A3221297
:102753002756223400F583123CB3E875F00BA4F836
:102763002212269EF508A3E039F50922E8F0A3E931
:10277300F0E5082403FAE50912277F22122785646E
:1027830001223400FB120A6EE92274F3120363740C
:10279300E61208A3126251750C0175080075090051
:1027A300750A00750B00851882851983E4F0EE2401
:1027B30003FCEF3400FD7403120A5512283FE96449
:1027C300017023740B120A5512354C7401120A5509
:1027D3001249CC7003A3E06960518518828519837F
:1027E300858208858309740D120A55E412284674FC
:1027F3000E120A55123555740D120A55AA82AB836F
:10280300120A8CE96401700B740D120A5585820A51
:1028130085830B780A1207FCAC08AD09EEFAEFFBCF
:10282300121C2C740212080FE9F50CEEFAEFFB12DE
:102833000A86A90C741A12080F022685122B30126D
:102843000A92221234B6123CAF22C082C0837800AF
:102853007900800312293D122605E89AE99B502945
:10286300E8FAE9FBEA75F00BA4FAACF075F00BEBB0
:10287300A42CFB900332E02AFCA3E03B8C82F5837B
:10288300E0540F70CF790080027901023355C08282
:10289300C0839021BC123D05EC75F012A4FCA8F096
:1028A30075F012EDA428FD79FF7AE07B0B12131A61
:1028B30002335574F7120363E9FEEAFF7A007B00E3
:1028C300780079008028E8FCE9FDEC75F012A4FC9F
:1028D30085F00875F012EDA42508122D70C39E40F3
:1028E3000AE0FCEFC39C4003122E5F12293D122D18
:1028F3006440D3023388C082C083780079008003A8
:1029030012293D122931501F122D74F470F2E8750B
:10291300F012A4F8AAF075F012E9A42AF974E028D9
:10292300FA740B39FB80047A007B00023355902143
:10293300BC122E2DC3E89AE99B22E8240108E9344E
:1029430000F92274F012036374F31208A38A0A8B4A
:102953000B8C0C8D0D8908EC450D6016AA0CAB0D84
:10296300120AE08A0E8B0FAE0EAF0FEE4F6003021A
:102973002A04120AB68A0E8B0FA80EA90FE8FEE9E5
:10298300FFE849607C9021C8122A846022740365A1
:102993000860067404650870167A047903120AB095
:1029A3009021C8122A9B40077A007B00022A81905B
:1029B30021CA122A84601B740165086006740265CB
:1029C30008700F7A027901120AB09021CA122A9B69
:1029D30050D68518828519837401F0120A55124C5A
:1029E300F1AC0CAD0D7403120A55122B29740B12A2
:1029F3000A5512335C123908E4124CD9120F548071
:102A030004EE4F6068780074FF2508C394045002F5
:102A130078048E828F83124CF18E828F83A3A3A3BB
:102A2300A3E508F0E88E828F83A3A3A3A3A3124C8C
:102A3300F9120212E88E828F83A3A3A3A3A3A3A3F5
:102A4300A31236EC74011236ECA3F0EE24101251EB
:102A530003E4F0A31231C5A3F0123067E4F09080D1
:102A630063120A32EE240C125103120A3E122A890F
:102A7300400590114BE4F0120E2EEEFAEFFB023CF0
:102A8300B9124E0D49227A047900120AB09021BC82
:102A9300125919EA98EB9922122AB4758321758287
:102AA300BCE493C398F8A3E49399F9C3EA98EB9928
:102AB30022E493F8740193F92274F212036374F31A
:102AC3001208A38A088B09ECFEEDFF750A00EEFAE3
:102AD300EFFB120AE08A0C8B0DA80CA90DE84960E4
:102AE3003E88828983E065087004A3E06509602F4E
:102AF30088828983A3A3A3A3E0C394055021125121
:102B03001C8518828519837401F0120A551251200D
:102B1300EEFCEFFD7403120A55122B29750A01A965
:102B23000A740D0247B7122B30120A9E22AA82ABF7
:102B330083120A68851882851983AA82AB8322745B
:102B4300F6120363122B7E600FA3A3A3A3E014C3A7
:102B530094045004790180027900022E2874F6123D
:102B63000363122B7E600FA3A3A3A3E014C39402F9
:102B73005004790180027900022E28120ADA8A822F
:102B83008B83E58245832274F6120363122B7E60E6
:102B93000BA3A3A3A3E07004790180027900022EA2
:102BA30028C082C083EAFCEBFD7A007B000233522B
:102BB300C082C0837C007D0002335274F41203632D
:102BC30074F31208A3EAFEEBFF8C0A8D0BC3EC949B
:102BD300F8ED94FF4007EE4F7003022C7775080061
:102BE300750900802E8518828519837401F0122FD0
:102BF300B2120A55122FC060137403120A55AC8225
:102C0300AD83EEFAEFFB121B24E97049E5082401BA
:102C1300122E109021BCE4125B8DE50898E509990A
:102C23005052E50875F012A4F8AAF075F012E50900
:102C3300A42AF912593860D4EE4F70A974FF650ABB
:102C4300700474FF650B60C4122FA2650A7004A39D
:102C5300E0650B70B7E50875F012A4F508A8F075E8
:102C6300F012E509A428F50974E02508FA740B3578
:102C730009FB80047A007B0002492974F412036380
:102C830074F31208A3750800120AE08A0A8B0BAECC
:102C93000AAF0BEE4F602A851882851983740112DF
:102CA30034B0F8A3E0F9740B120A551235D0120AA6
:102CB300807C127D0079FFEEFAEFFB12131A750880
:102CC30001122A89500990114B7401F0120E2EA99A
:102CD3000802492974F7120363E9FE74FE6A70035C
:102CE30074FF6B780079007005805212293D122D14
:102CF30064504AE8FCE9FDEC75F012A4FCAFF075F2
:102D0300F012EDA42F122D70F460E0E8FCE9FDEC65
:102D130075F012A4FC75F012EDA42FFD74E02CF5F0
:102D230082740B3DF583E06A7003A3E06B70BC8093
:102D330009122D7414C39404401712293D1229312A
:102D43005018EE70EC122D7464016005E06403709A
:102D5300E9122F93FAA3E0FB80047AFE7BFF023390
:102D6300889021BC123D09C3E89CE99D22122E9450
:102D730022E8FAE9FBEA75F012A4FAACF075F01256
:102D8300EBA42CFB74E42AF582740B3BF583E0225D
:102D9300120AF2023355C082C083790180F274F0C3
:102DA3001203638A0A8B0B7A047901120AB08A0C24
:102DB3008B0DEA450D603EEAC333FAEB33FB121386
:102DC300B08A088B09AE08AF09EE4F60237AFE7B09
:102DD300FF120AF874FE6A700374FF6B601B8508A8
:102DE300828509831234BBE5082402122E1080E188
:102DF300750C0080047E007F00850A82850B83E5C5
:102E03000CF0EEFAEFFB023CBEE5082407F508E5FB
:102E1300093400F509229021BC123D09C3EA9CEB59
:102E23009D2212080F7F020205CAE493FA740193EC
:102E3300FB22C082C0837A007B00800419122E5FBC
:102E4300122E195010122E7EC3940550F0E970EC27
:102E5300122E6880047A007B00023355EA24010AAB
:102E6300EB3400FB22EA75F012A4FA75F012EBA41E
:102E730028FB74E02AFA740B3BFB22EAFCEBFDEC23
:102E830075F012A4FCA8F075F012EDA428122E948C
:102E930022FD74E42CF582740B3DF583E02274F774
:102EA30012036374F31208A37E007F00022F46E52A
:102EB3000875F017A4F8A9F0125BA0FAA3E0FBEEE3
:102EC300F8EFF9E875F012A4F8ACF075F012E9A484
:102ED3002C122FA16A7003A3E06B603FE50875F025
:102EE30017A4F8AAF0EA125B9FF8A3E0F9740112A1
:102EF3000A55E0687003A3E0696020E50875F017E0
:102F0300A4F8EAF974A428FC740D39FD7403120AB9
:102F130055AA82AB83121B24E96014E50875F017E8
:102F2300A4F8A9F074A228FA740D39FB120F6005F6
:102F3300089021DEE493F8E508C3985003022EB20B
:102F4300122F8A9021BC125EE65039EEF8EFF91287
:102F53002F93F47003A3E0F460E685188285198348
:102F63007401F0EEF8EFF9E875F012A4F875F012B9
:102F7300E9A42AF9122FB2120A55122FC060C175A3
:102F8300080080AD023383EE24010EEF3400FF22EC
:102F9300E875F012A4F8AAF075F012E9A42AF91260
:102FA3002FA62274E028F582740B39F583E022748E
:102FB300E228F582740B39123CAD740B22E8F0A3BE
:102FC300E91235D8120A98E922C082C083900339E6
:102FD3007420F0A3740DF090033B741AF0A3740DE6
:102FE300F090033F7470F0A3740BF002335574F741
:102FF300120363EAFEEBFF900370E06408601BE0DA
:10300300640460168E828F83E05403640170481257
:103013003067123A00E06406703D8E828F83A3A36B
:10302300E064FE7003A3E0F4602D8E828F83A3A37C
:10303300123548900361E0687003A3E069700BEEFA
:103043002415F582EF12591F6008120DCEE9F50819
:103053008008120DD480F67508C2EEFAEFFB121346
:10306300B6022507EE12306C22240BF582EF3400F2
:10307300F5832274F41203638A088B098A828B8393
:10308300E0F8A3E0FAE82AFAE43400FB1213B08A6A
:103093000A8B0BAE0AAF0BEE4F6060850882850981
:1030A30083E0FC7D00790012131A8E828F83A3A321
:1030B30012625B120E108E828F83A3A3A3A312341A
:1030C300BB850882850983E0F8EE28F8EF34001207
:1030D3003550850882850983A3E0C0E0125100D0F2
:1030E300E0F0120E22EE240E125103E912491FE002
:1030F300C0E0EE2411125103D0E0F0EEFAEFFB0230
:10310300492E74F612036374EB1208A3EAFEEBFF75
:1031130012454260030231A97A077B001213B09073
:1031230003351234BB12454260788E828F83120AB4
:1031330032900336123A03120A3E12611FC0E012A4
:1031430031B5D0E0F0EE2405FAEF3400FB8A088BAA
:10315300098A82F583E0C0E01231B0D0E01231C5B4
:10316300E0C0E01231B0A3D0E012352F120A32854D
:103173001882851983120A3E88828983E0C0E0742D
:1031830005120A55D0E0F0850882850983E0C0E086
:103193007404120A55D0E0F07407120A551232EF84
:1031A30080067910800279017415022E251231B53B
:1031B300A322900335E0FAA3E0F5838A82A3A3A3B5
:1031C300A32212391022C082C083124542600D909F
:1031D3000335124E45900335E4F0A3F0120D3E1271
:1031E3000F0002335574F012036374EB1208A3EC5F
:1031F300FEEDFF89087425120A55780C1209F8743C
:1032030029120A55E0F9742A120A55E0FC742B12AC
:103213000A55E0FD740F697005740F6C601290110C
:1032230094E06402700579C10232EAE9C39C40F676
:10323300900371780C120A16E508900377F0E99071
:103243000375F0ECA3F0ED900378F074FF6A70035C
:1032530074FF6B701D9011A0E0F47003A3E0F47091
:1032630005121326800C9011A012336DE8F0A3E928
:10327300800790036EEAF0A3EBF0EE4F6017EEFACF
:10328300EFFB120FC0E96401700BEEFCEFFD7A82D5
:103293007B03121B2A900361E4F0A3F0900364F014
:1032A300A3F0900381F0901194E0640270089003FE
:1032B30075740FF0A3F09003707405F014120A559F
:1032C300E4F0900371120A32851882851983120A79
:1032D3003E900377E0C0E07405120A55D0E0F07425
:1032E30007120A551232EF7415023CBBE41235D8AB
:1032F300121B6622C082C083900334E0700312164F
:10330300E6120B3A804CC082C083900334E09011E4
:103313004A7004E4F0802D7401F0900334E0F4600B
:10332300237C41E0C394415002E0FCECF8E0C398F5
:10333300F0EC75F0E8A4CCA8F075F003A428FD7AAE
:1033430080123D117A4A7B117941121B548003127A
:103353000AE6D083D0820207C112336022122747C4
:10336300A322E0F508A3E0F50922123CAF90036E17
:103373002274F7120363EB900378F0120D2C80058F
:10338300740D12080F7F010205CA74F712036374E8
:10339300E91208A3EAFEEBFF7508008E828F83A370
:1033A300A3A3E0C0E07406120A55D0E01234B0C003
:1033B300E07408120A55D0E0F07409120A5574013A
:1033C30012352AF8A3E0F9E849600D8E828F831243
:1033D30049C8120A6EE970467407120A55E4F012DE
:1033E3000E0A7404120A551234BB900370E064048D
:1033F300700E120E167402120A55EAF0A3EB800B3C
:103403007402120A5574FDF0A374FFF07402120AD9
:1034130055AA82AB83120E4CE9F5080234A985182C
:1034230082851983AC82AD838E828F831249C81241
:103433000A7A8E828F83A3A3A3A3E0702474071256
:103443000A5574011234C17402120A551235558E8D
:10345300828F831235487404120A55E8F0A3E98079
:10346300AA123542740A120A551235557414120AF7
:1034730055740112579CE0C0E07415120A55D0E050
:10348300F07416120A55E412352AFCA3E0FD740CFD
:10349300120A55AA82AB83121B2A740A120A55AA6E
:1034A30082AB8312160EA90874170233851234B641
:1034B300A3E02212352FA322EAF0A3EBF022123568
:1034C30035F8A3E0F92274F712036374F81208A322
:1034D300EAFEEBFF7900900370E0640870448518FE
:1034E3008285198374FDF0A374FFF0120E0A74022F
:1034F300120A551234BB7405120A55E41234B6E0AD
:10350300C0E07404120A55D0E012352AC0E07406F4
:10351300120A55D0E0F07407120A55E41235D4129A
:103523000E4C740802338512352FE022F08E828F01
:10353300832212353AE022F0851882851983228589
:103543001882851983123CAF22E0F8A3E0F9EE124A
:10355300306CE8F0A3E9F022C082C0839003427488
:10356300CAF0A3740BF09003E874A6F0A3740EF0F2
:103573009003467400F0A3740CF090034874CAF0EF
:10358300A3740BF090034A7406F0A3740CF0023397
:103593005574F412036374F91208A38A088B098C17
:1035A3000A8D0B8518828519837808120A1674040C
:1035B300120A55E9F07405120A55E4F07406120A6A
:1035C30055E41235D4120B22740702492BE8F0A3F9
:1035D300E91235D82212353AAA82AB832274F41247
:1035E30003638A088B098A828B83125278EE4F70A9
:1035F300030236E990030E12454560158A828B83D8
:10360300A3A3E0F9EEFAEFFB90030F123A03121CA7
:10361300F48E828F83A3A3A3A3A3A3A3A3A3E06492
:103623000270718E828F83A3A3A3A3A3A3E054028A
:1036330070030236BB850882850983A3A3E064E98E
:1036430060768E828F83A3A3A3A3A3A3A3A3A3A321
:10365300E07014901197E0048E828F83A3A3A3A339
:10366300A3A3A3A3A3A3F08E828F83A3A3A3A3A344
:10367300A3A3A3A3A3E0141236EC7404F09011984F
:10368300124CCBE8F0A3E9125D838B0BEA450B7078
:103693000312576A8E828F83A3A3A3A3A3A3A3A317
:1036A300A3E0640260128E828F83A3A3A3A3A3A3C8
:1036B300A3A3A3E06406702E8E828F83A3A3A3A388
:1036C300A3A3E0A2E0501F850882850983A3A3E09A
:1036D300F9EEFAEFFB121C148E828F83A3A3A3A32C
:1036E300A3A3E054FEF002492E123910A3A3A32290
:1036F30074EC12036374DD1208A3EAFEEBFF8C087B
:103703008D097437120A55780C1209F8750A00747A
:1037130005120A55AC82AD83121BB47412120A55FA
:10372300E070087415120A55E060207405120A55FA
:10373300E0A2E6501E8E828F83A3A3A3A3A3A3A319
:10374300A3A31249C8120E82E960087903121B125F
:103753000238F67405120A55E0540C6404700575BA
:103763000B018003750B00E0A2E55019750A01E512
:103773000BA2E040101262621249C4121C20E960DD
:1037830004790480C87405120A55E0A2E650227435
:1037930006120A55E0540370187405120A55E054D2
:1037A3000C640C600CE0540C640860057510018017
:1037B300037510007405120A55E05403F874026887
:1037C300700C1262621249C4121CDA0238F67401D8
:1037D30068703AE510A2E050031238FE7405120A2D
:1037E30055A882A9837403120A55E8F0A3E9123C91
:1037F300A3851882851983123908E0C0E074021288
:103803000A55D0E01235D4121CC80238F6E860031A
:103813000238F6900358E0640170108E828F83A300
:10382300A3A3A3A3A3E070030237847422120A554F
:103833007402123CA3741A120A55123555E510A2EC
:10384300E050087405120A551238FEE50BA2E05049
:103853006AEE240FF582EF12591FC0E07417120AA3
:1038630055D0E0F090031012454570030238F6126C
:103873000E108A128B13A812A913741A120A55E098
:10388300687003A3E069706B780C1207F4780A126E
:10389300080078081207FCA910740C120A55AC82B0
:1038A300AD837421120A55AA82AB83900310123A96
:1038B30000121CF4740712080F8038780C1207F4F6
:1038C300780A12080078081207FC90036E12069912
:1038D300EE2412F582EF12565D7423120A55AC8260
:1038E300AD83740E120A55AA82AB83121C0E74099F
:1038F30012080F742312080F025D4E126262124EF9
:1039030053121BAE22E8F0A3E9123910221257A07A
:10391300A3A3A32274F71203631215DE0233887480
:10392300F71203631215E402338874F71203631268
:1039330015F0023388C082C0831215EA023355742E
:10394300F71203631215F602338874F712036374D4
:1039530009120A55E0F508780812080012160274D5
:1039630001023385C082C08312160E023355C08212
:10397300C08312161402335574F712036312161A16
:1039830002338874F7120363EAFEEBFF89087401BC
:10399300650870147900120C429021DCE493FC79E1
:1039A30000EEFAEFFB120BB802338874F4120363D0
:1039B30074F91208A3E9FE8A088B098C0A8D0B742B
:1039C30013120A551249C8900A651245456027EE3D
:1039D300851882851983F07401120A557808120A32
:1039E30016EAF8EBF97405120A551235D0900A65F8
:1039F300123A00121CF40235CBFB900344E0F8A307
:103A0300E0F583888222C082C08312164A023355AE
:103A1300123CB38882898322123CAFEE2212592BC7
:103A2300692274F6120363120CBA7A007B008025B4
:103A3300EAF8EBF9E875F006A4F8ACF075F006E9DE
:103A4300A42C124E2C12612DA3E4124F22F0A312C8
:103A530061331262AA9021C2122A9340D37A007B67
:103A630000801C8A088B09740378081209451248E0
:103A7300E6A374FEF0A304124D0BA3E41262AA9012
:103A830021D0123AC440DC7A007B00801D8A088B67
:103A9300097403780812094574CA1255A7741012E1
:103AA3005DE574FEF0A3041262AA9021D6123AC413
:103AB30040DB9021DFE49390034CF0123ACE022EC8
:103AC30028E493F8C3EA98EB9400227CE87D037A18
:103AD300107B009003BBE0F912146A2274F0120306
:103AE3006374F51208A38A088B09890A8C0BE9A26F
:103AF300E050147508FC7509FFA2E15005D2E402F9
:103B03003BA1D2E3023BA11247A67003A3E0697075
:103B1300057900023C6EAC0A7902AA08AB09120CC3
:103B230096E960EDE50AF50C780C12080079027C41
:103B3300FE7DFFAA08AB0912452112080FE96003B5
:103B4300023C6CE50AC2E5F50A9003AEE07051E56C
:103B53000AA2E6404B7403120A55AC82AD83AA084D
:103B6300AB09120A74E97032123E428A0C8B0DA81B
:103B73000CA90DE8FEE9FFE8496025EE24020A0AD4
:103B8300EF122785601AEE2402FCEF3400FD740364
:103B9300120A55AA82AB83121B2AE50AD2E5F50A5B
:103BA300900341E0F50C900361E0F50EA3E0F50FFF
:103BB300780E1207FC7D017C00900341E0F9AA0E08
:103BC300AB0F120C4E740212080FE9F8900341E098
:103BD30004F0E86003023C6CE50AA2E55004740EAD
:103BE30080027406C0E07401120A55D0E0125289B3
:103BF3008A0E8B0FAE0EAF0FEE4F6069123C8C1224
:103C03003CA3888289837401F07478550AA31262F5
:103C130072E50C126272A3E508F0E509123C7BE43D
:103C2300F0E50AA2E5500F7403120A55AC82AD8386
:103C3300E82406123C728E828F83A3A374FDF0A343
:103C430074FFF0E50B60159021DDE493F8E50BC3F9
:103C5300985009EE2413125103E50BF0EEFAEFFB33
:103C6300120B1680067910800279C7740B8049FA0B
:103C7300E93400FB121B2A2288828983A3A3A3A30E
:103C8300123C8722124FFBA322EE241712306E74CC
:103C930001F0120E0AEE241A12306EEAF0A3EB22A0
:103CA300F01262663400123CAD22F583123CB3225B
:103CB300E0F8A3E0F922740D12080F7F080205CA89
:103CC30074F61203637A007B10125777600890032F
:103CD300CD7401F08029900B02E06401901195707E
:103CE30006E0FC79018004E0FC79037A007B001292
:103CF3000BB89021BE123D057A007B10123D1302D2
:103D03002E28123D0922E493FC740193FD227B00CB
:103D13009003BBE0F91214642274EC1203638A0863
:103D23008B098C0C8D0D890E7414120A55124700E1
:103D33007416120A55E0F510A3E0F511120E82E98C
:103D430060077AFF7BFF023E3F901194E0640260BC
:103D530003023E327900AA08AB09120C9CA90E1289
:103D63000C908A128B13AE12AF13EE4F7003023E08
:103D73001A8E828F83A3A3A3A3A3E064018E828FF1
:103D830083A3A370691249C88E828F83A3A3A3A3BD
:103D9300A3A3E0541860439021DBE4938E828F83C6
:103DA300A3A3A3A3F0EA650C7003EB650D6014EA0B
:103DB300650A7003EB650B600AEA65107003EB6537
:103DC30011701F78101207FCAC0AAD0BAA0CAB0DD7
:103DD300120F7E740212080F80089003601257615D
:103DE300A3F074FE6A700374FF6B601D804EA3A37F
:103DF300A3E0640360298E828F83A3A3A3A3A3E01C
:103E0300640470057AFE023D478E828F83A3A3A3C9
:103E1300A3A3E0640270089003ADE0640270101283
:103E23003E428B0BEA450B6006AA08AB09800DAA3C
:103E330008AB09900342123A00121CF4025D4E9043
:103E4300036E124527120F422274F7120363EAFE30
:103E5300EBFF120AC8E9700AEEFAEFFB120AD4E983
:103E63006006EEFAEFFB80047AFE7BFF0233887470
:103E7300F01203638A0A8B0B8C0E8D0F8909750868
:103E830000120E82E979006003023FE9AA0AAB0B34
:103E9300120C9CA909120C908A0C8B0DAE0CAF0D61
:103EA300EE4F60198E828F83A3A3A3A3A3E06402C2
:103EB30070559003ADE064027003023FE7AA0AABBA
:103EC3000B900348123A00121CF4120ADA8A0C8B84
:103ED3000DA80CA90DE8497003023FE78882898386
:103EE300A3A3A3A3A3E0A2E04003023FE7750C0151
:103EF300A2E150687901AC0AAD0BAA0EAB0F120B0D
:103F0300E8E97064023FE78E828F83A3A3A3A3A390
:103F1300E064037005750C0280528E828F83A3A325
:103F2300A3A3A3E064016003023FE790036E12437F
:103F3300518E828F8312433D8A0C8B0DA80CA90DE1
:103F4300E84960D19021D4E493FA88828983E0C35D
:103F53009A50C2A3E06003023FE780B98882898355
:103F6300A3A3A3A3A3D2E1F0EE4F603A8E828F8383
:103F7300A3A3A3A3A3A3E05418602B7508018E8207
:103F83008F83A3A3120699750CFE750DFF780C128F
:103F930007FC7900AC0AAD0BAA0EAB0F120CAE7482
:103FA3000412080F803E900361E0650E7004A3E0E5
:103FB300650F70149021DCE493FCA909AA0AAB0BEA
:103FC300120BB8750801801CA90CAC0AAD0BAA0E24
:103FD300AB0F120BE8E9700C750801A909AA0AAB2B
:103FE3000B120C42A908023CBE74EA12036374F07C
:103FF3001208A38A0C8B0D8C088D097426120A559E
:10400300E0F514A3E0F5157512069003EE1245458D
:10401300602390036E124351AA08AB09120F6C8AF6
:10402300108B11EA4511600D8A828B83A3E0700522
:104033007900024325E50C241DF50EE50D3400F54A
:104043000F850E82124531F51388828983A3A3A3BA
:10405300E0FA88828983A3A3A3A3E0F9EA2400FEFC
:10406300E439FFAA08AB09120C48850E82850F8339
:1040730012436FE029F50BE50AA2E5500375120E12
:104083007487550A70177418550A6418600FE50C85
:104093002417F582E50D12591F6512600779011285
:1040A3001B12808C530A78C3EE94F8EF94FF501DD3
:1040B3007900EEFAEFFB12432F601288828983A303
:1040C300A3A3A3A3A3E05418600302403378081208
:1040D30007FC7D0012436212080FE9F8740368704D
:1040E30003024033E8600302419E7418550A7003CB
:1040F300024253E50AD2E0F50AA2E45004D2E1F504
:104103000AA90A1249C112432F605388828983A3E3
:10411300A3A3A3A3A3E05418604488828983A3A321
:10412300A3A3A3E064017036E5104511603090034A
:104133006E1243518882898312433D8A0E8B0FA8E6
:104143000EA90FE849601788828983A3E0600F8571
:104153001082851183A312547E5003024033E50A73
:10416300F50E780E12080012435512080FE9702B52
:104173007C007D0085148285158374FFF0A3F08590
:104183000C82850D83A3A3A3A3A3A3A3A3E060032E
:10419300124346A90B1249C11216088514828515CC
:1041A30083E0F47003A3E0F460399003ADE06402AC
:1041B30070030240331246F1E0FAA3E01239FC1215
:1041C3001CF4EA65087003EB65096003024033EEF3
:1041D300FAEF1239FC121CF4851482851583EAF078
:1041E300A3EBF078081207FC7D0112436212080F5B
:1041F300A90AEEFAEFFB120C9C8A088B09A808A9FE
:1042030009900361E0687003A3E069600302431649
:10421300EEFAEFFB120ADA8A088B09A808A909E863
:1042230049606E88828983A3A3A3A3E06401600D20
:1042330088828983A3A3A3A3E064027054851882B0
:10424300851983AC82AD83EEFAEFFB120A748055B5
:1042530090035AE0600FE50AF50E780E120800127B
:10426300435512080FE50AF50E780E12080079027D
:104273007CFE7DFFEEFAEFFB12452112080FE96089
:104283000302419E85148285158374FFF0A30241C6
:10429300E5120E0AEAFCEBFD851882851983AA82D2
:1042A300AB83121B2A850C82850D83A3A3A3A3A32F
:1042B300A3A3A3E06401700F1243467408120A55C6
:1042C300AA82AB83121B2A1244FB12510A4430F513
:1042D3000878081208007401120A5585820885833C
:1042E3000978081207FC740B120A55858208858326
:1042F3000978081207FCE513F50878081208007915
:1043030000EEFCEFFD1249C1120BE2740612080F16
:104313000240331244FB12510612436FE50BF012B5
:104323000E22741012080F7F0E0205CA120C908A17
:104333000E8B0FA80EA90FE84922A3A3124E571202
:104343000F6C22E50C2415F582E50D123071124C29
:10435300E5227901AC08AD09124E4C12452122AC7D
:104363000BA913124E4C120C4E740222125112A3BB
:10437300A3A3A32274F012036374F01208A38A0C9C
:104383008B0DECFAEDFB750F089003EE12454560BB
:10439300141254778A828B83E58245836007A3E0F6
:1043A30070030244F61244FB3400124531F50B88C6
:1043B300828983124504E0FBEC2400FEE43BFF8882
:1043C300828983A3A3124504A3A3E0FBECF508E4CD
:1043D3003BF50988828983A3A3A3A3A3A3A3E0F541
:1043E3000EE50AA2E45003750F10A2E55006740807
:1043F300250FF50F748F550A700FE50C2417F582FE
:10440300E50D12591F650F60087901121B12024452
:10441300F6530A707800E50AA2E450221244FB1214
:10442300591F2408FCA3E03400FD7408120A55AA9E
:1044330082AB83121B2A7808E50AC2E4F50AE50A6F
:10444300A2E550281244FB12591F28F8A3E03400B8
:10445300F9E82408FCE93400FD851882851983AA4C
:1044630082AB83121B2AE50AC2E5F50AAC0EA90B3F
:10447300EEFAEFFB120C54E9F874036860759003CD
:1044830061E06E7003A3E06F605EE87054E50AF5C7
:104493000F780F12080012451212080FE9705478B2
:1044A3000A1208007401120A5585820C85830D785F
:1044B3000C1207FC740B120A5585820C85830D7848
:1044C3000C1207FCE50BF50A780A120800A90EACDA
:1044D30008AD09EEFAEFFB120BE2740612080F8027
:1044E30012740468700D80B7780A1208001245121E
:1044F30012080F7410023CBBE50C241DF582E50D78
:1045030022A3A3A3E0FC88828983A3A3A3A3227984
:10451300011246F812307112452712452122120C5E
:104523000C740122E0FCA3E0FDAA08AB0922F58389
:10453300123A13A3E0F50A88828983A3A3E02290A9
:104543000335124EB32274E812036374F51208A301
:10455300EAFEEBFF8C088D0989147423120A55E0D7
:10456300F50F7424120A55E0F512A3E0F51374262F
:10457300120A55E0F516A3E0F5177428120A55E060
:10458300F50EA90F120C5A8A108B117401120A55D9
:104593007408F0E50EA2E450037410F0E50EA2E5F2
:1045A3005004E02408F0851882851983AA82AB831E
:1045B300120E6A8A0C8B0DEA450D70030246D8EA87
:1045C3002417F582EB1246EA120E0AE50C241AF5BB
:1045D30082E50D1251061234BB7403120A55AC82E4
:1045E300AD83AA10AB11120A74E9601D1246E2747E
:1045F30003120A55A882A983E50C2418F582E50D58
:10460300125106E8F0A3E98024E50EA2E4501FE569
:10461300106E7003E5116F70151246E2E50C241855
:10462300F582E50D125106E512F0A3E513F01246EB
:10463300F1124700850A82F5837402F0A3E50E1296
:104643004708E50FF0EE850A82850B83A3A3A3F049
:10465300EF850A82850B83A3A3A3A3124708A3A311
:10466300A3E508F0E509850A82850B83A3A3A3A329
:10467300A3A3F0AA10AB11120C48E92514850A82F2
:10468300850B83A3A3A3A3A3A3A3F0750800E50E3F
:10469300A2E45011AC12AD13E50A2408FAE50B129B
:1046A3003C74750808E50EA2E55014AC16AD17E589
:1046B3000A2508F8E50B3400F9E82408123C728552
:1046C3000C82850D83A3A3E510F0A3E511F0AA0CDA
:1046D300AB0D120B16740B12080F7F100205CAE5FF
:1046E3000C2416F582E50D1230717401F022124686
:1046F300F812307122E50C12626DE50D22E0F50A25
:10470300A3E0F50B22F0850A82850B83A3A3227411
:10471300F21203638A088B09ECFEEDFF890A790024
:104723001247A67003A3E069700479018073750BC7
:1047330001900361E065087004A3E06509601F75DB
:104743000B00780B120800A90AEEFCEFFDAA08ABD8
:1047530009120EBE740112080FE9F50B80417900AE
:10476300EEFAEFFB120C90EA4B602B8A828B83A349
:10477300A3A3A3A3A3E05418601C7508FE7509FF47
:1047830078081207FC8A828B83A3A312069912600E
:104793008212080F80097901EEFAEFFB120BA0A930
:1047A3000B8014120C9C8A0C8B0DA80CA90D900382
:1047B30061E0682212080F7F060205CA74F412032F
:1047C3006375081275090F7A10125D8A8B0BEA451F
:1047D3000B7003123ACE90034CE014F0700C90214E
:1047E300DFE49390034CF0120CA87E007F00806CF2
:1047F300850882850983A3A3A3A3E06059F46056C7
:10480300E5082404F582E50912575B70498508829F
:10481300850983A3A3A3A3A3E06403701979028585
:104823000882850983124351850882850983A3A3DE
:104833001249C8120BE8850882850983A3A3A3A3A1
:10484300A3E06401601085088285098374FEF0A3E8
:1048530004124918E4F0122F8A122E0C9021C4126C
:104863005EE6408C7E007F008039120DB08E088F8B
:104873000974037808120945748A2508FC741035F5
:1048830009FD7AF47B0B120D9EEA4B70DD8E088FC7
:1048930009740378081209451248E612612DE4F001
:1048A300122F8A9021D0E493F8C3EE98EF9400502E
:1048B3001B8E088F09740378081209451248EEE825
:1048C3002407F582E912575B70D680A17E007F0032
:1048D300800A1248F9600214F0122F8A125EE34034
:1048E300F180481248EE8882898322748A2508F869
:1048F30074103509F922EEF8EFF9E875F006A4F81B
:10490300AAF075F006E9A42AF9742A28F58274102E
:1049130039F583E02212491FA3A3A322F08508825D
:10492300850983A3A322740D12080F7F040205CA0D
:1049330074F712036374E11208A3ECFEEDFF75082C
:1049430000EE4F60728A828B83E0241C12578C1214
:10495300454560638A828B831249C885188285190D
:1049630083AC82AD83EA241BF582EB12565DEA2405
:104973001CF582EB1249C4120DF2740B120A551284
:1049830049CC7003A3E069702E7402120A55E064E7
:10499300017024741D120A55123A00E06401701765
:1049A300741D120A55123A02A3A3E0F88E828F8374
:1049B300E0687003750801A908741F023385124665
:1049C300F83400F583124E5722122743E06822740D
:1049D300F4120363E970247900900346123A00123B
:1049E3001CF48A0A8B0BAE0AAF0B74FE6E70037451
:1049F300FF6F701A9021D7E49360137901900346F7
:104A0300123A00121CF48A0A8B0BAE0AAF0B120E79
:104A13002E0230FE74F612036374F31208A312130A
:104A2300268A088B09AE08AF09900361E06E700314
:104A3300A3E06F60E9120E16EA6E7002EB6F60DEA0
:104A4300EEFAEFFB120E82E970D4EE4F60D08518B8
:104A530082851983E4F004120A55EEF0A3EF124A9B
:104A63007AE970BA74FE6E700374FF6F60B0EEFA89
:104A7300EFFB740D022E251235D8120A8C22C08248
:104A8300C083120E2E0233557F0A0205CA74F21236
:104A93000363EAFEEBFF8C0A8D0B8908740E120A7E
:104AA30055E0F50974FC6E700374FF6F70057900AF
:104AB3000247BA7900120C9C8A0C8B0DAE0CAF0D19
:104AC300900361E06E7003A3E06F7006E509A2E650
:104AD30050DCA909125F70706179007AFE7BFF12C6
:104AE3005F707056741855097003024BC7780079CC
:104AF30000800312293D9021C41229344003024B44
:104B0300C7E8FAE9FBEA75F007A4FAACF075F00719
:104B1300EBA42CFB74182AF582740F3BF583E05445
:104B23001870D0E875F007A4F8AAF075F007E9A4A7
:104B33002AF9741228F8740F39F988828983A3A398
:104B4300A3A3A3A3E05418600974185509700302C2
:104B53004AB188828983EEF0A3EFF074FE650A7090
:104B63000474FF650B6003124CEB88828983A3A353
:104B7300A3A3A3A3E509F0A2E0500D88828983A330
:104B8300A3A3A3A3A3D2E2F0740165088882898357
:104B9300A3A3A3A3A370387401124D0BE0541860B0
:104BA300289021DBE49388828983A3A3A3A3124CD7
:104BB300D9120F6C8B0DEA450D6003024AB17800E0
:104BC300790080397902024AB3900360E080D7E02C
:104BD30064017003024AB188828983A3A3A3A3A3B8
:104BE300A3E0541860079021DBE493800490035FF3
:104BF300E0123C7BE508F0024AB112293D9021DE28
:104C0300E493FAC3E89AE994004003024AB17A00B4
:104C13007B00804BEAFCEBFDEC75F007A4FCAEF0E7
:104C230075F007EDA42EFD74142CF582740F3DF579
:104C330083125278E8FCE9FDEC75F017A4FC85F0CB
:104C43000975F017EDA42509FD74A22CF582740DE6
:104C53003DF583E06E7003A3E06F609E122E5F90BC
:104C630021C4122E1C40AD123D05EC6A7002ED6B9F
:104C73007088E875F017A4F8AAF075F017E9A42A6C
:104C8300F974A228FE740D39FF7C177D007900EEBC
:104C9300FAEFFB12131A8E828F83124CF190036E7C
:104CA300124CCBA3A3A3A3A3A3E8F0A3E9124CD173
:104CB3007401F0EE240E1251037401124CF9120226
:104CC30012125100E8024BF9123360A3A322F0EE53
:104CD300240F12306E22F0124CE2AA0AAB0B229080
:104CE300036EE0FCA3E0FD2288828983A3A3E50A87
:104CF300F0A3E50BF022F09021D4E4932401F8E42F
:104D03003400F97A027B0022123C87A32274ED124D
:104D130003638A088B09890E124E35400579050213
:104D23004E0A121650AA08AB09124F079021C2125D
:104D33004E0D650A7003E9650B70077AFE7BFF125F
:104D43004F079021C2125912E50B994003024E08F6
:104D5300124E126012E50A75F006A4F875F006E526
:104D63000B124E5D1213B6E50E6018E50A75F006D8
:104D7300A4F8AAF075F006E50B124E89701A7901B2
:104D8300024E0AE50A75F006A4F8AAF075F006E5E6
:104D93000B124E6AE4F0A3F0E50A75F006A4F8AA34
:104DA300F075F006E50B124E2AA312512088828972
:104DB30083A3AA82AB83124E788A828B83E06041FD
:104DC300124E12603C8E108F11751200781012076C
:104DD300F8E50EC333FCE433FDE50A75F006A4F5EC
:104DE3000AA8F075F006E50BA428F50B742E250A26
:104DF300F5827410350B1249C612130E7403120890
:104E03000F790080027907025F86122AB4E822E54F
:104E13000A75F006A4F8AAF075F006E50B124E65C4
:104E2300F8A3E0F9E84922A42A124FBE88828983B5
:104E3300A322ECFEEDFF9021D2E493F8E9C398227C
:104E4300F583124E571213B622E50C12626DE50D6F
:104E53003400F583E0FAA3E0FB22124E65FAA3E0E7
:104E6300FB22124E6AE022A42AF9742E28F58274DA
:104E73001039F58322E50EF0901196124E8222E04E
:104E830088828983F022124FE2F50CE93400F50D94
:104E9300E50EC333FAE433FB1213B0850C82850DA0
:104EA30083EAF0A3EBF0850C82850D83124EB322C7
:104EB300123CB3E8492274F4120363ECFEEDFF7471
:104EC3000C120A5512354888088909124F07AC0A93
:104ED300AD0BECF8EDF99021C2124F0F5021E8759C
:104EE300F006A4F8AAF075F006E9124E2AE08E82C5
:104EF3008F83124F22124F18123555790080027991
:104F03000402492E120C1E8A0A8B0B22122E2DC369
:104F1300EC9AED9B22123CAF85088285098322120D
:104F23004FF72274F61203637E007F008028EEF8A9
:104F3300EFF9E875F006A4F8ACF075F006E9A42CD7
:104F4300F9742C28F5827410125B916A7003A3E044
:104F53006B6057122F8A125EE340D3125EDE70023B
:104F6300E96F704674FE6A700374FF6B703C7E00D9
:104F73007F008003122F8A125EE3502E1248F970CD
:104F8300F3EEF8EFF9E875F006A4F8124FB4124FF8
:104F9300E96017124FD0F8E9124FC88882124E43C6
:104FA300850882850983E4F0A3F0EEFAEFFB022E75
:104FB3002875F006E9124FBC22A42AF9742A28F8AE
:104FC300741039F9223400F98808890922EEF8EFC0
:104FD300F9E875F006A4F875F006E9124FE222121B
:104FE3004FBCE8240422A3A374FE124FF4124EB361
:104FF30022F0A304124FFB22F088828983A3A3A388
:10500300A32274F6120363EA241DF582EB12510AFC
:10501300F9604BEA241DF582EB12591F2402FCA30D
:10502300E03400FD124E3940030250F3780080292A
:105033008C828D83E0F508A3E0FFE5082400E43FBC
:10504300F509E833FEE433FF74722EF58274103FE2
:10505300F5831251201250F608E8C39940D28A8290
:105063008B83A3A3A3A3A3A3A3A3A312435190033B
:1050730061E06C7003A3E06D700F7C727D101226EB
:10508300AC1249C4120C128067EA2411F582EB12A8
:10509300591F605CFC74FF2CF07508017808120836
:1050A3000075087275091078081207FCE9F508788D
:1050B30008120800EA2412F582EB12591FF508784A
:1050C30008120800EA2415F582EB1251061206991C
:1050D300ECF91226AC12434E8A828B83A3A3A3A3BB
:1050E300A3A3A3A3A31249C8120C2A740712080F7F
:1050F300022E28EC24020C0CED3400FD22EE240DCC
:10510300F582EF12307122123071125112E022E057
:10511300F8A3E0F5838882A32288828983E508F0D7
:10512300A3E509F02274EA12036374FD1208A38A4B
:10513300148B158C0E8D0F890D7419120A5512528A
:1051430078741B120A55E0F511741C120A55E0F528
:105153000C741D120A55124700741F120A55E0F50C
:10516300106008E50CC333240480027402C0E074A9
:1051730001120A55D0E01252898A088B09EA4509BF
:1051830070030252698A828B83A3A3E514F0A3E51B
:1051930015125D79E50EF0A3E50FF0EA2413F5820D
:1051A300EB125106E50DF0EA2414F582EB125106D9
:1051B300E511F0EA2417F582EB12591F64017040E0
:1051C300120E108A0E8B0FA80EA90F85088285096F
:1051D30083A3A3A3A3E0687003A3E0696022EE4F57
:1051E3006011E508241AF582E509125106EEF0A3D1
:1051F300EF800CE5082417F582E509125106E4F067
:1052030012526E1252788E828F837405F0A3E510CA
:105213007004E50C80487401250C1252827A0080D8
:1052230028850A82850B83E012527E850A82850BCC
:1052330083A3E08E828F83F0E50A2402F50AE50B4F
:105243003400F50BA30EAF830AEAC3950C40D212C8
:105253000E10EA12527E120E10EB8E828F83F0AA8A
:1052630008AB09120B1674030243271226BD123032
:105273007122900330E0FEA3E0FF228E828F83F041
:10528300A3AE82AF83221235D8120E6A22C082C027
:1052930083E9C333FCE433FDEA2CFAEB3DFBEA2458
:1052A300FEF582EB34FF1249C602335574F2120342
:1052B3006389098A0A124E354004790080407508D3
:1052C3000080020508E508C39509502AE508C333A1
:1052D300F8E433F9EE28F582EF39F583C082C08311
:1052E300120E108A0C8B0DD083D082E0650C7004F3
:1052F300A3E0650D70CDE50A650870BE790102472C
:10530300BA74F012036374F31208A38A088B098C2E
:105313000A8D0B890C750D00120E82E9790060036A
:10532300025406AA08AB09120C9CA90C120C908A11
:105333000E8B0FAE0EAF0FEE4F70030254048E822E
:105343008F83A3A3A3A3A3A3E0A2E2400302540475
:10535300120E10EA650A7003EB650B7011780D12DB
:105363000800E4F50EF50F780E1207FC8044AA0A34
:10537300AB0B120ACEE96401706885188285198324
:105383007404F07401120A55124CF18518828519C0
:1053930083AA82AB83120A8CE964017045750D01FF
:1053A300780D120800E4F50EF50F780E1207FC7560
:1053B3000D00780D120800780D1208007408120A07
:1053C3005585820E85830F780E1207FC9021DDE44C
:1053D30093F9AC0AAD0BAA08AB09120C2A74071295
:1053E300080F8E828F83A3A3A3A3A3A3E0A2E1400C
:1053F3000D8E828F83A3A3A3A3A3A3C2E2F0750D93
:1054030001A90D023CB974F6120363E9FE79001297
:105413000C9CEEF9120C908A088B09A808A909E8DC
:105423004960061262B4F980027904022E2874F6E8
:105433001203637E07900355E070341254778A0891
:105443008B09A808A909E849602590035AE064017B
:1054530088828983A3A3700B12547E888289835028
:1054630001A3A3E0F9120F8AE9FEEE70027E07EEB4
:10547300F9022E28124CE2120F6C22E0FA8882897C
:1054830083A3E0C39A2274EE120363EAFEEBFF895F
:105493000A8C0C8D0B7412120A5512336512555374
:1054A300124E3C5051890E750F007403780E120989
:1054B300457490250EF5827410350FF583E0F8E5F9
:1054C3000CC398502DE50B602475110074037810FC
:1054D300120945748A2510F874103511F9888289E8
:1054E30083A3A3A3A3A3A3E50C12555DF079000244
:1054F3004A8B790380F979007AFE7BFF125553E4D6
:105503009365107004790280E6E50B60E0890E75FF
:105513000F007403780E120945748A250EF874106F
:10552300350FF988828983A3EEF0A3EF12555D123C
:105533004D0BE50C123C8374FF126133E50AF090C6
:10554300035FE088828983A3A3A3A3A3A3A3809C6F
:10555300120C8AE9F5109021D022126276A3E50895
:10556300F0A3E5092274F6120363ECFF120C8A9090
:1055730021D0124E3C50278908750900740378081E
:10558300120945748F1255A77410125DE5E0F8EF08
:10559300C3985006EFF079008006790380027904FE
:1055A300022E28EA2508F5822274F4120363EAFE28
:1055B300EBFF120C8AE9F50A9021D0124E3C5019E8
:1055C300750B007403780A120945748D250AF58258
:1055D3007410350B1249C680189003441245456078
:1055E3000CEEFAEFFB123A03121CF480047AFE7BF2
:1055F300FF02492E74F61203638A828B83A3A3A34B
:10560300A3A3E4F0F88001089021D6E493F9E8C35A
:1056130099501E88081256558C828D83A3A3A3A389
:10562300A3A3A3A3E06970DFECFAEDFB120DB68030
:105633001EE4936870198C828D83A3A3A3A3A3A3F1
:10564300A3A3A37406F07A008C828D831257800281
:105653002E2874122508F582741112592BF922741D
:10566300F4120363EAFEEBFF8E828F83A3A3E0149D
:10567300125797A3E0F9120D928A088B09EA45099C
:1056830070030257588E828F83A3A3E070358A82FA
:105693008B83A3A3A3A3A3A3A3A3A3E064028A82EC
:1056A3008B83A3A3A3A3A3A3A3A3A360107406F054
:1056B3007AF08508828B831257800257587406F05C
:1056C3000257588E828F83A3A3A3A3A3A3E060737F
:1056D3008E828F83A3A3A3A3E0607AEE2403F582D3
:1056E300EF12575B706F90034E125761125797E09A
:1056F30014125D70E06403705C8E828F83A3A3A396
:10570300A3E0700DAC08AD09EEFAEFFB120C60805C
:10571300448A828B83A3A3A3A3A3A3A3A3A37404F5
:10572300F0121326EA540F04850882850983A3A384
:10573300A3A3F0A3E4F07A20FB1257777017125754
:105743006A80128A828B83A3A3A3A3A3A3A3A3A385
:10575300E0640360AF02492E12592B14F022E08E4D
:10576300828F83A3A3A3227A207B009003BBE0F95B
:1057730012136822125D8C8B09EA450922E0240C7E
:1057830012578CE0F9120CD822F8A3E03400F98800
:105793008289832212579CA3221257A02212352FEB
:1057A300A3A3A32274F612036379007E0080258EDF
:1057B300087509007403780812094574CA2508FAA4
:1057C30074103509FB8A828B83A3A3E06005120C56
:1057D3006679010E9021D6E493F8EEC39840D0E9A0
:1057E300A2E07A407B009003BBE0F95015121476D7
:1057F3008B09EA4509700E7C647D007A40123AD425
:105803008003121470022E2874F4120363ECFEED6D
:10581300FF7508CA7509107C0080458508828509D3
:1058230083A3A3A3A3A3A3A3E0F8EA2412F582EB23
:1058330012591F68701F8508828509831235481223
:105843005923687003A3E069700B85088285098377
:10585300A3A3E070200CE5082408F8E509124FC85B
:105863009021D6E493F8ECC39840B0E4936C7005B0
:10587300790002492E850882850983A3A3A3A3A3E4
:10588300A3E07004790180EA125F7E120F428B0B52
:10589300EA450B600F850882850983A3A3A3A3A30D
:1058A300A3E014F07C0080010C8C0A9021BC1259F7
:1058B30012E4995020EC12593160ED122FA26E7050
:1058C30003A3E06F70E2850882850983A3A3A3A3E2
:1058D300A3A3E014F09021DEE493F89021BCE493B9
:1058E30028F8A3E4933400F9850882850983A3A3E8
:1058F300A3A3A3A3E0FAC3E89AE99400508685081A
:1059030082850983A3A3A3A3A3A3E4F00258871268
:105913005919E50A9822E4122AB5C32212592B22F7
:1059230012626CEB12592B223400F583E02275F0DE
:1059330012A4F8A9F074E428F582740B39F583E016
:10594300F42274EA120363EAFEEBFF8C148D1589CB
:10595300127CCA7D10750801750900750A00750B64
:10596300009021DEE493780812077D908063780C21
:105973001209F87A0080128C828D83A3A3E0601E43
:105983000AEC2408FCED3400FD9021D6E493F8EAF8
:10599300C39840E3E4936A70057900025B878C82C5
:1059A3008D83A3A3A3A3A3A3E4F0FA802E640160D1
:1059B30005E06403701D8E828F83A3A3A3A3A3A317
:1059C300A3A3A3E0F47003A3E0F47007780C7908B1
:1059D3001209910A7401780812077D8A10125B8AF2
:1059E300E51098E499504DEA75F012A4F8ABF0EB8A
:1059F300122FA165147004A3E0651560D6125D68CB
:105A0300900361E0687003A3E06960C7EA75F01270
:105A1300A4F8EBF974E428F582740B125B91640427
:105A23006003E070888C828D83A3A3A3A3A3A3E068
:105A330004F0809F7A008066EA75F017A4F8ABF053
:105A4300EB125B9F65147004A3E06515604F125B56
:105A5300A064FE7003A3E0F4604374AC28F5827481
:105A63000D39F58312336DE0687003A3E069702D7F
:105A7300EA75F017A4F8EBF974B028F582740D12E7
:105A83005B91601974B128F582740D125B91600DFE
:105A93008C828D83A3A3A3A3A3A3E004F00A902184
:105AA300DEE493F8EAC398408F8C828D83A3A3A38B
:105AB300A3A3A3E0F89021D5E493C398500DE493F6
:105AC3008C828D83A3A3A3A3A3A3F08C828D83A332
:105AD300A3A3A3A3A3E0600DEE2411F582EF125953
:105AE3001F6401700B8C828D83A3A3A3A3E4800D99
:105AF30090034FE0048C828D83A3A3A3A3F09003B0
:105B030054E08C828D83A3A3F090034E125B961214
:105B13003CA38C828D831235558C828D83A3A3A3E2
:105B2300A3A3E512F0EE2412125103125B96A3A372
:105B3300A3A3F0E50C450D450E450F60337A0080B5
:105B4300010A9021D6E493F8EAC39850238A0812F5
:105B53005BD412591F6004651270E6750900E512E3
:105B6300F074027808120945125D53780C120A1674
:105B73007A407B0012577770097C647D007A40126B
:105B83003AD4790102432A9021BC12591A2239F5D9
:105B930083E022E08C828D83A3A3A322F974A2283D
:105BA300F582740D39F583E02274F4120363750AE8
:105BB300008002050A9021D6E493F8E50AC39850C1
:105BC3000D850A08125BD4123A2070E7E4F002490B
:105BD3002E74122508F58274112274EC1203638A61
:105BE300108B118A828B83A3A31249C8120D98EAE2
:105BF3004B6003025CF2908063780C1209F875081D
:105C030001750900750A00750B009021DEE4937895
:105C13000812077DFE80080E7401780812077D8E36
:105C230012125B8AE51298E4995026EE12593160FC
:105C3300E6125D68851082851183A3A3E068700373
:105C4300A3E06970D285080C85090D850A0E850BC2
:105C53000F7E0080057A007B000E9021D6E493F836
:105C6300EEC3984003025CF28E08125BD412591FF4
:105C730060E775090074027808120945125D5385BF
:105C83000C08850D09850E0A850F0B780812096B20
:105C9300E5084509450A450B60BF8E0812565512A3
:105CA3000D92EA4B60AF8A828B83A3A3A3A3A3A322
:105CB300A3A3A3E06405709D850C08850D09850EDB
:105CC3000A850F0B78081209C88E12751300740227
:105CD3007812120945741B2512F58274113513F5D8
:105CE30083780812097E9021D6E493FE025C5CEA75
:105CF3004B60128A828B83A3A3A3A3A3A3A3A3A30F
:105D0300E06405601D851082851183A3A3A3A312FC
:105D13004351851082851183A3A31249C8121B9096
:105D23008029851082851183A3A3125D60E0FCA303
:105D3300E0F5838C82E8F0A3E9125D707401125DD3
:105D4300838B09EA4509700312576A7F0C0205CA5F
:105D5300741B2508F58274113509F58322123CAFB3
:105D63008A828B8322122FA6F8A3E0F922125D798F
:105D7300A3A3A3A3A322F08A828B83A3A3A3A32217
:105D8300F07A20125D8A227B009003BBE0F91214A3
:105D9300762274F6120363E9FC79008001099021ED
:105DA300D0124E3C503989087509007403780812E3
:105DB3000945748B1255A77410125DE5E06A7003F0
:105DC300A3E06B70D8890875090074037808120979
:105DD30045748A1255A77410125DE5E06C70BE021B
:105DE3002E283509F5832274F712036389085308B3
:105DF300407E007F008056EEF8EFF9E875F007A4C7
:105E0300F8ACF075F007E9A42CF9741228F5827444
:105E13000F125B916A7003A3E06B702E74FE6A70BD
:105E23000374FF6B7003025EBEEEF8EFF9E875F0E2
:105E330007A4F875F007E9A42CF9741828F58274FF
:105E43000F125B91544065086071122F8A9021C430
:105E5300125EE640A2125EDE7002E96F707674FE97
:105E63006A700374FF6B706C7E007F008003122FD7
:105E73008A9021C4125EE6505BEEF8EFF9E875F004
:105E830007A4F8AAF075F007E9A42AF9741628F50F
:105E930082740F125B9170D6A908EEFAEFFBEA75D4
:105EA300F007A4FAA8F075F007EBA428FB74122AF4
:105EB300F582740F3B1249C6120C42EE75F007A42B
:105EC300FEA8F075F007EFA428FF74122EFA740FE2
:105ED3003FFB80047A007B00023388124E0D6E2252
:105EE3009021C2125919EE98EF992274F2120363AA
:105EF3008A088B09890B8C0A7900120C9CA90A1257
:105F03005F70601988828983A3A3A3A3A3E0650BB1
:105F1300700B88828983A3A3125278800A74016567
:105F23000B7045AE08AF0974FE6E700374FF6F60AB
:105F330037125F7E120F6CEA4B60239003EE12451B
:105F430045600C8A828B83A3E060137900801B90E9
:105F530021D4E493F88A828B83E0C39840EDE5086B
:105F63006E7003E5096F70BB79010247BA120C909A
:105F73008A0C8B0DA80CA90DE84922124CE2EEFA0B
:105F8300EFFB227F0B0205CA74F4120363EAFEEBF4
:105F9300FFE9A2E6501B79FF121BC08B0BEA450BEE
:105FA3006009900361E0FAA3E080327AFE7BFF8010
:105FB3002D120ADA8A0A8B0BA80AA90BE849601A80
:105FC30088828983A3A3A3A3E0640160D58882891F
:105FD30083A3A3A3A3E0640260C8EEFAEFFB024924
:105FE3002E74F2120363890BEAFEEBFF8C088D0912
:105FF300740E120A55E0F50A7402650B703A7900C3
:10600300EEFAEFFB120C90EA4B60608A828B83A35B
:10601300A3A3A3A3A3E0541860517508FE7509FF59
:1060230078081207FC8A828B83A3A3120699126055
:106033008212080F790180307401650B7028AC0A55
:106043007901120C96E9601EE508450960B0EEFA85
:10605300EFFB120C1E9021C2122A9350A1850882D5
:106063008509837401F079000247BA9021DCE49337
:10607300FCA90AEEFAEFFB120BB8E970E980B579D7
:1060830000900361124CE58A828B83124E57120CE7
:10609300AE74042274F41203637C0079057A007BE6
:1060A30000120D8C8A088B0980677C007905EEFA53
:1060B300EFFB120D8C8A088B098E828F83A3A3A317
:1060C300A3124545604B12611F24FFF0A3E034FF88
:1060D30012613312454570398E828F83A3A3A3A324
:1060E300A3A3E0540460118E828F83A3A3A3A3A36D
:1060F300A3A3A3E0F9120C7E8E828F83A3A3A3A391
:10610300A3A3A3A3A37406F07AF08E828F831257FE
:1061130080AE08AF09EE4F709102492EEE2404F8C9
:10612300EF3400F988828983E022A374FEF0A3048C
:10613300F0888289832274EC1203638A108B11EC3A
:10614300FEEDFF7414120A55E0F50CA3E0F50D748F
:1061530016120A55124700E9600C750800780812F8
:106163000800790B80657900EEFAEFFB120C908A38
:10617300088B09EA4509605B8A828B83A3A3A3A3E7
:10618300A3A3E0A2E0504C78101207FCAC0CAD0DB9
:10619300AA0AAB0B120F7E740212080F8A0A8B0B2A
:1061A300A80AA90B74FE68700374FF69602585084B
:1061B30082850983A3A31235557508007808120850
:1061C30000790CAC10AD11EEFAEFFB120EBE7401A8
:1061D30012080F025D4E74F71203637812790F7C75
:1061E300007D00804388828983A3A3A3A3A3A3E0A4
:1061F300A2E0402E88828983A3A3E06A7003A3E010
:106203006B701F88828983A3A3A3A3A3E064017097
:106213001188828983A3A3A3A3A3740312627212B6
:10622300625B12624812623F9021C4E493FE7401E0
:1062330093FFC3EC9EED9F40AC023388E82407F83C
:10624300E93400F922EC24010CED3400FD22EAFECE
:10625300EBFF12626612307174FEF0A304F022ACFD
:1062630082AD83EE12626DEF22EA240BF5822212D5
:10627300627622F088828983A3A322C082C08378B6
:1062830012790F7A007B0080131262B488828983AB
:10629300A3A3A3A3A3A31262AA12623F9021C412D1
:1062A3002E1C40E5023355F0EA24010AEB3400FBCF
:1062B300228882898374FEF0A30412627614124F3B
:1062C300F4E4123C87F022C082C0837C057D037A0C
:1062D3001E7B0A121B2A120B100270EF74F51203B5
:1062E30063E9FF8A08EBFEEF705A74026508703D9C
:1062F3009011737408F0750A00780A120800ECF51F
:106303000A780A120800EEF50A780A1208009011BA
:106313008712069590118BE0F97C037D0B9011A0F9
:10632300126B8B120B2E740712080F801474016505
:106333000870119011737408F07B00EEFAF9120BD8
:1063430040E960107CE87D037A017B00900A32E02B
:10635300F91214647F030205CA74F41203638909F2
:1063630090049EE0FEA3E0800F8A828B83A3E5095D
:10637300F08E828F8312783DFFEE4F60528E828FB4
:1063830083A3A3126BA360E98E828F83A3A3A3E0ED
:10639300F5838882A3126BA3F5087AD1F91213440B
:1063A300EA4B70C57A027B0012132CEA4B700E7A0B
:1063B300107B00900A32E0F912136880B48A828B52
:1063C3008374D1F0A3E509F0A90812133880A2124F
:1063D3000E10900A14126B2E120E0A80007F040214
:1063E30005CA74F1120363890A8C08740F120A55E3
:1063F300126B5A7411120A55126AE8750900750E68
:1064030000804AE50B1264B2F50CA3E0F50DE50E2E
:10641300C333FEE433FFEA2EF582EB3FF583E065F9
:106423000C7004A3E0650D7019E509C333FEE43372
:10643300FFEC2EF582ED3FF583E50CF0A3E50DF0BF
:106443000509050BE50BC3950840B8050EE50EC31A
:10645300950A5005750B0080EBA909026BCA74F409
:10646300120363890B740C120A55126B5A750A00D6
:106473008002050AE50AC3950B502F7D0080010DAC
:10648300EDC39C50EDE50AC333FEE433FFEA2EF57A
:1064930082EB3F1264C2F509ED1264B26508700421
:1064A300A3E0650970D97901800279000263E0C332
:1064B30033FEE433FFE82EF582E93FF583E022F56E
:1064C30083E0F508A3E02274F612036312654F70AC
:1064D30003A3E06D701775083575090A780812076C
:1064E300FCEEFA121740740212080F801A750802A4
:1064F30075098078081207FC8C088D097808120743
:10650300FC12657812080F02658F74F6120363128A
:10651300654F7003A3E06D701775084275090A781B
:10652300081207FCEEFA121746740212080F801ABB
:1065330075080375098078081207FC8C088D0978A3
:10654300081207FC12657812080F8040EAFEEBFF81
:10655300126567FAA3E0F9EA2400FCE439FD900A26
:1065630014E06C22126B9C126B4DE0F8A3E0F988E7
:10657300828983E022EE127724EF1277CFFD7C80AD
:10658300126BB412175874042212080F7F0202050B
:10659300CA74F612036374FE1208A3EAFEEBFF85C6
:1065A3001882851983E4F0A3F0126BD7FA888289E5
:1065B30083A3A3E0F97509007508006005C394F18E
:1065C3004005750882802F900A14E06A7003A3E0E7
:1065D3006B7020851882851983AA82AB831212EA15
:1065E300E9F50985188285198312704170087508C9
:1065F300838003750881851882851983126AE8A947
:1066030008EEFAEFFB12174CE50960148518828532
:10661300198312704160098518828519831270FDF0
:10662300740202658C74F2120363EAFEEBFF750ACF
:1066330000750B0012669B120E10EA65087003EBDF
:10664300650970121212F6E914F50A79017A6B7B67
:106653000A1212FC8003750B801276FFF50C780C7E
:10666300120800750C6B750D0A780C1207FC780A7A
:1066730012080078081207FCE50BF50878081208E1
:1066830000126B75F582EF126B717A057B8012171E
:1066930052740712080F8014126B34126B5E8882D7
:1066A3008983127877F508E439F509227F06020514
:1066B300CA74F6120363E9FE7F00802F8A828B83FC
:1066C3001264C4F9E5082400E439F509EF33F8E46A
:1066D30033F9EC28F582ED39F583E508F0A3E509F4
:1066E300F0EA24020A0AEB3400FB0FEFC39E40CC0E
:1066F30002658F74E812036374FB1208A38A168B76
:1067030017851882851983E4F07403120A55E4F09F
:10671300A3F004120A55E4F0127695F50AA3E0F506
:106723000B850A82F583127873FEE439FF850A82AA
:10673300850B83A3A3E0FA850A82850B83A3A3A316
:10674300E0F9EAF508E439F509E50A2404F50AE570
:106753000B3400F50BEEFAEFFB120E82E9640170C5
:106763002C1274F6120800E4F508F50978081207EC
:10677300FC7808120800900A1412069975088078AC
:1067830008120800126B0312080F026AD6EEFAEF22
:10679300FB120E82E9700C900A14E06E7003A3E002
:1067A3006F70BE126AEE8814602EC333FAE433FBB3
:1067B3001213B07403120A55126B2E7403120A5586
:1067C30012704160137403120A55126AE0A914127D
:1067D30016DA8A0A8B0B8003751400126AEE880F8F
:1067E300602AC333FAE433FB1213B07401120A555F
:1067F300126B2E7401120A55127041600F7401124C
:106803000A55126AE0A90F1216DA8003750F009079
:10681300049E805D850A82850B83A3A3A3A3A3A300
:10682300A3A3E4F0A3F0AA0AAB0B8512828513831A
:10683300A3A3126AFE126BA3F91213388510828583
:106843001183E0C0E0851882851983E0F8746B2812
:10685300F582740A1277F8D0E0126DD204F0E515D0
:10686300A2E05007AA10AB111213B685128285134A
:1068730083E0F512A3E0F513E51245137003026AF2
:106883004E851282851383A3A3126BA360DD851249
:1068930082851383A3A3A3A3A3A3A3A3E0A2E0508E
:1068A300CA851282851383A3A3A3A3127041851201
:1068B30082851383A3A3601F126BA3FA7901851248
:1068C30082851383A3A3A3A3126BA8121CF48A10BB
:1068D3008B11751501800F126AFEA3A3E0F510A3B7
:1068E300E0F511751500E510451170030268618527
:1068F3001082851183A3E065087004A3E065096035
:1069030003026861851082851183A3A3A3A3A3A3B4
:10691300A3120699851082851183A3A3A3A3A3A31E
:10692300E0FC7405120A55126B8BA9141216BC7481
:106933000212080FE9703C851082851183A3A3A37B
:10694300A3A3A3A3A3A3A3120699851082851183EE
:10695300A3A3A3A3A3A3A3A3A3E0FC7403120A55B5
:10696300126B8BA90F1216BC740212080FE9700385
:10697300026861E50F2514C333240AFA7B0012135E
:106983002C8A0A8B0BEA450B700302683F8A828BC1
:106993008374D2F0851682851783A3A3126B5A8A58
:1069A300828B83126B648A828B83A3A3A3A3E514D4
:1069B30012787DE50FF0E5146038EA2405FAEB342C
:1069C30000FBE50A240AF8E50B3400F98A828B837D
:1069D300126B667403120A55126B211207F8E51441
:1069E300C333FCE433FD8A828B831271FA12080FDE
:1069F300800D8A828B83A3A3A3A3A3E4F0A3F0E572
:106A03000F7003026817E514C333F8E433F9E50A9A
:106A130028F8E50B39F9E8240AFAE93400FB850A7A
:106A230082850B83A3A3A3A3A3A3A3A3126B2E7497
:106A330001120A55126B211207F8E50FC333FCE468
:106A430033FD12774912080F0268298518828519C8
:106A530083E060271274F612080075086B75090A43
:106A630078081207FC7403120A5512750012080005
:106A7300900A141206997508008029EEFAEFFB12AA
:106A83000E82E9702A1274F612080075086B7509F4
:106A93000A78081207FC7508007808120800900AA3
:106AA300141206997808120800126B0312080F7467
:106AB30003120A5512704160087403120A551270CA
:106AC300FD7401120A5512704160087401120A55CF
:106AD3001270FD740512080F7F100205CA126AE8CE
:106AE300AA0AAB0B22E0FCA3E0FD22850A82850BF8
:106AF30083E0F8A385820A85830B22126BA8A32265
:106B0300E5162402FCE5173400FDE516126B6CE56F
:106B130017126BC17A067B80121752740722E0F5B5
:106B23000CA3E0F50D750E00780C22EAF0A3EBF050
:106B330022126B9C126B4D22EE2412F582EF22EE91
:106B43002415F582EF22126B4D223400F58322EED9
:106B53002404FE1276E222126B5E22E0F8A3E0F92F
:106B630022A3A3E8F0A3E9F022240FF58222126BFB
:106B7300C122EE2402FCEF3400FDEE240F22AC828E
:106B8300AD83851882851983126B8F22E0FAA3E007
:106B9300FB22FB12172E740522EE2413F582EF223B
:106BA300126BA8E022E0F8A3E0F5838882220207B3
:106BB300C1EE2402FAEF3400FBEE126B6CEF126BA2
:106BC3004DE0F92212080F7F070205CAF0851882EB
:106BD30085198322126567FCA3E0FBEC2274F6128D
:106BE300036374E01208A3EAFEEBFF85188285199C
:106BF30083AC82AD8312171C120FA27402120A55C2
:106C0300126B81120EACE964017003026DCD74182E
:106C1300120A55AA82AB83120E1C7402120A55ACD7
:106C230082AD837418120A55AA82AB83121B24E91E
:106C33006032120E168A088B09A808A909851882E2
:106C4300851983E0687003A3E0696018851882855D
:106C53001983126B5A900364126B667A647B03790F
:106C63004B121B54EE2411F582EF1277F8C082C049
:106C730083120E108A088B09D083D082E0650870D6
:106C830004A3E06509603E7402120A55AA82AB832D
:106C9300120AE08A088B09A808A909E8496026882E
:106CA300828983A3A3A3A3E06401600D88828983FF
:106CB300A3A3A3A3E06402700C7402120A55AA8270
:106CC300AB83120AEC120E108A088B09A808A909D3
:106CD300851882851983E0687003A3E069601174E5
:106CE30002120A55126B81120AC2E960031216449A
:106CF3007402120A55126B81120F847900126B858C
:106D0300120C42740B120A55E4126DD2F8A3E0F987
:106D1300740C120A55126B66740B120A55AA82ABD5
:106D230083120A8CE9604B7C087D00790074181289
:106D33000A55AA82AB8312131A740E120A55AC8237
:106D4300AD837418120A55AA82AB83121B24E9601F
:106D5300217402120A55AC82AD83740E120A55AA2D
:106D630082AB83120A68740B120A55AA82AB831290
:106D73000A9E7402120A55AC82AD83740E120A5530
:106D8300AA82AB83120A68740B120A55AA82AB83D8
:106D9300120A92E96034740C120A55126B5A851860
:106DA30082851983E0687003A3E069601D851882FA
:106DB300851983126B5A740C120A55126B66740B85
:106DC300120A55AA82AB83120A9E742002658C12A2
:106DD3006BCFE02274F112036374F61208A3EAFE88
:106DE300EBFF750800900A9F12704170407A377B61
:106DF30000126FFFEAF0A3EB12755D60197C377D1B
:106E030000790012131AEEFCEFFD900A9F126B8BB0
:106E13001216FEE9700B8518828519837488026F38
:106E2300621270067401F01274A4026FF4127006F9
:106E33007402F0EEFCEFFD1274971216FEE9700C6B
:106E43008518828519837488F0750801750A6B7536
:106E53000B0A780A1207FC900A9FE024291274D2C5
:106E6300120699900A9FE0242812701524151270B7
:106E730029241412701E12080FE9C0E0900A9FE043
:106E830024311274D2D0E0F0127527603C126FF9EE
:106E9300E0243212704A6025750C6B750D0A750E6D
:106EA30000780C1207F8127527C333FCE433FD9006
:106EB3000A9FE024321271F612080F800C851882A3
:106EC3008519837488F0750801780A1207FC900A03
:106ED3009FE024121274D2120699900A9FE02411A3
:106EE300127015242C127029242B12701E12080FF5
:106EF300E9C0E0900A9FE024341274D2D0E0F0128B
:106F03007709602E126FF9E0243512704A603F75DD
:106F13000C6B750D0A750E00780C1207F8127709C1
:106F2300C333FCE433FD900A9FE024351271F6125B
:106F3300080FE508A2E0401F127527700512703193
:106F430060157B007A007900121704026FF485182C
:106F5300828519837488F08518828519837486F075
:106F63007409120A557402127045127521120A55DA
:106F7300126B668E828F83A3127500120800740150
:106F8300120A5585820885830978081207FC75085B
:106F93002075098078081207FC79017406120A55D6
:106FA300AC82AD83EEFAEF126B9512080F127512D5
:106FB300703C7409120A557402F0127519120A55BD
:106FC3001275641208007401120A558582088583BC
:106FD3000978081207FC75082075098078081207DC
:106FE300FC79017406120A551274B212080F1216B4
:106FF300F8740A026BC7C333FAE433FB1213B0907D
:107003000A9F2212700A22900A9FE0242EF812741B
:10701300DB22127531FC900A9FE02218127532F9B7
:107023001216B674042212710B900A9FE022900A82
:107033009FE02434080808127532221274D61272A3
:10704300292212774FA3221274D6EAF0A3EB127708
:107053003BF8A3E0F9E84922C082C083900A9F125B
:10706300704170030270EF900A9FE0243512703E66
:107073006009900A9FE02435127104900A9FE0246E
:107083003212703E6009900A9FE02432127104901C
:107093000A9FE0241212703E6009900A9FE02412B6
:1070A300127104900A9FE0241512703E6009900A41
:1070B3009FE02415127104900A9FE0242912703E68
:1070C3006009900A9FE02429127104900A9FE0242A
:1070D3002C12703E6009900A9FE0242C12710490D8
:1070E3000A9F1270FD900A9FE4F0A3F0D083D08230
:1070F3000207C1F582EF3400F583126B8F1213B6CA
:107103002212710B1213B622F8127536FAA3E0FBA2
:107113002274F1120363EAFEEBFF8C088D09750AF2
:10712300018C0C8D0D750E00780C1207F87C177D01
:107133000012774912080F126B3B127667126B42EB
:107143001276732411F582E509127705602AEE247D
:1071530012127201601FE50824121271EA1207F875
:10716300E50824111271DF126B3C1277F81271FAE1
:1071730012080F8003750A00E5082414F582E50957
:107183001277056025EE2415127201604AE5082482
:10719300151271EA1207F8E50824141271DF126B55
:1071A300431277F81271FA12080FE50AA2E040229F
:1071B300126B3B1277F81270416006EE24121270C4
:1071C300F6126B421277F81270416006EE24151224
:1071D30070F6A90A026BCA750A0080D41277CBC372
:1071E30033FCE433FDEE221277CBF50CA3E0F50D6F
:1071F300780C22081274D7126B8F12774922F8EF9A
:107203003400F9880C890DE0C333FAE433FB12131D
:10721300B0850C82850D83EAF0A3EBF0850C8285A3
:107223000D8312722922E0F8A3E0F9E8492274EEF3
:1072330012036374ED1208A3890A8A0E8B0F750C6F
:1072430000750D00750BFF7510FF7511FF750800B4
:10725300750900851882851983E412755D700579B7
:10726300000274807403650A60067402650A700D77
:10727300900A9FE0243012770F650F70E27C0A7D3D
:10728300177A007B00121CCE7401650A700B8518F7
:10729300828519837485F08043E50A60067403656B
:1072A3000A7019900A9F1274EDF07403650A70282E
:1072B300E50E602885188285198380DA7402650AD1
:1072C300701AE50E900A9F70051274ED80C8E024D1
:1072D3002F1274D2740280BEE50A6019127506700B
:1072E30014900A9FE0243108081277107005127079
:1072F30031600214F0127527900A9F60141264C45F
:107303001274C0243212753B241D12748A24258002
:10731300201270346020900A9FE02417F508A3E040
:1073230034001274C0243512753B240612748A2467
:107333000E12770FF50B7409120A557402126DD2EF
:1073430060030273F2E508450970030273F21275D4
:107353000670047E2280027E2185088285098312BD
:10736300751F120A55126B66900AA1E0C0E0900ADD
:107373009FE024301274D2D0E0F07412120A5574D4
:1073830003F0AC0CAD0D740A120A55AA82AB83123A
:107393001B2A850882850983A3E0F50C780C120863
:1073A30000780B120800740C120A5585820C858331
:1073B3000D780C1207FC78101207FCE5082406F57B
:1073C3000CE5093400F50D780C1207FC127722E561
:1073D30009126B717409120A55AC82AD83EEFA7B04
:1073E3000012175E740812080F1274A402747E123E
:1073F3007519120A551275641208007401120A55A0
:1074030085820885830978081207FC7508207509A9
:107413008078081207FC79017406120A551274B2B7
:1074230012080F1275127050900A9FE024191274FB
:10743300D2127521120A55126B66900A9FE0241826
:107443001274D21275001208007401120A55858253
:107453000885830978081207FC7508207509807868
:10746300081207FC79017406120A55AC82AD831227
:107473007497126B9612080F1216F879017413128F
:10748300080F7F0A0205CAF50CA3E03400F50D903E
:107493000A9FE022900A9FE02417FAA3E03400FB3E
:1074A300227C0A7D17900303126B8F121CCE22AC31
:1074B30082AD83900A9F126B8F126B9622F5098817
:1074C300828983E0C333F8E433F9900A9FE0221200
:1074D30074D622F81274DB221274DF22A3E0127432
:1074E300E5223400F98882898322E0242F1274D69E
:1074F300740122E516127724E517126B49E0F508AB
:10750300780822900A9FE0242F1275316401221219
:10751300700AE0640222900A9F126BA8A3A3126B65
:107523005E740122900A9FE0243112753122F81211
:107533007536221274DFE022FAA3E012772928F8C5
:10754300A3E039F9E824FEF582E934FFF583E0F599
:1075530010A3E0F511900A9FE022127576F9E8492D
:1075630022E8F0A3E9127576F5838882A3E0F50893
:10757300780822F0900A9FE0F8A3E022C082C0833B
:107583007B007A8579011217040270EF74F41203F9
:10759300638C088D09EA240F1277FC1277D4126BDF
:1075A3005A8C828D83126B64EA240E1277FC127656
:1075B30095FEA3E0127844A3A3A3A312785824064C
:1075C300FAE5091276D4C0E01277F0D0E01276EC37
:1075D300F8E508240F1277F4E81277142412F582E1
:1075E300E5091276732415F582E5091276678E8212
:1075F3008F83E0A30EAF83C0E0E50824111277F474
:10760300D0E0F0601FE50824121276AB6016E5089F
:10761300241212768424111276798A0A8B0BAE0A0D
:10762300AF0B8007E50824111276F58E828F83E075
:10763300A3AE82AF83C0E0E50824141277F4D0E050
:10764300F06017E50824151276AB600EE5082415E3
:1076530012768424141276798007E50824141276AE
:10766300F50263E012766B22126B4DE4F0A3F02275
:1076730012766BE50822F582E509126BC11216DA60
:1076830022F582E509126B49126AE8EEFAEFFBE58F
:107693000822A3F012769B2212769F22EA2413F586
:1076A30082EB3400F583E022F8E5093400F9880A17
:1076B300890BE0C333FAE433FB1213B0850A8285E6
:1076C3000B83EAF0A3EBF0850A82850B8312722900
:1076D300223400FB121B2AEE2408FE1276E222EF6C
:1076E3003400FF8E828F83E0221277E0FAA3E0F961
:1076F300EA22F582E509126B49E4F022EE240EF545
:1077030082EF1277CF22900A9FE02434F812753269
:107713002212771AE50822F0A3E9F01277C122E5D5
:1077230008240EF582223400FB8A828B83E0227FB9
:10773300010205CA12773B22F088828983E022EA9C
:107743002413F582EB2212130E74032212775322B1
:10775300F08E828F83A32274F7120363EA2413F853
:10776300EB1274E5E0FAA3E0F5838A821278021241
:107773007737F8A3E0F988828983A3E0FA888289BE
:1077830083A312784FA3126B67027732FAE50934A9
:1077930000FB121B2A22FAA3E0F9EA850882850975
:1077A30083228E828F83E0850882850983A3A3A326
:1077B300A3A3221277BA221277530EAF8322EE24A9
:1077C300020E0EEF3400FF22F582E509126B4DE045
:1077D300221277D822F08A828B83A3A322127753B3
:1077E300AE82AF83E022E0FAA3E0F9EA22E50824BF
:1077F3000EF582E509126B4922F582EB126B49E023
:107803008C828D832274F61203638C088D0912789F
:107813003612783D12784412785824021278628521
:107823000882850983A3A3A3A3A3A3A3A3A3A3F06C
:1078330002658F127742126B4922126B5EE8FEE9F2
:1078430022FF8E828F83E012784E22FAA3E0F9EAB8
:107853008C828D832212771AEEFCEFFDE50822124B
:10786300778F8E828F83A3A3A3A3A3A3A3A3E022D3
:10787300127877221277E9240022127885A3A3A332
:10788300A3221277D8A32274F61203638C088D09FE
:107893001278F5850882850983120A3E126B528598
:1078A3000882850983A3A3A3A312791AC39406505C
:1078B300051277A98038850882850983A3A3A3A32A
:1078C300E064FE600E850882850983A3A3A3A3E079
:1078D300F4701C1277A5A31277B6850882850983F5
:1078E300A3A3A3A3E0F4700712790AF0A3E9F002BB
:1078F300658F1279027904EEFAEFFB12132022123C
:10790300769FFEA3E0FF228E828F83E0127799A3F6
:10791300A3A3A3A3A3A32212774FAE82AF832274A0
:10792300F5120363EAFEEBFF740B120A55E0F50848
:10793300A3E0F509A3E0A908AA09FB8E828F83803F
:107943000D120829F0E9240109EA3400FAA3127997
:107953005F70EEAA82AB837F030205CAECFEEDFFE4
:10796300EE24FF1CEF34FFFDEE4F2274ED12036390
:107973007413120A55E0F510A3E0F511A3E0F51214
:1079830089088A098B0A85100C85110DECF8EDF92D
:10799300E824FF1CE934FFFDE8496036A908AA0979
:1079A300AB0AE92401F508EA3400F509850C1085D2
:1079B3000D11E50C2401F50CE50D3400F50D12084D
:1079C30029F8A910AA11AB121208296860BE790020
:1079D300800279017F0B0205CA74F6120363E9FE84
:1079E3008C088D0978081207FC8E08AC087D0012FC
:1079F3001BA8740212080F027D1074F0120363E9CE
:107A0300FE74026E701D8A828B83127A95780C1233
:107A1300077D7808790C12091FAA08AB09AC0AADD7
:107A23000B805774036E70168A828B83127A8F12BF
:107A3300077D7808790C12091F127A8080CF7404AD
:107A43006E8A828B83702D127A8F12077D78087964
:107A53000C12091F127A80780C12077D7808790CB2
:107A630012091F8A828B83A3A3A3E0F50CE4F50E0E
:107A730074188099E0FAE4FBFCFD027FC28A828BD2
:107A830083A3A3E0F50CE4F50D741022127A957824
:107A93000C22E0F508E4F509F50AF50BA3E0F50C73
:107AA300E4F50DF50EF50F740822C082C08312149D
:107AB300A6807574F6120363EAFEEBFFEE4F7006C1
:107AC3007A007B00803DEE2405FAEF3400FB1213AD
:107AD300B08A088B09A808A909E84960E388828964
:107AE30083E4F0A3F088828983A3A3EEF0A3EFF0ED
:107AF30088828983A3A3A3A374FFF0E82405FAE98A
:107B03003400FB027D10C082C083EA4B7004790508
:107B13008016127B8360047904800DEA24FBFAEB60
:107B230034FFFB1213B67900D083D0820207C174ED
:107B3300F7120363E9FEEA4B7004790580409080F5
:107B430069E0F8EEC39840071213327903802FEAF5
:107B5300127C67EB127DA4127CAE7005127B8360EE
:107B63000512133280D4EEF0EAFCEBFD7AA07B041D
:107B730012134A7A007B80EEF912136879008011A0
:107B8300EA24FFF582EB34FFF583E0F422A2E092CE
:107B9300AF7F010205CA74F2120363890B750C00EF
:107BA300750D007E007F00A2AFE433F50AC2AF90EB
:107BB30004A08014EE4F700685080C85090DE508B6
:107BC300127C67E509127DA4E0F508A3E0F509E559
:107BD3000845096023E50824FFF582E509127DA421
:107BE300E0650B70CFEE4F7006AE08AF0980CF7A19
:107BF300007B80121368800B7A007B8012136EEE79
:107C03004F6015780C1207FCEEFCEFFD7AA07B04A5
:107C1300121C80740212080FE50AA2E092AFEEFA7A
:107C2300EFFB7F060205CAC082C083EAF8A2AFE475
:107C330033FCC2AF9004A08008EA127C67EB127D8C
:107C4300A4127CA46015EA24FFF582EB127DA4E064
:107C53006970E68A828B83E06870DEECA2E092AF03
:107C6300027B2BEC24FBF5822274F7120363A2AF91
:107C7300E433FEC2AF127DA9127CAA70098A828BFB
:107C830083800B127DC2127C9A70F8127D9EECF0F9
:107C9300A3EDF0EE027B90E824FBF582E934FFF5D7
:107CA30083127DBCEA4B228A828B83E0F8A3E0F93E
:107CB300E8492274F612036378007900A2AFE43333
:107CC300F508C2AF8A828B83E0FCA3E0FDEC4D6034
:107CD300328A828B83127DCCE824FBFCE934FFFDDE
:107CE3008C828D83E0FEA3E0FF8A828B83EEF0A378
:107CF300EFF08C828D83E4F0A3F0E824FF127DA1E2
:107D030074FFF0E508A2E092AFE8FAE9FB7F020214
:107D130005CA74F7120363E5A8FEC2AF8A828B8398
:107D2300127DCC127C66ED127DA4E8F0A3E9F08A03
:107D3300828B83ECF0A3EDF0EEA2E7027B9274F763
:107D43001203637409120A55127DCCA2AFE433F512
:107D530008C2AF8A828B83E0FEA3E0FFEC6E700261
:107D6300ED6F7011127C66ED127DC88A828B83E8F9
:107D7300F0A3E98011127C66ED127DA4127DB81286
:107D83007D9EEAF0A3EBF0127DA9EC24FFF582EDD2
:107D9300127DA474FFF0E508027B90E824FBF582D2
:107DA300E934FFF58322EC24FBF582ED34FFF58300
:107DB300E4F0A3F022127DBC22E0FAA3E0FB22E868
:107DC30024FBF582E934FFF583E0F8A3E0F922749C
:107DD300F7120363E9FE7F00A2AFE433F508C2AFF5
:107DE300127CAA700C8A828B838012EE6015127D3E
:107DF300C21E127C9A70F4EE6009127D9EECF0A311
:107E0300EDF00FE508A2E092AFEFF9027B9474F76F
:107E1300120363E9FD908069E0F8EDC3985029E50A
:107E2300A8FEC2AFEDC333F8E433F99004E5E028CC
:107E3300FCA3E0398C82F583E04AF0A3E04BF0EE3B
:107E4300A2E792AF790080027903027B9474F71260
:107E53000363E9FE908069E0F8EEC398501FE5A83C
:107E6300FFC2AFEAF4FCEBF4FDEE127F73E05CF0CB
:107E7300A3E05DF0EFA2E792AF79008002790302FD
:107E83007B94E9F874FF687006D2AF7900800279B9
:107E9300070207C1E9F874FF687006C2AF79008072
:107EA3000279070207C1C082C0831213A49004A001
:107EB300E4F0A3F012144C12144012148E1213AAFD
:107EC3007900027B2BC082C08312138C80FB74F673
:107ED30012036375080012139E1217F4E508127F4C
:107EE30073127CAE700D0508908069E0F8E508C355
:107EF3009840E9908069E0F8E508C3985066E5A8E2
:107F0300FCC2AFE508C333FEE433FF9004E5E02E83
:107F1300F8A3E03FF988828983127DB88882898338
:107F2300E4F0A3F0ECA2E792AFE508901171F0F949
:107F330074002EF58274803FF583127F6A121CF45D
:107F430090117174FFF0E5A8F9C2AF9004E5E02E3B
:107F5300F8A3E03F8882F583E04AF0A3E04BF0E921
:107F6300A2E792AF027D10E0F8A3E0F583888222B6
:107F7300C333F8E433F99004E5E028FAA3E0398A3F
:107F830082F5832274F01203637410120A55780C7D
:107F93001209F88A828B83E50C127FE6850C08852B
:107FA3000E0A850F0B7410780812085CE508F0A31D
:107FB3007418780C12085CE50CF0A3AA82AB837FDB
:107FC300080205CA74F01203637410120A55780C80
:107FD3001209F8850C088A828B83E508127FE67400
:107FE3001080CFF0A3850D09E509F0A3220207C194
:10800000AC11C60CEE17D41CC61B8A156E165A1579
:108010000C00000001000300000000730000007469
:1080200001040F010000016780016780000000006B
:1080300000000000FFFFFFFFFFFFFFFF82003A008C
:108040003B000508050001E8030000640000000093
:10805000000C000100000000F8FF073000000000E5
:108060005800000000000001000874F7120363E9E3
:108070009003BBF0900370E4F0121B009003CFE478
:10808000F0A3F09003BCF0A3F0120F3C120AAA1266
:108090000BB2121B06900335E4F0A3F09021DA93A3
:1080A000FA7902121B7802C7F974F2120363EAFE2E
:1080B000EBFF548060699003BBE0F912133E8A081D
:1080C0008B09EA4509604F7C0080010CEC75F003D8
:1080D000A4F8A9F074CC28F582742039F583E493D0
:1080E000F4602CE493F88508828B83E06870DCAA46
:1080F00008EC75F003A4F874CD28F582742039F5E6
:1081000083E493C0E0740193F583D082121CF4AA37
:1081100008AB09121332EEFAEF6480FB0282E2EF41
:108120005420601D120DC28A088B09EA4509600AB5
:10813000120CFCAA08AB09121332EEFAEF6420808D
:10814000DAEE54207003028223750C0012A7468BCE
:1081500009EA4509700B7C027D007A207B0012D071
:10816000B87C0079047A007B00120D8C8A088B0998
:108170008018850882850983A3A3A3A3A3A3A3A32F
:10818000A37401F0850A08850B09E5084509606DAF
:108190007C007904AA08AB09120D8C8A0A8B0B7536
:1081A0000C01E5082404F8E50912A4D124FFF0A38A
:1081B000E034FF12E06570CC850882850983A3A3B3
:1081C000A3A3A3A3A3A3A3A3E0640170A58508822E
:1081D000850983A3A3A3A3A3A3E0540470948508F3
:1081E00082850983A3A3A3A3A3A3A3A3A37406F0D7
:1081F0007AB785088285098312844A8087120D5CCC
:108200007C0079017A007B00120D8C8B09EA45090C
:108210007009E50C70057A201282E5EE6420FAEF11
:1082200002811BEE54106008120BEEEE641080EE1B
:10823000EE54406008120C6CEE644080E1EE548015
:108240006008120B34EE648080D4EF540160169005
:1082500003EE12AAF6600612BB77121CF4EEFAEFD8
:10826000640102811BEF5408602E120BBE900B00BC
:10827000E06401701B900B01E06015FC75F0E8A450
:10828000CCA8F075F003A428FD7A007B0812D0B8C2
:10829000EEFAEF640802811BEF541060139003CDD7
:1082A000E06005E4F0120BBEEEFAEF641002811BF1
:1082B000EF5402600B120F06EEFAEF640202811B0C
:1082C000EF5404601912BF6C12BDD7790190036E90
:1082D00012C2F7120B82EEFAEF640402811B7A00DD
:1082E0007B000286617B009003BBE0F912147022D0
:1082F00074F712036374E11208A3EAFEEBFFEE4F7A
:108300006033851882851983AC82AD83120DF274B7
:1083100006120A55E0601E7417120A55E0FD74013A
:10832000120A55E0FCEEFAEFFB7900121C7AE960C4
:108330000479A48002790002C7F474F6120363EA98
:10834000FEEBFF8E828F83A3A3A3A3A3A3E05440DD
:10835000601312CBCA12863C60067AFF7BFF8070E6
:1083600012842C806190035BE0A2E150568E828FD4
:1083700083E0241C12A4E012DF8DE0FA8882898356
:1083800012C2FBE0F9EA2400FCE439FD8E828F83FF
:10839000A3A3A3A3A3A3A3E0541060047940800285
:1083A00079007508FE7509FF78081207FCEE240EA7
:1083B00012842512069912842C120BC4740412081C
:1083C0000F8003120E1674FE6A700374FF6B604117
:1083D00012CBCA12C4FD120E82E98E828F83600610
:1083E000128438E480051284387401F07CCC7D0C52
:1083F0008E828F8312C2F7121B72E9F5087015EE98
:108400004F60097901EEFAEFFB120D68A90802BB73
:10841000957508CDAA088E828F8312844AE960DFA1
:1084200080EAEE240BF582EF12AA27228E828F8338
:1084300012A9FAFAA3E0FB22E0240D12843F2212D3
:10844000844322F8A3E012B2BC22E0240C12A4E47C
:10845000F9120CD82274F6120363E9FEEAFF7A0FD0
:108460007B0012132CEA4B60198A828B83740CF008
:10847000EEA3A3F0EF8A828B83A3F012BDC0790034
:10848000802FEEF9120D928A088B09A808A909E835
:1084900049601C88828983A3A3A3A3A3A3A3A3A346
:1084A000740612DAEEE0F9120C7EEEF9120D6E7916
:1084B0001002BB959003BBE0F912146422C082C085
:1084C00083790090035BE0A2E1EA501112A9D61271
:1084D00006F101010ADA8400EF8409801212A9D69C
:1084E00024FD60F61460F324FD60EF24FD60EB02D0
:1084F000B77874F2120363EAFEEBFF8C088D0989EA
:108500000A740E120A5512B0B8850C82F583E4F095
:10851000A3F0128620601712864970128E828F8314
:1085200012AB69850C82850D8312BDD78003750A55
:108530000012861AEF12A9DA14602414603914604C
:108540005D14606514603E14607F24FE7003028534
:10855000E31470030285F714700302860A803578ED
:108560000C1207FCAC08AD09EEFAEFFB120BD67447
:108570000212080F028613AC08AD09EEFAEFFB12E7
:108580000BDC02861612862F700AEEFAEFFB120C35
:1085900024028616750A007901121B128078A90A36
:1085A000EEFAEFFB120EC4806A12967E640270E44B
:1085B000E50A700A12CF777003A3E0697058EEFAEB
:1085C000EFFBA90A120E52804A12CF777003A3E084
:1085D0006970C112967E640270BAEEFAEFFB120E59
:1085E0003A80339003F012AAF6602BEEFAEFFB12FA
:1085F000BB77121CF4801F12CF777003A3E0697061
:1086000093EEFAEFFB120ED0800CEEFAEFFBA90A04
:10861000120EDCE9F50AA90A8047EE241DF5822234
:10862000EE241D12AA2412A9FAF9120E64E9228E70
:10863000828F83A3A3A3A3A3A3A3A3A312864022F1
:1086400012A4F8FB120E82E9228E828F83A3A3A3C9
:10865000A3A3A3A3A3A31286406402227403120857
:108660000F7F060205CA74F412036374DE1208A3B6
:108670008A088B098A828B83A3A3E0F9120D928A60
:108680000A8B0BAE0AAF0BEE4F700302876B8508A7
:1086900082850983A3E064F16033850882850983BC
:1086A000A3E064CD6027850882850983A3E0641A6E
:1086B000601B850882850983A3E064E9600F850853
:1086C00082850983A3E064E160030288088E828FBB
:1086D00083A3A3A3A3A3A3A3E054087003028773F7
:1086E0008E828F83A3A3A3A3A3A3A3A3A37405F044
:1086F0009003F412AAF6600612BB77121CF49003E2
:10870000F612AAF6603690035BE0A2E1502E8E824C
:108710008F831288CDA3A3A3A3A3A3A312A83D88EC
:108720008289831292AFEA4B6012850882850983A1
:10873000A3E0F99003F612CBCE121CF48E828F8345
:10874000A3A3A3A3A3A3A3A3A3E0640270108E8298
:108750008F83A3A3A3A3A3A3A3A3A37406F0850855
:1087600082850983A3A3E0F9120D6E120D5C7422B9
:1087700002A02C7900120D68E970030288089003AA
:108780005BE0A2E140030286F012AAEC70030286CD
:10879000F08E828F8312C2F77403120A5512CD38FD
:1087A000850882850983A3E064E9701B1288D912C9
:1087B0000800850882850983A3E0F50A780A120873
:1087C00000129BE712080F740C120A551288C3128C
:1087D000DF7D12BDD77408120A55E060047940802D
:1087E000027900740E120A5512A83D740C120A5533
:1087F0001292A770030286F08E828F83A3A3A3A395
:10880000A3A3E044200286EF850882850983A3E0C4
:10881000C0E07402120A55D0E012AF17EEF0A3EFD9
:10882000129C06851882851983AA82AB8370051273
:108830000B5E8003120E5E7402120A55E064E9704A
:10884000141288D9120800750AE9780A1208001271
:108850009BE712080F90035BE0A2E1400302873C14
:108860008E828F83A3A3A3A3A3A3A3A3A3E06402E5
:1088700070388E828F83A3A3A3A3A3A3E0540460C4
:108880002912CBCA12863C8E828F83700F12CBCEF8
:1088900074FFF0A312A510740502875DA3A3A3A320
:1088A000A3A3A3A3A3740302875D8508828509831C
:1088B000A3E064E9600302873CEEFAEFFB120EE2EC
:1088C00002873CE0F8A3E0F98E828F8322E0F8A3D0
:1088D000E0F988828983A3A3228E828F8312AAFB68
:1088E000FAE9FB750A01780A2274F4120363EAFEBE
:1088F000EBFF7508007509008E828F83A3A3A3A3E5
:10890000A3E060427508088E828F83A3A3A3A3A36C
:10891000A3A3A312AE398B0BEA450B601075082C8C
:108920008E828F83A3A3A3A3A3E0D2E0F08E828FD5
:1089300083A3A3A3A3A3E05403640160030289E615
:108940004308110289E6EE24181296816044EE2451
:108950001A129681701D12CF777003A3E06970061A
:108960007508220289E6900370E064047078750946
:10897000018073EE241BF582EF128A05241AF5821A
:10898000EF129DF7EE24191289FD120C36E970568C
:1089900080DC128649700375080112CF777003A33B
:1089A000E0697006E508D2E1F508E50860158E82F9
:1089B0008F83A3A3E07006E508D2E58004E508D222
:1089C000E6F50812862F64017006E508D2E0F50886
:1089D0008E828F83A3A3E0600D128620640160065F
:1089E000E508C2E0F508E508A2E1400CE509A2E0CF
:1089F0004006E508D2E7F508A90802A02FF582EFA6
:108A000012DAD8F9223400128A0B22F58312A84513
:108A1000EE22C082C08379018A828B83A3A3E0C344
:108A200094024001198A828B83A3A3A3A3E0C39479
:108A300002400279008A828B83A3A3A3A3A3A3A3EA
:108A4000A3A3E064F87003A3E0F460458A828B83FB
:108A5000A3A3A3A3A3A3A3A3A3E064F97003A3E028
:108A6000F4602E8A828B83A3A3A3A3A3A3A3A3A3AF
:108A7000E064FA7003A3E0F460178A828B83A3A3F7
:108A8000A3A3A3A3A3A3A3E064FB7003A3E0F470D8
:108A90000279008A828B83A3A3A3E0F890035EE0AF
:108AA00068600279009021DDE493C394805013EA5A
:108AB000241112DACB9021DDE493C333C398500222
:108AC000790002B77874EC12036374DC1208A3EA2D
:108AD000FEEBFF7403120A5512969675100075117D
:108AE000007405120A55AC82AD838E828F83A3A3D6
:108AF000A31288C512C2F5120DF2E9600F740512B7
:108B00000A55AA82AB83120CF6E970087901121B90
:108B1000120290A0EE241B12842512AB7274121262
:108B20000A5512BDD7740B120A55E06021741C124D
:108B30000A55E0FD7406120A55E0FC8E828F8312FE
:108B4000C2F57901121C7AE96004790280C07405CB
:108B5000120A55AA82AB83120CF0E9F509740B12C4
:108B60000A55E0702A900358E06024742255096485
:108B700022601C74425509644270CF7422120A5557
:108B80001292BC600A7422120A551292C870BBE994
:108B9000A2E6503C7405120A55AA82AB83120CDE81
:108BA000E97003028B0C7422120A551292B6700CF3
:108BB0007422120A5512C1B9640D60147405120AA8
:108BC00055AA82AB83120EB8E9640170030290A02B
:108BD000EE242C1284251297FE7003A3E069701C0A
:108BE00075080078081208007808120800EE242E94
:108BF0001289FD1292D6129BFD12080F740B120AF5
:108C000055E07003028CB21292D61292AF8A0A8B90
:108C10000BEA450B7003028D3F7406120A55E0F80B
:108C20008E828F83A3A3E028F8A3E03400F9E82420
:108C30000DF582E912DACE8A828B83A3A3A3E068C2
:108C4000601CE88A828B83A3A3A3F0908063120A3E
:108C500032850A82850B83A3A3A3A3120A3E79045B
:108C60007406120A5512CCA92AF8A3E034008882AF
:108C7000F583A3AA82AB831213208A0C8B0D8C0E72
:108C80008D0F850A82850B83A3A3A3A3780C1207FB
:108C90005E40030290A0908053780C12090C850A64
:108CA00082850B83A3A312D3B1F0A3E50EF0A3E555
:108CB0000FF090035BE0A2E15003028DD9900370A6
:108CC000E064046008E0640960030290A0E509A282
:108CD000E54003028D81129308C0E07401120A5529
:108CE000D0E0129300C0E07402120A55D0E0F07494
:108CF00016120A55E0640170207410120A5512927F
:108D0000E77003A3E0697011740E120A55128656BB
:108D100070077416120A55E4F0EE2424128425120A
:108D200006957404120A55AC82AD837409120A5573
:108D3000AA82AB83120B64740412080F0290A090F5
:108D400003B5E064016003028CB27422120A55126A
:108D500092BC7009E509A2E65003028CB2741212AB
:108D60000A55E0F47003A3E0F470030290A0EEFC57
:108D7000EFFD7405120A55AA82AB83120D02029010
:108D8000A0A2E640030290A07422120A5512C30862
:108D9000701E741C120A55E0640260030290A074F5
:108DA00005120A55AA82AB837900120E520290A0D6
:108DB0007422120A551292C860030290A0741C1209
:108DC0000A55E0640460030290A07405120A55AAD3
:108DD00082AB83120E460290A07416120A55E06010
:108DE0002212B2B312DF851412A50BF8A312BB77BF
:108DF000A3A3A3A3A3A3E0C0E07416120A55D0E076
:108E0000F07006E509C2E7F509E509A2E3506175CE
:108E10001110A2E25018740A120A55E054E3F074DB
:108E20000A120A55E0131313541FF8E0802CA2E431
:108E3000502A740A120A55E01313543F5407F8607D
:108E400009740768600B18E87007C3E509C2E7F505
:108E500009E8333354FCF8E054E348F0740A120A8A
:108E600055E0C0E08E828F83A3A312A5E8D0E0F086
:108E7000900370E064046005E064097068740E1289
:108E80000A5512CF847003A3E0696019740E120AA8
:108E900055128656600F740A120A55E05403640195
:108EA00060030290A07407120A55E0701B12930829
:108EB000C0E07401120A55D0E0129300C0E07402C1
:108EC000120A55D0E0028D187422120A5512C308F6
:108ED0007003028D927422120A551292C860030226
:108EE00090A0028DBD750800746155097003029051
:108EF000A5E509A2E0507512A8377405120A55AA13
:108F000082AB83120C72E97060120E22E9F50874CC
:108F100016120A55E0700F7410120A551292E7707B
:108F200003A3E069604612A8357405120A55AA82A7
:108F3000AB83120C78E96026E509A2E3500B7403B9
:108F4000120A5574FFF0A3800F740E120A55129284
:108F5000C2120A55E8F0A3E9F0751004800EE50985
:108F6000C2E5F509750800800353099FE509A2E5EC
:108F7000503C129308C0E07401120A55D0E01293DD
:108F800000C0E07402120A55D0E0F0EE24241284EE
:108F9000251206957404120A55AC82AD8374091229
:108FA0000A55AA82AB83120B64740412080FE509F8
:108FB000A2E6503B7403120A5585820A85830B781A
:108FC0000A1207FC12A8357407120A55AA82AB834D
:108FD000120CE4740212080FE9F5086012742212F0
:108FE0000A5512A9DD6401700674104510F510745D
:108FF00003120A55E064FE7003A3E0F470037508E1
:1090000000E509A2E740030290A0E5087003029082
:10901000A08E828F83A3A3A3A312B2C48A0A8B0B50
:10902000EA450B607BEE2404F512EF3400F5138E55
:10903000828F83A31292F21207F88512828513831E
:10904000E0FC7D0012B64E12080F7407120A55128A
:1090500093187401120A55E4F012AF1685820C853C
:10906000830D780C1207FC78101207FC78081208A0
:1090700000EE24121284251206998512828513832C
:10908000E0F9740A120A5512A83DAA0AAB0B120D98
:10909000DA740712080FE96007AA0AAB0B1213B6BD
:1090A000742402BB7B7407120A55E06401703474A7
:1090B00022120A5512A9DD640570287403120A559C
:1090C00085820885830978081207FC790012A83781
:1090D0007407120A55AA82AB83120CE474021208B8
:1090E0000F80BD7416120A55E0700F7422120A55D3
:1090F0001292B66003028D6E80A6120D62E970A016
:10910000741D120A55E070030291E27420120A5590
:1091100012A83D741F120A55E0FA741E120A55E097
:10912000F9120C36E970030291C0741F120A55E05F
:10913000701F740E120A551292C2120A5512BDD730
:109140007403120A5512A0198B0BEA450B70688044
:10915000637420120A5512C2F7741F120A55E0F9FF
:10916000120C307403120A5512C4FD740D120A5504
:10917000E06004780880027800E82408FA740C1291
:109180000A55E06004780880027800E82AFA740A38
:10919000120A55E06004780180027800E8042AF899
:1091A0008E828F83A3A3E028FAA3E034008A82F59D
:1091B00083E014F0751040120E22E9F508028FEFDB
:1091C0007808120800790B740F120A5512A83D7422
:1091D00011120A5512C2F7120EBE740112080F02C4
:1091E00090A0740E120A551292C2120A5512BDD7DF
:1091F000E509A2E3500474408001E4F50878081200
:109200000800741E120A55AC82AD83740F120A5501
:1092100012C2F7740A120A55E0F9120CA274011274
:10922000080FE9600F7510208E828F83A3A312A907
:10923000DD543FF0741D120A55E06022740E120ACC
:109240005512A83D741E120A55AA82AB83120DEC6A
:109250007403120A5512C4FD74404510F5107407CA
:10926000120A55E06401601579007410120A551253
:10927000A83D740E120A5512C2F7120C3CE509A261
:10928000E350047940800279007410120A5512A844
:109290003D740E120A551292A770030291B7742002
:1092A0004510F5100291B71293B1120BD0E92212BA
:1092B00093B1120F6C2212A9FA64032212A9FA6464
:1092C000062212AF337403221292CFE0640722A366
:1092D000E0F583888222EE242AF582EF3400128A98
:1092E0000B241212AA242212AF33EE241212DAD562
:1092F0006822A3E0F50CA3E0F50D750E00780C22B2
:10930000F0EE243012DAD522EE242E12AA24129383
:1093100018EE242F12DAD522E0851882851983F001
:109320002274F4120363EAFEEBFF8C088D09900BA4
:1093300000E0600F12CF777003A3E0697005120B95
:10934000BE804F790012C2EA120C908A828B83E5AC
:109350008245836035A3A3A3A3A3A3E05418602A86
:10936000E508241BF582E50912842812069912A14A
:10937000C0128428120699EE24181289FD129395C2
:10938000120CAE740412080F800879001293951223
:109390000BE802A02F8E828F83A3A3A3A3A3A3A372
:1093A000A3A3128A0D12D65FEF1293AD223400F5FB
:1093B0008312A4F8FB2274F012036374EA1208A368
:1093C0008A0A8B0BEA2402F50EEB3400F50F0A0A29
:1093D000FB120AE08A088B09AE08AF0975080185FF
:1093E0000A82850B83A3E0F50C750901AC0EAD0F65
:1093F000851882851983AA82AB83121B2A740812EE
:109400000A55129696740A120A557402F0741312D1
:109410000A55E4F090114AE0700EEE4F700AE50C28
:1094200070067508C30295C4900370E06408600676
:109430007508C20295C0850A82850B83A3A3A3A3E6
:10944000A3A3A3A3A3A3E0A2E1500EA2E35005753A
:109450000904800C7509038007A2E3500375090213
:10946000EE4F70030294ED8E828F83A3A3A3A3E03B
:109470006404600D8E828F83A3A3A3A3E0640370B2
:109480000C74046509602C7403650960268E828F54
:1094900083A3A3A3A3E06402600D8E828F83A3A3A2
:1094A000A3A3E06401702874026509600674016575
:1094B00009700F8E828F83129F3C120A5512BDD7FE
:1094C000802B8E828F83A3A3A3A3E06402600D8E02
:1094D000828F83A3A3A3A3E06401700A8E828F838B
:1094E00012A020121CF41296887E007F00740812CD
:1094F0000A55E064FE7003A3E0F47042120AA4E986
:10950000703CE50C60179003ADE06402700F9011A1
:109510004E129F3C120A55E8F0A3E98020850A828A
:10952000850B83A3A3A3A3A3A3A3A3A3A3E0540294
:10953000F9120BFA7408120A55EAF0A3EBF074085A
:10954000120A55E064FE7003A3E0F470057508C7C5
:10955000806EE50CF50D780D120800850A82850BEA
:1095600083A3A3A3A3A3A3A3A3A3A3E0F912967326
:109570007409120A5512C2F7120B88740112080FEF
:10958000E9703DA9091296737408120A5512978260
:109590008A0E8B0FAE0EAF0FEE4F601C7402650C7F
:1095A000700BEE240512968154FB4408F0740A12E5
:1095B0000A55E4F0F50880087408120A55129696C8
:1095C000E50C700F851882851983AA82AB83121B64
:1095D0005A8010FCA909851882851983AA82AB8359
:1095E000120E40E9F8EE4F6053E50C60208E828F3A
:1095F00083A3A3A3A3A3E0D2E6F07402650C700DCD
:109600008E828F83A3A3A3A3A3E0D2E5F0850A8271
:10961000850B83A3A3A3A3A3A3A3A3A3A3E0A2E671
:10962000500D8E828F83A3A3A3A3A3E0D2E7F08E75
:10963000828F83A3A3A3A3A3A3E004F0E508700390
:10964000E8602BFC7D007A017B10121B0CEE4F6052
:10965000031296887408120A55E064FE7003A3E0B2
:10966000F4600B7408120A5512A020121CF4741630
:1096700002CB0FE50A2402FCE50B3400FD22EE24A8
:1096800017F582EF12DAD822E50A2402FAE50B3444
:1096900000FB120AEC2274FEF0A304F02274F7120D
:1096A000036374F71208A3EAFEEBFF900370E06413
:1096B00003600DE064016008E06409600302977DC7
:1096C0008E828F83A3E0600302975C7C007D007A2A
:1096D000027B00121B0CEE2402FAEF12A4D812C671
:1096E0005D12BDD77953121B547900129789E0643B
:1096F00009600990036E12C2F7120F668518828501
:109700001983740112BBAD9003707404F0740112DC
:109710000A55AA82AB83794A121B4E7401120A556C
:10972000AC82AD837A667B03121B2A900364E064EB
:10973000FE7003A3E0F4601179007401120A55ACC5
:1097400082AD8390036412978290035BE0A2E350A2
:1097500004D2F08002C2F012BB9A801E8E828F83E8
:10976000A3AE82AF83FC7D007A037B10121B0C8EAC
:10977000828F83E0F9129789E4F0120D3E7409029A
:10978000C7F61293B1120ABC2290036E1293B11263
:109790000B8290037022C082C08390033512AAF618
:1097A000701F900370E014600924FC600A14600CC0
:1097B000800F90033D8032900339802D90033B80D1
:1097C00028E8496008900336129BE1700C8A828B6E
:1097D00083A3E0F9120B6A801B90033612A25C701F
:1097E00005120EFA800E9003F212AAF6600612BB62
:1097F00077121CF402B778A3E08E828F832212D0F6
:109800000BE0682274F012036374EB1208A38A82DF
:109810008B83A3A3A3A378081209F878081209C8B8
:10982000900371780812097E75087F75097F7900A9
:10983000750C01750D00750E00750F00E9780C129E
:10984000077D900371780C12096BE50C450D450EF0
:10985000450F602778009003BC80118E828F83A310
:10986000A3E069700108EE241412842512A89870F0
:10987000EAE8C3950850048808890909E9C3941BDC
:1098800040AE8A828B83A3A3A3A3780C1209F8E5C8
:109890000C450D450E450F6064EA2404F8EB12B246
:1098A000B8120A32900371120A3E88828983120A22
:1098B00032851882851983120A3E7404120A55747F
:1098C00001F0900377E0C0E07405120A55D0E0F093
:1098D0007407120A55129A21806B90036E12C2F718
:1098E000120BAC8A0A8B0BA80AA90B90036EE8F046
:1098F000A3E912B68E687003A3E06960299003BCE7
:1099000012A89860218E828F831297FE7003A3E0C5
:1099100069700B8E828F83A3A3E0650960BCEE247F
:109920001412842580DAE509900363F0120D2CE906
:109930006013900370E4F090033F12AAF6600612E1
:10994000BB75121CF4741502CB0F74F4120363740C
:10995000EB1208A38A828B8312AB69E8FAE9FB79E0
:1099600000750801750900750A00750B00E9780893
:1099700012077D900371780812096B12BCDB602F0F
:109980008908EA250812DACB90114DE0C398501FE0
:10999000750801750900750A00750B00E978081251
:1099A000077D78081209C8900371780812097E09AA
:1099B000E9C3941B40AB90037178081209F812BCFC
:1099C000DB603D900371120A32851882851983127B
:1099D0000A3E7404120A557401F07407120A557491
:1099E00001F0900377E0C0E07405120A55D0E0F072
:1099F0007407120A55129A219003707406F0801CA5
:109A0000900370E4F0FCFD7A047B10121B0C9003B1
:109A10003F12AAF6600612BB75121CF4741502A060
:109A20002CE412C670121B662274F512036374D8FC
:109A30001208A38A088B098A828B83A3A3A312A985
:109A4000FF7415120A55AC82AD838A828B83A3A35F
:109A5000A3A3A3A3A312A9C612C2F2120D50741598
:109A6000120A55E0706B850882850983A3A3A3A31E
:109A7000A3A3A3A3E0C3940B40578E828F83A3A319
:109A8000A3A3A3A3A3A3E064027046EE240B129643
:109A900081F4703D900370E06402603AE064066017
:109AA0003590033512AAF66005129BE1604F9003D2
:109AB00070E064086005E0640470167417120A55BB
:109AC000E0F9741C120A55AC82AD8312C2EA120D81
:109AD00056742802DD8890033512AAF6701F7508A7
:109AE0000078081208007808120800EE241012848A
:109AF0002512D67D12A5E0129BFD12080F8E828FD3
:109B00008312C25912A51012AB727402120A5512B6
:109B1000BDD7EE240D129681C0E07404120A55D010
:109B2000E0129C06F508A3E0F509740F7808120A04
:109B3000077405120A55E508F07419120A55E0C0B9
:109B4000E07406120A55D0E0F0741B120A55E0C00A
:109B5000E07407120A55D0E0F07416120A55E0C0FE
:109B6000E07409120A55D0E0F07417120A55E0C0EB
:109B7000E07408120A55D0E0F0EE2410129681C06D
:109B8000E0740A120A55D0E0F0741A120A55E0C0C7
:109B9000E0740B120A55D0E0F07427120A55E0C0A9
:109BA000E0740C120A55D0E0F0741C120A55A98218
:109BB000AA8389088A09750A0078081207F87C08C0
:109BC0007D007410120A55AA82AB8312B64E120899
:109BD0000F851882851983AA82AB83120B7C029AA7
:109BE000D112A262640122E508240CF582E5091273
:109BF000AA2712A9CBA3A3A3A3A312C9751293B139
:109C0000120E28740222F012D65E12DAD72274F6EF
:109C100012036374C91208A39003EC12AAF660063B
:109C200012BB77121CF4900370E064087003029C6E
:109C3000C29003ADE06402702C9021BCE4939003C9
:109C400052F09021BCE493900350F0908053120A9C
:109C500032900379120A3E908053120A3290037DAB
:109C6000120A3E805D900381E0F874DE28F582746C
:109C70000B129DF7900352F074DF28F582740B12DB
:109C80008A00900350F07508FF7509FFEA78081202
:109C90000945E508F4FCE509F4FD3395E0FE900381
:109CA00079129DFC7508FF7509FFE9C39A780812BF
:109CB0000945E508F4FCE509F4FD3395E0FEA3123F
:109CC0009DFC851882851983E412BBB67904121BAA
:109CD00054900381E07009741E120A5574018006C5
:109CE000741E120A55E412AF17740FF090114C1243
:109CF000C2647946121B547401120A55E4F09011A3
:109D00008CE0C0E07402120A55D0E0F090035EE0EF
:109D1000C0E07403120A55D0E0F07404120A55E44E
:109D2000F07405120A55E4F07407120A55E4F09035
:109D30000381E0C3940F500CE0C0E07406120A5592
:109D4000D0E080077406120A55740FF07C827D0300
:109D50007408120A55AA82AB83121B2A7C037D0069
:109D600079FF7410120A55AA82AB8312131A90035A
:109D7000BAE0C0E07413120A55D0E012BD44740179
:109D8000120A5512BCCA120E2E900375E0C0E07480
:109D90001C120A55D0E0F0900376E0C0E0741D126A
:109DA0000A55D0E0F0900363E0C0E0741A120A553F
:109DB000D0E0F090036E12AB727418120A5512BD07
:109DC000D77420120A55E4F0900378E0C0E0741FC5
:109DD000120A55D0E0F07434120A55E4F0742912D6
:109DE0000A55E4129E077414120A55AA82AB831214
:109DF0001B6C743702BB9212DAD8FA22ECF0A3ED96
:109E0000F0A3EEF0A3F022F07A617B037953129E67
:109E10001222121B547A647B03794B121B5422C00A
:109E200082C0838A828B83A3E09003706004E4F095
:109E300080427408F0900381E0701A90033F12AAE8
:109E4000F66008790012BB77121CF490036E12A81A
:109E50003D7A05801A7900120B7690036112A83DB5
:109E60007A067B00121B0C90036412A83D7A047BD7
:109E700000121B0C02B77874F412036374EA120820
:109E8000A3EAFEEBFFEE24020A0AEF3400FB120AFB
:109E9000E08A088B09EA45097003029F378A828BA2
:109EA00083A3A3A3A3E0640160278A828B83A3A377
:109EB000A3A3E06402601A8A828B83A3A3A3A3E016
:109EC0006403600D8A828B83A3A3A3A3E064047060
:109ED00066EE2402FCEF3400FD851882851983129A
:109EE000C24B129F3C120A5512BDD7740A120A5572
:109EF0007401F07413120A55E412C264121B6089D3
:109F00000AAC0A7D007A077B00121B0C850882854B
:109F10000983A3A3A3A3A3E0C2E012C08EA3A3A3BB
:109F2000A3129F42120212E8850882850983A3A327
:109F3000A3A3A3A3A3A3F0741602A02C12AF33749F
:109F400008227401F012D68C2274F7120363900376
:109F5000BC12A4F88012EA2414F582EB12842812B1
:109F6000A9FF1213B6EEFAEFFBEA4B70E99003BCBF
:109F7000E4F0A3F002C7F974F4120363EAFEEBFF06
:109F8000EE24131296816403700DEE240BFAEF3465
:109F900000FB120AE0800CE06402707812D460EFDB
:109FA00012A0168A088B09E508450960678E828F22
:109FB00083A3E0700F850882850983A3A3A3A3A3CD
:109FC000A3E4804F64F1600A8E828F83A3E064E192
:109FD0007025850882850983A3A3A3A3A3A3E064B6
:109FE00001701485088285098312A020121CF4EEEA
:109FF000240BFAEF12968F850882850983A3A3A309
:10A00000A3A3A3E0600E850882850983A3A3A3A36D
:10A01000A3A314F0801912AA271293B1120ADA220C
:10A020001293B190034A12CBD222740312080F7F0D
:10A03000040205CA74F11203638A088B09ECFEED71
:10A04000FF890A8A828B8312CA678A828B8312975E
:10A05000F712A0F28A828B83A3A3E0C454F0FA889B
:10A06000828983E04A12A1021297F712A0FCE03322
:10A070003354FCF88E828F83E04812A0FCA3E033B7
:10A08000333354F8F88E828F83E04812A0F28508AB
:10A09000828B83A3A3A3A3A3A3E0A2E0E4331313BF
:10A0A000FA88828983E04AF0E5082407F50CEB1270
:10A0B000B6541207F87C0812B64812080F12CC2CBE
:10A0C000E508240FF50CE5093400F50D780C1207AE
:10A0D000F87C0312B64812080FE50AC3940F400D2E
:10A0E00012A1C01284281297F8A3A3A3F07F07023D
:10A0F00005CAF0EEF8EFF9A30EAF832212A102A376
:10A10000A322F08508828B83A3A32274F112036338
:10A11000EAFEEBFF890A8C088D098E828F83E08C22
:10A12000828D8312AE4EAE82AF83E012B71312B6A9
:10A130008DC412B71312A1C9E054038C828D83120F
:10A14000B68BA2E2E4338C828D8312B68A1313138A
:10A15000541F12B71312B689A2E7E4338C828D83A1
:10A16000A3A3A3A312A1C98E0C8F0D750E00780CAA
:10A170001207F87C087D00E508240712CBBE120800
:10A180000F12CC2C8E0C8F0D780C1207F87C037DEF
:10A1900000E508240F12CBBE12080FE50AC3940F86
:10A1A00040148E828F83A3A3A3E0C0E012A1C0124B
:10A1B0008428D0E0800612A1C012DABAF002A0ED25
:10A1C000E5082412F582E50922A3A312AE520EAFD0
:10A1D000832274F412036374F91208A3EAFEEBFFFE
:10A1E000890890033512AAF6600E12A25C7009EE7F
:10A1F000FAEFFB120EF4805F90036EE06E7003A323
:10A20000E06F70537401650860097A827B0312C1A4
:10A21000B470447A007B0212A74A8B0BEA450B709C
:10A2200036900371120A32851882851983120A3E0C
:10A23000900377E0C0E07404120A55D0E0F0740592
:10A24000120A557401F07406120A5512C262120BFA
:10A2500022E9609B120B28740702A02C12A26264F0
:10A2600002221292D0A3A3A3A3A3A3E022E0F902A7
:10A27000B778F002B77874F61203639003CEE070FB
:10A280001B7C0079017A007B00120D8CEA4B600C7C
:10A290008A828B8312AAF66003120CD202BB95C08D
:10A2A00082C08312A732401079FF120D86E9F89020
:10A2B00021CEE493C398500479018002790002B75B
:10A2C0007874F01203638A088B09890B750C008A75
:10A2D000828B83A3A3A3A3A3A3A3A3E0F9120D924C
:10A2E0008A0E8B0FAE0EAF0F750A01EE4F600302A0
:10A2F000A3A1850882850983A3A3A3A3A3A312A86E
:10A300003D850882850983A3A3A3A3A3A3A312B4B5
:10A310004A12C2F7120D7A8A0C8B0DAE0CAF0DEEFD
:10A320004F700302A4C98E828F83A3A3A3A3E4F07A
:10A33000A3F0E508240B12A4D5E0C0E0128422D0DB
:10A34000E0F0120E8EEE240CF582EF12C4F9E5084F
:10A35000240EF582E50912842812AB72EE240EF564
:10A3600082EF12BDD4750C01EE2406F8EF12A4D1D1
:10A37000547FF0A3E054FC12A50B5404600302A424
:10A380002690118512B39D740778081209458E82B4
:10A390008F83A3A3A3A3A3A3E04508F0A3E04509EB
:10A3A000F08E828F83A3A3A3A312A501740778085C
:10A3B000120A07E5085407F508E50B60798E828FCD
:10A3C00083A3A3A3A3A3A3A3A3A3740212B68E245F
:10A3D0000D12A4E0A2E2500B90035C12BEAEA3A348
:10A3E00012BDD7E508700302A498EE2406F8EF34F6
:10A3F00000F9E8FAE9FB8A828B83E0547FFCA3E052
:10A4000054FCFDE50824FFF508E434FFF509740762
:10A410007808120945EC4508F8ED4509F98A828B60
:10A420008312BDD780728E828F83A3A3A3A3A3A31D
:10A43000E0448002A3A0E5087005750A0080598EEB
:10A44000828F83A3A3A3A3A3A3E0542060121213BB
:10A4500026EA547F245F8E828F83A3A3A3A3802345
:10A460008E828F83A3A3A3A3A3A3E05410600A1238
:10A470001326EA540F240A80DD8E828F83A3A3A3C0
:10A48000A37401F0A3E412A510740412A7418B0970
:10A49000EA4509700312BB83E50CA2E0502E8E82C0
:10A4A0008F83A3A3A3A312C7DEF9EEFAEFFB120D6D
:10A4B00080E96018EE240C12842512AAF6600312BB
:10A4C000A4E9EEFAEFFB1213B6750A00A90A02CB53
:10A4D0001212BF8022FAE5093400FB8A828B8322A4
:10A4E00012A4E422128443E02212AA2112A4F02230
:10A4F00012A4F8FB1213B622E0FAA3E0228E828F98
:10A5000083A3A3E0F508A3E0F5092212D3ABE02270
:10A5100012BDE2A3A3A32274F412036374F712081A
:10A52000A37E00120D92EA4B700302A5D98A828B9A
:10A5300083A3A3A3A3A3A3A3A3A3E064066003022E
:10A54000A5D98A828B83A3A3A3A3A3A3A3E0FF8A95
:10A55000828B8312A5E8E0C0E07408120A55D0E0AF
:10A5600012A9F312C1C012BDD7120DB0EF5408608A
:10A570006685188285198312A83D7A007B00120D2A
:10A58000748B0BEA450B704F90036E12AB76121B67
:10A59000847C007D007A007B0080288E828F83126D
:10A5A000A9DDF47003A3E0F4602D90036E12A5E022
:10A5B00012C2F7121860E9641A601C7C007D00EE7C
:10A5C000FAEFFB120D748A0A8B0BAE0AAF0BEE4F3B
:10A5D00070C97900121B8A7E01EEF9740902A02C61
:10A5E00012A8418E828F832212C2FFA3A3A322C08E
:10A5F00082C083EA4B70059003CF80068A828B83EA
:10A60000A3A312A7F960258A828B83A3A3A3A3A384
:10A61000A3A3E0540860E5EC4D60158A828B831299
:10A62000A9DD6C7003A3E06D70D280047A007B001A
:10A6300002B77874F2120363EAFEEBFF890A8C0812
:10A640008D097A107B001213B0EA4B60408A828B2E
:10A6500083A3A3A3A3A3A3A3A3A3E412A9E1A3E5B4
:10A660000A12D019A312DD7E8A828B83A3A3A3A32F
:10A67000E4F0A312A9ED12A69012CE63EA240CF521
:10A6800082EB12DAC512A690A3A3F0A3F0028661B2
:10A69000A312A69522F08A828B832274F41203639C
:10A6A000EAFEEBFF89088C0A8D0BEE4F60547401B3
:10A6B000650870147901120D86E9F89021D1E493B0
:10A6C000C398500F7911806774046508702E12A723
:10A6D0003240F18E828F83A3A3A3A3A3A3A3A3A33A
:10A6E000E50812B67712CC0F8E828F83A3A3E4F015
:10A6F000A3F09003CF12AAF6601F800D74026508C4
:10A7000060D179C18029E0F8A31288D012A7F98816
:10A71000828983A3A370EF80039003CFEEF0A3EFB1
:10A7200012A7418B0BEA450B700312BB8379000221
:10A73000A02F7904120D86E9F89021CFE493C398F5
:10A7400022F012A746227A207B009003BBE0F91288
:10A75000147622C082C083E9F879009003CF801D6F
:10A760008A828B83A3A3A3A3A3A3A3A3A3E068606C
:10A770000574FF687001098A828B83A3A312A7F96D
:10A7800070DE02B77874F7120363EA4B700590032A
:10A79000CF80068A828B83A3A312A7F960248A82C2
:10A7A0008B83A3A3A3A3A3A3A3A3A3E06970E4EC57
:10A7B00060148A828B83E0240D12CCC5A2E240D3C0
:10A7C00080047A007B0002C7F9C082C0839003CF67
:10A7D00080068A828B83A3A312A7F960128A828BD8
:10A7E00083A3A3A3A3A3A3A3A3E06970E580047A32
:10A7F000007B0002B7783BF5831293B1EA4B22C08D
:10A8000082C0839003CF800688828983A3A312AA83
:10A81000F6601B88828983E0FCA3E0F5838C82E0EC
:10A820006A7003A3E06B70E0E8FAE9FB80047A0049
:10A830007B0002B778A908EE241212AA2412A841BC
:10A840002212A84522E0FCA3E0FD2274F212036369
:10A850008A0A8B0B8C0C8D0D750800750900EA4572
:10A860000B602E9003CF80068E828F83A3A312A845
:10A8700098601EAC0CAD0DEEFAEFFB850A82850BDD
:10A8800083121CF4E9640170DFEEF8EFF98808899F
:10A8900009AA08AB09028661E0FEA3E0FFEE4F22A1
:10A8A00079000207C174F71203639003CF12AB72F1
:10A8B0007C007D00800BE8FCE9FD8882898312AB77
:10A8C00070E8496030EA687002EB6970E99003CF84
:10A8D00012C2F7E86A7002E96B88828983A3A370C9
:10A8E0000812AB729003CF800912AB728C828D83F9
:10A8F000A3A312BDD702C7F974F7120363EAFEEBF4
:10A90000FFEE4F6015120DAA12AA0512AAF66003F7
:10A9100012A4E9EEFAEFFB1213B602C7F974F712AC
:10A9200003638A828B8312A9DDFCA3E0FD9003CF31
:10A9300012AB727508007E00803188828983A3A3E0
:10A94000A3A3A3A3A3A3A3E0640570180E88828920
:10A9500083E0FFA3E0F5838F82E06C7003A3E06DDA
:10A96000700205088882898312AB70E84970CB9029
:10A9700021CD12D8D350089021CC12D86D400F8A27
:10A98000828B83A3A3A3A37401F0A3E4800C9003A0
:10A990005CE0F812A9C6E8F0A3E912A9ED7405126B
:10A9A000A9E1E0440812A9F3F47003A3E0F4600EF7
:10A9B00090036E12C96E121B7EE9641A700579014C
:10A9C000121B8A02C7F9A312A9CB22E0F98A828B53
:10A9D00083A3A3A3A32212861BEB12AA2712A9FA10
:10A9E0002212A9E52212D021A3A3A3A32212A9E532
:10A9F000A3A32212A69512A9FA2212CBD6E022E036
:10AA0000FEA3E0FF228E828F83E0241C12A4E4FACE
:10AA1000A3E0FB1213B68E828F8312A4F012AA2138
:10AA200022EE240CF582EF3400F58322C082C0832D
:10AA3000EAFCEBFDEC4D700479058046EC24FBF557
:10AA400082ED34FFF58312AAF6700712AA85E0F4AE
:10AA5000600512133280E19003BBE0C0E012AA85CA
:10AA6000D0E0F09021D3E493F97AD17B0312136202
:10AA7000E96401700B7A007B2012BB8779008002A9
:10AA8000790402B778EC24FFF582ED34FFF58322D8
:10AA900074F4120363A2AFE433F508C2AF9003D19C
:10AAA00012A898603AEE24FBF582EF34FFF583128A
:10AAB000AAF67A007B209003BB600512BB8A800552
:10AAC000E0F912136EE4F50AF50B780A1207FCEEB2
:10AAD000FCEFFD7AD17B03121C80740212080FE593
:10AAE00008A2E092AFEEFAEFFB02A02F8E828F83D6
:10AAF000E0241C12843F12AAFB492212AF37E8223D
:10AB0000C082C08374E11208A3EA2413F582EB1219
:10AB10009684C0E07411120A55D0E012AF2A74096D
:10AB2000120A5512AF232404F8EB3400F9E8FCE9CB
:10AB3000FD8C828D8312AB72740B120A5512AF23F7
:10AB40002414F582EB129684C0E07412120A55D0D8
:10AB5000E0F0EA240EF582EB128A008C828D8312DB
:10AB6000AB76120C78741F801DA3A3A3A3A3A3A389
:10AB7000A3A312AF332212A841851882851983AA94
:10AB800082AB8322740212080F02B77874F01203AA
:10AB90006374FC1208A3EAFEEBFF750B00750A0054
:10ABA0007508FE7509FF120D62E96005791102AEA4
:10ABB00025EE2415129681603D90119EE0C4335419
:10ABC000E0F8E0333354FC48C0E0EE24151284254D
:10ABD000D0E012AE4E12AE398B0DEA450D60147501
:10ABE0000B017508FFEE240F129681440412BDEF8D
:10ABF000D2E0F0750A408E828F8312863A6006EEAC
:10AC0000241212DAC2EE241312968170109021DD04
:10AC1000E493C0E0EE2413128425D0E0F08E828FFE
:10AC200083E0A2E750045403801CEE2414129681A2
:10AC3000701590034DE0C0E0EE2414128425D0E09E
:10AC4000F090034DE004F0EE24111296816401703F
:10AC500016900AF5E0600D900358E0700A8E828F1E
:10AC600083E0700312DABF90035BE0A2E1504AE593
:10AC70000BA2E040188E828F8312863A603B8E8250
:10AC80008F83E06008EE240B128623602CEE240FE5
:10AC900012968154406015EE24131296816401705F
:10ACA0000BEE240F12968154FBF0800DEEFAEFFBB1
:10ACB000120DC8E9700302ABAC8E828F83E0640191
:10ACC000700E12D460EF12A9DA6402700312AE3172
:10ACD000EE240F1296815440600302AD92E50BA260
:10ACE000E0500302AD9290035BE0A2E1400302ADAD
:10ACF00092E50AF50B780B120800EE2406FCEF34FF
:10AD000000FD8E828F8312C2F5EE24121289FD128D
:10AD10000CA2740112080FE96009EE241212B65E4B
:10AD200012AE2A8E828F83A3A3A3A3A3A3E0603EC7
:10AD3000EE2402F50CEF3400F50D850C82128A0723
:10AD40002407FAEF3400FB120DEC8A088B09850CFE
:10AD500082850D83E065087004A3E06509700C8EA0
:10AD6000828F83A3A3A3A3A3A3E4F012AE318E82A8
:10AD70008F83E064016008A90A12AE43120C3CA95B
:10AD80000A8E828F8312AE43120BD0E96004EE125A
:10AD9000AE2A851882851983AC82AD83EEFAEFFB6B
:10ADA000120DE08A0A8B0B74FE6508700474FF654F
:10ADB00009700312A4FDEA450B60668E828F83E062
:10ADC000C0E07401120A55D0E0F07402120A551264
:10ADD000CE637401120A5585820C85830D780C129E
:10ADE00007FCEE240F128425120699EE240E12960B
:10ADF00081F50C780C120800900361120699740713
:10AE0000120A55E0F9AC08AD09120DDA7407120800
:10AE10000FE9FE74106E700BAA0AAB0B1213B6800A
:10AE2000027E10EEF9740402CB0F12DAD34420F044
:10AE300022EE12DAD34440F022A31293B179FF122A
:10AE40001BC022A3A3A3A312C7EA1293B12212AE7E
:10AE50005222F08E828F83A322C082C08374DE12BE
:10AE600008A38A828B8312AB6E740E120A55E8F027
:10AE7000A3E912AF2A740C120A5512AF23240DF560
:10AE800082EB129684C0E0741A120A55D0E0F0EA00
:10AE900012D461EB12842812AB727420120A55127C
:10AEA000AF232415F582EB129684C0E07408120AD1
:10AEB00055D0E0F0EA241CF582EB12842812AB7224
:10AEC0007412120A5512AF232411F582EB129684E4
:10AED000C0E07409120A55D0E012AF1774FFF07485
:10AEE00001120A5574FFF07402120A5574FFF090B3
:10AEF00080631206957404120A55AC82AD83740700
:10AF0000120A55AA82AB83120B64740412080F79DB
:10AF100000742202AB86A312AF1B22F08518828533
:10AF2000198322E8F0A3E9F0EA2212A695A312AF52
:10AF30003222A312AF3722E0F8A3E0F92274EA121A
:10AF4000036374EE1208A38A148B15ECFEEDFF89DF
:10AF50000E7428120A5512B0B8742A120A55E0F578
:10AF60000F742B120A5512A503742D120A55E0F521
:10AF700012A3E0F513750A107A1E7B001213B07449
:10AF800002120A5512C4FD7402120A5512AAF67072
:10AF90000302B0AC750B00EEFAEFFB120ADA8A106E
:10AFA0008B11A810A911E849602688828983A3A380
:10AFB000A3A3E06401600D88828983A3A3A3A3E017
:10AFC0006403700CE5085440700674044509F509E3
:10AFD000E50954046003750B01851882851983AA5D
:10AFE00082AB83795012B96712C2F77402120A5504
:10AFF00012A5E8A312C4FD7410120A5512D3B3F0BF
:10B000007402120A55E0240B12843B7402F0120AF7
:10B010005512A5E87402F0120A5512CBCE12CE6377
:10B020007402120A55E0241B12843BE50EF07402F0
:10B03000120A55E0240C12843BE50FF07402120A48
:10B0400055E0241C12843BE514F0A3E515F07408C8
:10B05000120A5512DD80740A120A55E50FF08512A6
:10B0600082851383C082C083740D120A55AC82ADF1
:10B0700083D083D082740312073DA90B7402120A95
:10B0800055AA82AB83120D68E964017017E50BA223
:10B09000E0500CA90F120D92EA4B6003120DB67529
:10B0A0000A0080087402120A5512A4ECA90A74124C
:10B0B00012080F7F0E0205CAE0F50CA3E0F50D2281
:10B0C00074EE120363EAFEEBFF8C088D098E828F0B
:10B0D00083A3740812BED2E060088E828F83A374AB
:10B0E00010F012967E60098E828F83A3E02408F010
:10B0F000EE241512968160088E828F83A3E004F0FF
:10B100008E828F83A3A3A3A3A3A3E060198E828F53
:10B1100083A3A3A3A3A3A3A3E0C3332402F88E8233
:10B120008F83A3E028F0EE24111296816005750B41
:10B130000E8003750B008E828F83A3C082C083EEC6
:10B14000240D129681D083D082F8E028250B8C82C2
:10B150008D83F0EE2411129681600512B66528F0F9
:10B16000850882850983E0C39475400975080075D8
:10B17000090002B29E12B2C48A088B09EA4509701E
:10B180000302B29EEEFAEFFB120DE6EA8508828515
:10B19000098312C4FE12B2B312B44212B2E6F0EE48
:10B1A0002404080812B2B712B8A3A312B2E6A3A3EC
:10B1B000F0EE241312B2CCF0EE241412B2CCA3F0B1
:10B1C000750A08EE24161296816010EE241812A853
:10B1D0003AE508240812D664750A1012967E6016A5
:10B1E000EE241A12A83A850A0CE508250C12D6643A
:10B1F0007408250AF50A8E828F83A3A3A3A3A3A3B1
:10B20000E06058EE2407F510EF3400F51185108248
:10B21000F583E0C0E012B2A7128428D0E012B2D6C3
:10B22000E0C0E012B2A7128428D0E012B2D6129287
:10B23000F21207F8851082851183E0C333FCE433F2
:10B24000FD850A0CE508250C12CBBE12080F8510EF
:10B2500082851183E0C333250AF50AEE2415129680
:10B2600081600BC0E012B2A7128428D0E0F01284F3
:10B27000221292F31207F8EE240D129681FC7D0043
:10B28000850B0A8E828F83A3E0F8E50828F8E5098C
:10B290003400F9E8250AFAE912CBC112080FAA080E
:10B2A000AB097F0A0205CA850A0CE508250CF58260
:10B2B000E50922EE2402F8EF12B2BC223400F9882C
:10B2C00082898322E0FA7B001213B02212AA241290
:10B2D000B2F0A3A3A322F0050A8E828F83A3A3A3B7
:10B2E000A3A3A3A3A322A3A312D3ABA312B2F022BE
:10B2F00012B8A7A3A32274F61203638A828B83E099
:10B30000FC90035E12B39D74027808120945EC4567
:10B3100008FCAD09EA241212B397740678081209E2
:10B3200045EC4508FCED4509FDEA2415F582EB12D4
:10B3300096846004780180027800E4C8F9ED49FD44
:10B34000EA2411F582EB129684F5088809740978CD
:10B3500008120945ED4509FDEA241612B397740B4E
:10B360007808120945ED4509FDEA241712B39774D0
:10B370000C7808120945ED4509FD8A828B83A3A349
:10B38000A3A3A3A312B39D740A7808120945ECFA8B
:10B39000ED4509FB02BB95F582EB12AA27E0F50803
:10B3A0007509002274F412036374FD1208A38A085D
:10B3B0008B09ECFEEDFF7401120A5585820A858324
:10B3C0000B780A1207FC7402120A55AC82AD83EEA8
:10B3D000FAEFFB120C18740212080FE9705D851861
:10B3E0008285198312B442F07401120A55E0F812F2
:10B3F000B44AA3A312BDD7851882851983E0602DB6
:10B400001485088285098312AF16E0C333F8E4334C
:10B41000F97401120A55E028F8A3E039F9E824FE8E
:10B42000F582E934FFF58312A4F8FB8012850882C7
:10B43000850983A3E4F0EEFAEF80EF7AFE7BFF024A
:10B44000A02AE085088285098322A3E0F985088285
:10B450008509832274EE1203638A0A8B0BECFEEDDE
:10B46000FF750F01E9C394085005790002B6458EB7
:10B47000828F83E912A69112B8CCE96003750F00A0
:10B4800012B8B08E828F8312B8F612D460EF12B861
:10B49000EBC0E0EE2411128425D0E012B8E3C0E046
:10B4A000EE2412128425D0E012AE4E740812B67744
:10B4B000A3A3A3E0601512B898EE2413F582EF124F
:10B4C000BDD48E828F83A3E02408F08E828F83A365
:10B4D000A3A3A3A3A3A3A3E060218E828F83A3854C
:10B4E000820885830912B8D7EE2415F582EF12BDC4
:10B4F000D4850882850983E02408F08E828F83A397
:10B50000A3A3A3A3E0601A8E828F83A385820885FC
:10B51000830912B8BF8E828F83A3A3A3A3A312B6FD
:10B520007EEE241912B65E241B12DAC2A312BECA22
:10B53000E0700302B5DBEE2419F8EF3400F98E82D7
:10B540008F83A3858208858309E0FAE50A2AF582BC
:10B55000E50B1296848882898312B67EFAE50A2A60
:10B56000F582E50B129684C0E0EE241A128425D0F1
:10B57000E012B67E88828983E06059F89021D2E497
:10B5800093C398500575110C8008EE24191296810A
:10B59000F5118E828F83A3E0F8E50A28F50CE50B00
:10B5A00012B6541207F8E511C333FCE433FD7A7286
:10B5B0007B1012B64E12080FEE241B1284257472F3
:10B5C000F0A37410F0E511C333F885088285098370
:10B5D000E0288006EE241812DAB7F08E828F83A35B
:10B5E000E0F88E828F83E0C398500302B46AA3E030
:10B5F000FA8A08E50A2508F8E50B3400F912861ADC
:10B60000EF12C07512B68EC39AC0E0EE24171284F2
:10B6100025D0E012BDDD602BEE2417F8EF3400F9E1
:10B62000880889098882F583E024F212BF76240E07
:10B63000FAA3E03400FB8882898312C4FD12B66548
:10B64000C398F0A90F02B2A27D00EEFAEFFB12132D
:10B650000E7403223400F50D750E00780C2212AA28
:10B6600024E4F0EE22900359E0F9121C5CE9F8851D
:10B670000882850983E02212AE52A3A3A322F0859B
:10B680000882850983E004F022A3A3A3A3A3F08E7C
:10B69000828F83E02274F41203638A088B09EA1212
:10B6A000B71AF0EA1313543F12B713A3A3A3F0EA97
:10B6B000C4131312B71AA3A3F0EB12B72512B72DB8
:10B6C0007409780A120A0712B72312B72C740A7881
:10B6D0000A120A07E50A5401C0E0EC2418F582EDCD
:10B6E000128428D0E012B732740B780A120A0712BB
:10B6F000B723A312B72C740C780A120A0712B723C7
:10B70000A3A3A3A3A3A3A3A3F0740D7808120A070D
:10B710000289F8540F8C828D832254038C828D838E
:10B72000A3A322E50A54018C828D8322A3A3A3A3A1
:10B73000A3A3F08A0A8B0B22C082C08379008A827D
:10B740008B83A3A3A3A3A3A3E0900358600FE0708F
:10B75000228A828B83A3A3E07019098016E060130C
:10B760008A828B8312C2EE900361E06A7003A3E0C9
:10B770006B70E7800312C2F7D083D0820207C174D6
:10B78000F01203638A0A8B0B890C8C088D098A825C
:10B790008B8312B8CC12B8B085088285098312B8A1
:10B7A000F6E50812D461E50912B8EBC0E0E508241B
:10B7B00011F582E509128428D0E012B8E3C0E01246
:10B7C000A1C0128428D0E012C07D740812C0A76006
:10B7D0001112B898E508241312C07112C07DE0243C
:10B7E00008F0850882850983A3A3A3A3A3A3A3A329
:10B7F000E06017850882850983A312B8D3E5082481
:10B800001512C07112B68E2408F08508828509834E
:10B81000A3A3A3A3A3E06019850882850983A3AE2F
:10B8200082AF8312B8BF85088285098312B6890466
:10B83000F0AA08AB09120DFEE9F50D7056850882D5
:10B84000850983A3A3A3A3A3A312B8A37014E0FA4A
:10B850008A0EE50A250EF8E50B12BDC9E50CC39A60
:10B86000802112B8D3E8240EF8E912BDC99003591B
:10B87000E0F9121C5C8E828F83E0F8E50CC39824FB
:10B88000F2C399C0E0E5082417F582E5091284287F
:10B89000D0E0F0A90D02CB12E50A2408F8E50B343C
:10B8A00000F92212B8A722E0850882850983A32225
:10B8B000850A82850B83A3A312B90CE0F9EA22E082
:10B8C000F8E50A28F582E50B12DAD82212CB171216
:10B8D0000DF822AE82AF83E0F8E50A28F8E50B34D4
:10B8E00000F92212B91FA3A3A3E02212AA27E8128B
:10B8F000B918A3A3E022A3A3A3A3A3A3A3A3A31262
:10B90000B91812B90CA3A3E0F9EAF822E0FA850A03
:10B9100082850B83A3A3A322F0A3E912B91F22F00F
:10B92000850A82850B83A3A3A3A322C082C0837A46
:10B93000DF7B0379E2121B4E7ADF7B0302B778C00C
:10B9400082C08390036102B775C082C08374FE1207
:10B9500008A3851882851983AA82AB83794B12B913
:10B960006712C2F702AB84121B4E851882851983B9
:10B9700022C082C083794A121B4E02B77874F61235
:10B9800003639003E7E0FE04F0EEF9120D928B09D9
:10B99000EA450970EDEE60EAF902BB9574EC12031A
:10B9A00063EAFEEBFF8C128D13890A7414120A5598
:10B9B000E0F50E7415120A55E0F50B750C00750DC7
:10B9C00000120F6C8A088B09EA45097017E50B60B5
:10B9D0000302BAA5A90AAC12AD13EEFAEFFB120FDF
:10B9E0009002BB73E50A6021EA2402F582EB12960D
:10B9F00084850A102510F8E4340013E813F0700968
:10BA00008A828B83A3A37401F0E50B700302BA93BF
:10BA10009003F412AAF6600612BB77121CF4E50E2E
:10BA2000700E850882850983E4F0750D0102BABEA7
:10BA300090035BE0A2E1400302BAC69003F612AAAB
:10BA4000F6600CA90EAA08AB0912BB77121CF4858C
:10BA50000882850983E0FA12D694EA98E499C365CE
:10BA6000D033500A850882850983E02401F08508D7
:10BA700082850983E0F89021D4E493687040750CC6
:10BA800001EEFAEFFB120CB4850882850983A3E46A
:10BA9000F0802B8A828B83A3A3E0F89011A8E0C3E7
:10BAA00098501B80857401650B7013E50A600F9038
:10BAB000035BE0A2E15015EEFAEFFB120CB4900329
:10BAC0005BE0A2E140227401650B701CE50E90035F
:10BAD000F86013E004F0901186E0F89003F8E0C3FA
:10BAE000984005750C01E4F0E50CA2E0C0D0E50D2E
:10BAF000A2E092F0120932158172F0507690035B49
:10BB0000E0A2E15039EEFAEFFB120ADA8A088B095B
:10BB1000A808A909E8496026E50DA2E0500D888231
:10BB20008983A3A3A3A3A3E0C2E0F0E50CA2E050A5
:10BB30004288828983A3A3A3A3A3E0D2E0F0E50C0B
:10BB4000A2E0502F90035BE0A2E15012EEFAEFFB6F
:10BB5000120AC8E96008EEFAEFFB79008012900340
:10BB600064E06E7003A3E06F7009EEFAEFFB7901F9
:10BB7000120B9A800979C41292D02212080F7F0CFE
:10BB80000205CA7A207B009003BBE0F912136822F9
:10BB9000740112080F7F020205CAA2F0E43385186F
:10BBA0008285198312BBB67952121B542212BBB67E
:10BBB0007942121B5422F0AA82AB832274F412033E
:10BBC0006374EC1208A37401120A55AC82AD83129F
:10BBD000BD379003ADE0640270627405120A55E44B
:10BBE000F07407120A55E4F07A04F9120AB012D27E
:10BBF000CFEA98EB99507D120AA4E970779021C89A
:10BC000012BCE4600F7A047903120AB09021C812C2
:10BC1000BCEA50087405120A557401F09021CA124A
:10BC2000BCE4600F7A027901120AB09021CA12BCFA
:10BC3000EA50417407120A557401803790037978ED
:10BC4000081209F812BCDB600474018001E4C0E052
:10BC50007405120A55D0E0F090037D78081209F8B7
:10BC600012BCDB600474018001E4C0E07407120AB6
:10BC700055D0E0F090114CE0F97CBE7D03740112C8
:10BC80000A5512BCCA7407120A55E07011740512E5
:10BC90000A55E07009851882851983E480088518A3
:10BCA000828519837401F090114AE07583117582C1
:10BCB0004BF8E058F8851882851983E05812BBB616
:10BCC0007941121B54741402A02CAA82AB83120D6A
:10BCD0004A7ABE7B037945121B5422E50845094583
:10BCE0000A450B2212BD03E8492212BD03758321C8
:10BCF0007582BCE493C398F8A3E49399F9C3EA98D6
:10BD0000EB9922E493F8740193F92274F712036318
:10BD100074ED1208A3E9FE9003BA12C30E12BD37E8
:10BD20007412120A55EE12BD4485188285198312C9
:10BD3000BCCA741302C7F690114CE0F97ABE7B03BB
:10BD4000120D5022F090114CE0F97CBE7D0322745C
:10BD5000F4120363EAFEEBFF90114EE064FE700301
:10BD6000A3E0F470547A1612BF5F604D8A828B8311
:10BD7000740112BDDD8A828B83A360047402800289
:10BD8000740112C2688A828B83A3A3A3A3A3A3A373
:10BD9000A3A312BDEEFCA3E0FDEA24020A0AEB1203
:10BDA000D667E5082413F582E50912DAC512BDBC91
:10BDB00012842212C61912BDD702A02FAA08AB09FD
:10BDC0009003BBE0F9121338223400F9E508241D72
:10BDD000F582E50912AA27E8F0A3E9F02212BDE2F4
:10BDE000E022F08E828F83A3A3A3A3A3A322A3F0B8
:10BDF000EE241512DAD52274F212036374FD1208D0
:10BE0000A38A088B09890A8C0B7401120A557404E1
:10BE100012C0AE8A0C8B0DAE0CAF0DEE4F607912D6
:10BE2000D66E7407F0A3A882A983E508240812A49B
:10BE3000D512BEBF8A828B8312BEBE850882850959
:10BE400083A3A3A3A3A3A3A3A3A3A3E0888289831B
:10BE500012BED2740112BECA12DD8012C0B9EE2425
:10BE600013F582EF12CA61650A60067401650A70F3
:10BE70000712BEA37404800412BEA3E4F090114E16
:10BE800012BEAE12BDD77401650B700312DABFEE9D
:10BE9000FAEFFB120B168002791090114E12969653
:10BEA00002865CEE240F12AA247440F0A322E0F86C
:10BEB000A312BEB522E0F98E828F83A3A322A3E052
:10BEC00088828983F0A308A98322F0EE241812AA9D
:10BED0002422F0EE241612AA242274F4120363EA38
:10BEE000FEEBFF7A007B041282E712BF6C12BDD713
:10BEF0009003707409F0120E0A8A088B09AC08AD21
:10BF000009EE241312842512C2F712C1B464017021
:10BF10004B7A0F12BF5F60448A828B83740212BF18
:10BF200076FAA3E0FB8A828B83A3E0FC8A828B8370
:10BF3000A3A3E0FBEC850882850983A3A312C4FEBA
:10BF40008882898312CBCEA3A3A312B44212BDEE82
:10BF5000FAA3E0FB794A121B5412BDBC02A02F7B4E
:10BF60000012132C8A088B09EA4509229003371224
:10BF7000AF3390118122F0EE241DF8EF12BF802222
:10BF800012B2BCE02274F412036374FD1208A38A97
:10BF9000088B097401120A55740212C0AE8A0A8B0A
:10BFA0000BAE0AAF0BEE4F700302C05D12D66E747B
:10BFB00004F0A3E412C07DA3A3A3E0640170088889
:10BFC000828983A37420F0850882850983A3A3A3B3
:10BFD000A3A3E06401700988828983A3E0D2E6F01C
:10BFE000850882850983A3A3A3A3A3A3E0640170AA
:10BFF0000A88828983A3E0D2E78006EE241312DE4A
:10C000003E12C08EE06401700AEE241612C09A241B
:10C01000188008EE241712C09A241AF582EF12C075
:10C020007512C0A764017009EE240F12C062A3E468
:10C03000F085088285098312863C6009EE240F1280
:10C0400096814404F012C0B985088285098312BE26
:10C05000AE12BDD7EEFAEFFB120B1680027910027A
:10C06000A02AF582EF12C069223400F5837401F032
:10C0700022F582E50912AA27E8F0A3E92212C0817D
:10C080002212C08522F0850882850983A32212C06E
:10C09000922212C085A3A3A3A32212AA2474011280
:10C0A000C08112AF32EE2212C092A3A3E02212C0CE
:10C0B000B22212C674120E6A22EE2417F582EF1213
:10C0C000C069120E0AEE241A12AA24EAF0A3EBF0B9
:10C0D0002274F412036374F31208A38908EAFEEBD6
:10C0E000FF7C0D7D007900851882851983AA82ABBB
:10C0F0008312131A12861AEF12DACE12C1B9F8742B
:10C100001F58600A7901121B12790002C1ABE8A224
:10C11000E55008740C120A557401F0E8A2E75008C3
:10C12000740B120A557401F0E8A2E6740A50081262
:10C130000A557401F08008120A55E064017005EE9A
:10C1400024138003EE241512A83A7402120A55AA89
:10C1500082AB83121B2A12842212C1BF12BDD77474
:10C160000A120A55E06401703312862F703B120EDA
:10C17000168A0A8B0BA80AA90BEE240B129681686B
:10C180007003A3E0697022120E0AEAFCEBFD740250
:10C19000120A55AA82AB8312C1B4600D851882853C
:10C1A0001983AA82AB83120B94A908740D02A02CE8
:10C1B000EEFAEFFB121B24E9221292CFA3E022E059
:10C1C00012C1C422F8A3E0F985188285198322746C
:10C1D000F612036374F31208A38A088B09ECFEEDD0
:10C1E000FF7C0D7D007900851882851983AA82ABBA
:10C1F0008312D89AA3A3A3A3A3A3A3A3A312C25950
:10C2000012C268F8A2E55008740B120A557401F0C6
:10C21000E8A2E75008740A120A557401F0E8A2E691
:10C22000EE500424138002241512A83A7402120A54
:10C230005512C24BA3A3E0C0E0740C120A55D0E023
:10C2400012C264120B8E740D02BB92AA82AB8312CF
:10C250001B2A85088285098322E012C1C4E8F0A365
:10C26000E922740212C67022F0EE241D12AA2412D2
:10C27000CBD2A3E02274F712036374E11208A3EA9D
:10C28000FEEBFF8E828F8312C2FBA3E0A2E0505729
:10C290008E828F83A3E0F9E8FAE9FB8A828B83A37D
:10C2A000A3A3A3A3A3E054FE12C30E8A828B83E050
:10C2B000241B12A4E0F98A828B83E0241CFAA3E0F9
:10C2C00012A4D812C2F7120E04E9701B741D120AD0
:10C2D0005512C3087011851882851983AC82AD830D
:10C2E000EEFAEFFB120E5802C7F48E828F83A3A3DF
:10C2F000A3A3A3A3A3A3A31293B12212C2FF22124A
:10C30000CBD6A3A3A3A3A32212A9FA64042212AF3B
:10C310001BAC82AD8322E9F87900740468600A746A
:10C320000A6860057403687001090207C174F61297
:10C3300003638A828B837420F0A3A37401F0120B31
:10C340001C8A088B09AE08AF09EE4F60108E828FF1
:10C35000837401F09003AEE0700312C0B9EEFAEFFF
:10C36000FB02BB95C082C08390114D02A26DC082BA
:10C37000C083E990114D02A272C082C0839003D3A2
:10C380007401F0E9A2E350037403F0E9A2E1500460
:10C39000E0D2E2F002B77874F612036379007C0011
:10C3A0008A088B097808120610F8FF07CAC3C8C3A9
:10C3B000C8C3C8C3C8C3C1C3C5C3CAC3BEC30C8036
:10C3C000097C0480050C80F67C089003D3E05C6057
:10C3D00003098003EC60010902BB9574F412036346
:10C3E000EAFEEBFF8908120AE08A0A8B0BA80AA969
:10C3F0000BE849604088828983A3A3A3A3E014C308
:10C400009404503174016508601A88828983A3A35B
:10C41000A3A3E06401600D88828983A3A3A3A3E0A2
:10C420006402700A8882898312A020121CF4EEFA3A
:10C43000EFFB120AEC02A02F74F61203638A828BC0
:10C4400083E07012A312AAF6600C8A828B8312C258
:10C45000F6121CAA80047A007B0002BB95C082C041
:10C46000839003ADE06402700B900370E064087089
:10C4700003120EA002B778C082C0837C0012C4E50C
:10C480006A7003A3E06B70119021D8E493C0E012AE
:10C49000DAE3D0E0F079C580490CECC3940340DDC9
:10C4A0007C0012C4E564FE7003A3E0F47015EC1286
:10C4B000D71C12C4FD9021D8E49388828983F07937
:10C4C00000801F0CECC3940340D87C00EC75F00393
:10C4D000A4F8A9F012DADE60D50CECC3940340ECAA
:10C4E00079C702B778EC75F003A4F8A9F074D728DF
:10C4F000F582740339F583E0223400F583EAF0A372
:10C50000EBF02274F212036374DD1208A3EAFEEB6F
:10C51000FF750A00900361E06E7003A3E06F701E68
:10C52000EE4F700302C6099003E812AAF6700302E8
:10C53000C609750A0112BB77121CF402C612120A50
:10C54000DA8A088B09EA4509700302C6098A828BD8
:10C5500083A3A3A3A3E0640160108A828B83A3A3B7
:10C56000A3A3E06402600302C609851882851983CB
:10C57000E412AF2A740B120A5512C668120A98E91F
:10C58000700302C60985088285098312C61912BD87
:10C59000D77900120BFA85088285098312C4FD74CD
:10C5A00003120A55AC82AD83740D120A5512C24BA8
:10C5B00012AB727415120A5512BDD77417120A55B0
:10C5C000E4F07C02850882850983A3A3A3A3E0F994
:10C5D000740D120A55AA82AB83120E40850882851B
:10C5E000098312AB727401120A5512C668120A9EB0
:10C5F000750A01908063120A32E508240CF582E581
:10C6000009128428120A3E800990036E12D0121279
:10C610000F54A90A742302865E12AF3390114E2282
:10C62000C082C08374FE1208A3790190034612CB26
:10C63000CE121CF485188285198312C4FD851882D8
:10C6400085198312C65D12C6687953121B5485186A
:10C650008285198312C2F71215FC02AB8412C661DF
:10C660002212AF3790036122E8F0A3E912C67022CC
:10C6700012C6742212AF1BAA82AB832274F5120376
:10C680006374F31208A38A088B09ECFEEDFF750AA8
:10C6900012EA45097005790002C75E900361E06502
:10C6A000087004A3E065097014120E0AEAFCEBFDA1
:10C6B00012C1B07005750A018003750A00851882E1
:10C6C000851983E4F004120A5512DD8085188285ED
:10C6D0001983AA82AB83120A8CE960277403120AB9
:10C6E00055AA82AB83120A6EE964017016750A01BD
:10C6F0007403120A55AC82AD8312C1B06021750A71
:10C7000000801C7412650A70169003ADE06402701C
:10C710000EEEFCEFFDAA08AB09120AC2E970DFEECB
:10C72000FCEFFDAA08AB09120F72E9F8740A6870F1
:10C7300005750A01801D74A0687012EEFCEFFDAA59
:10C7400008AB09120F84AA08AB09120F9C7401658B
:10C750000A70097900AA08AB09120EB2A90A740D71
:10C7600002DD8874F6120363EAFEEBFF8908120EFD
:10C77000A0E508F5097809120800790DEEFCEFFD37
:10C780007AFC7BFF120EBE02BB9074F7120363EAC1
:10C79000FEEBFF8E828F83A3A3A3A3A3A3A3A3E097
:10C7A0006015EE24151284251293A2120EACE964D2
:10C7B000017004790180258E828F83A3A3A3A3A394
:10C7C000A3A3E06015EE241312842512C7DEFAA39A
:10C7D000E0FB120EACE9640160D97900801B12C73E
:10C7E000EAA3A3A3A3A3A3A3E02212A8458E828F4A
:10C7F00083A3A322741F12080F7F010205CA74F0DD
:10C8000012036374FD1208A38A088B09ECFEEDFF86
:10C81000890B7413120A55E0F50C750A01740112A4
:10C820000A55740412D4656049E50C601DEA2417AA
:10C83000F582EB12DABA12D0288A828B83E0D2E733
:10C84000F0EA2414F582EB12DAC5EA12D461EB1295
:10C85000D672740312CC11EE88828983A3A3F0EF01
:10C8600088828983A3A312A69012DD7E120B16E99B
:10C87000F50AA90A740302CB0F74F2120363EAFEED
:10C88000EBFF890A750B01EE241D1284251288CD59
:10C89000E0FA88828983A3A3A3E0F9EA2400F508DB
:10C8A000E439F50912967E640460087901121B12BE
:10C8B00002C969EE241D12842512C1B91206F102C3
:10C8C0000002D4C8030B42C9030C3AC90D27C90E94
:10C8D00042C93FC97900AB09120C90EA4B603D8A0E
:10C8E000828B83A3A3A3A3A3A3E05418602E128476
:10C8F000221206998A828B83A3A312069979008E4D
:10C90000828F83A3A3A3A3A3A3A3A3A312C96E127D
:10C910000CAE740412080F750B0080267901AA086A
:10C92000AB09120BA0801BAB09120E94AA08AB092D
:10C93000120E9AE964C5700A80DD12162080037514
:10C940000A0012862F6022EE2411129681C39402EF
:10C95000401712842212CF847003A3E069600AE5B5
:10C960000BA2E05004A90A8002790002866112C974
:10C97000751293B12212A8458A828B832274EC121D
:10C98000036374F51208A38A0A8B0B890C8C0E8D35
:10C990000F741F120A55E0F50D7420120A55E0F5C8
:10C9A00010A3E0F5117E01EE120A55740AF0E97049
:10C9B00007E50DC333240AF012CBDF700302CA5A15
:10C9C00012CBF47409F0A3E50CC43354E0450D1206
:10C9D000CC17E50C702D7C008023ECC333F8E433D6
:10C9E000F9E51028F8E51139F98882898312CA67B8
:10C9F000888289831297F7F0A30EAF830CECC3955E
:10CA00000D40D7E5082417F582E50912C065120E1E
:10CA10000AE508241AF582E50912C4F97403120A1A
:10CA200055AC82AD83AA0AAB0B120A74E96019E512
:10CA3000082416F582E50912CA61120A55A882A9CE
:10CA400083E508241812BDD085088285098312CC9D
:10CA50000DAA08AB09120B16E9FEEEF9740B02BB26
:10CA60007B12C069740322E08E828F83F0A3AE82B2
:10CA7000AF832274F012036374F81208A38A088B40
:10CA80000912CCB3F50A74E058F50BA3AE82AF835C
:10CA900012CC856078E50B706FE50AC333FA7B0032
:10CAA0001213B08A0C8B0DEA450D60617C00802268
:10CAB0008E828F8312CB17EC33F8E433F9E50C2820
:10CAC000F582E50D3912C4FBEE24020E0EEF3400A0
:10CAD000FF0CECC3950A40D8780C1207FC780A12B8
:10CAE00008007403120A55AC82AD837900E5081280
:10CAF000D461E50912842812CF70740312080FAABA
:10CB00000CAB0D1213B680057901121B12740812BA
:10CB1000080F7F080205CA12A4F8F9EA2400E439D4
:10CB2000FB2274EE1203638A0C8B0D890E8C088D28
:10CB3000097412120A55E0F50F7413120A5512CC3B
:10CB400005900A6712AAF66072E50FC333F8E43362
:10CB5000F9E8240EFAE93400FB12132C8A108B1129
:10CB6000AE10AF11EE4F60538E828F8374D4F012EB
:10CB7000D3B112B677E50EF0AC08AD09EE2405FA94
:10CB8000EF12D667EE240D128425E50FF0850A0812
:10CB9000850B09750A0078081207F8E50FC333FC06
:10CBA000E433FDEE240EFAEF12CBC112080FEEFAB9
:10CBB000EFFB900A6712CBCE121CF402B2A2FAE588
:10CBC000093400FB12130E7403228E828F8312CB62
:10CBD000D22212CBD622E0F8A3E0F5838882228508
:10CBE0001882851983AA82AB83120E6A8A088B0980
:10CBF000EA450922EA12D65FEB12DAD8FEA3E0FF7B
:10CC00008E828F8322E0F50AA3E0F50B22A3A3E531
:10CC10000AF0A3E50BF022F0A3AE82AF83AC0EAD19
:10CC20000FEEFAEFFB12CC2922121B2AEE2408FE8B
:10CC3000EF3400FF2274F612036374F81208A3891C
:10CC40000812CCB3F974E058F509A3AE82AF83742F
:10CC5000016960097901121B127900802312CC85C9
:10CC600060F7E50970EE8E828F83A312CCA9F9EAF2
:10CC70002400E439FB8E828F83E0F9120EEEA908BE
:10CC8000740802BB92EEFCEFFD851882851983AA19
:10CC900082AB8312CC29851882851983AC82AD833F
:10CCA0007A827B03121B24E922E0FA8E828F83A30F
:10CCB000A3E022EA12861BEB12DAD8240112CCC5BB
:10CCC000F8741F5822FEA3E03400FF8E828F83E0A9
:10CCD0002274F612036374E11208A3EAFEEBFF125A
:10CCE000AAEC604F8E828F8312C2F7851882851955
:10CCF0008312CD387409120A5512CF847003A3E051
:10CD000069603012CBCA1206997508FE7509FF7862
:10CD1000081207FC741C120A55E0F9740D120A552A
:10CD200012A83D740F120A5512C2F7120CAE740409
:10CD300012080F741F02BB92AC82AD83EA241BF56C
:10CD400082EB12DAD8F9EA241CF582EB1293AD12C9
:10CD50000DF22274F7120363E9FE7C007D00780077
:10CD60007900800D12CE11E02CFCA3E03DFD12DC19
:10CD7000AA12DD13502CE8FAE9FBEA75F012A4FAC6
:10CD8000AFF075F012EBA42F12DCB3F460E012CE1A
:10CD90001812A7F660D8EE60CB12CE11E4F0A3F023
:10CDA00080CC78007900800D12CDF1E02CFCA3E05E
:10CDB0003DFD12DCAA12DD065030E8FAE9FBEA7507
:10CDC000F017A4FAAFF075F017EBA42F12DCE270A5
:10CDD00003A3E0F460DC12CDF812A7F660D4EE6095
:10CDE000C712CDF1E4F0A3F080C8ECFAEDFB02C766
:10CDF000F912CDF83BF58322E8FAE9FBEA75F01762
:10CE0000A4FA75F017EBA42FFB74B72AF582740D02
:10CE10002212CE183BF58322E8FAE9FBEA75F012FC
:10CE2000A4FA75F012EBA42FFB74F02AF582740BB0
:10CE30002274F71203638908EAFEEBFF9003BAE05D
:10CE4000C39508501B120E349003EA12CE63900370
:10CE500054E075F064A4FCADF07A007B021284B457
:10CE600002C7F9EEF0A3EFF02274F6120363EAFEB4
:10CE7000EBFF9003D4801388828983E06E7003A354
:10CE8000E06F603A88828983A3A312AAF670E87AD9
:10CE9000047B001213B08A088B09A808A909E84985
:10CEA000601C8882898312CE639003D412C2F788F3
:10CEB000828983A3A312C4FD9003D412BDD702BB01
:10CEC0009574F41203637E009003D480070E888269
:10CED0008983A3A312AAF670F4EEC333FAE433FBFA
:10CEE0001213B08A088B09EA4509607E7F0090031F
:10CEF000D480248882898312A83DEFC333FAE433B7
:10CF0000FBE5082AF582E5093BF583ECF0A3EDF09B
:10CF10000F88828983A3A312AAF670D79003B61252
:10CF2000CF847003A3E069780870191207FCEEF54E
:10CF30000A780A1208007C827D0379009003B612F9
:10CF4000CF70801A1207FCEEF50A780A1208007CEE
:10CF5000827D0379009003B612C2F7120ECA7403E1
:10CF600012080FAA08AB091213B6120B2802A02F41
:10CF70001293B1120ED6228E828F83A3A3A3A3A3F2
:10CF8000A3A3A3A312C661E06822C082C08380105D
:10CF90008A828B8312AB709003D412BDD71213B662
:10CFA0009003D412A7F970E802B77874F6120363FD
:10CFB00090036E12A9FF9003EA12D00712BDD77A30
:10CFC000EA7B037950121B549003EA12D012120F1D
:10CFD000969003EA12A9FF900A6912AAF660257AD0
:10CFE000067B0012132CEA4B601A8A828B8374D55D
:10CFF000F0A3A3E412D0190412D028900A6912CB2E
:10D00000CE121CF402BB9512D00B2212AF37900344
:10D010006E22128A0DFAEFFB2212D01D2212D021AD
:10D020002212A695A3A3A32212D01DA3EEF0A3EF74
:10D03000F022C082C0839003EC7418F0A3740FF048
:10D040009003EE7412F0A3740FF09003F07430F0BC
:10D05000A3740F02A272C082C083900361E064FED9
:10D060007003A3E0F4600E90035BE0A2E1500612AF
:10D070000F78120F1E02B77874F61203639003AF95
:10D08000E06032FE75F0E8A4CEA8F075F003A428A5
:10D09000FF1213268A088B09A808A9099021C0E469
:10D0A0009358F8A3E49359F9EE28FCEF39FD7A0080
:10D0B0007B0112D0B802BB959003BBE0F912146A51
:10D0C0002274EC120363750C00750E00750F0012CC
:10D0D0000B0A7A047900120AB08A08AE087A02793B
:10D0E00001120AB08A087A037903120AB0EEC395D6
:10D0F00008C39AF50B120F4EEAF510E50B2510F553
:10D100000A850B088A12E5082512F8E43400F9E8CC
:10D1100049700302D2148808750900740278081255
:10D120000945AA08AB091213B08A0E8B0FEA450F06
:10D13000700302D211850A0875090074027808127A
:10D140000945AC08AD0979FF12131A750800750975
:10D15000008058A908120B048A128B13AE12AF1369
:10D16000EE4F60448E828F83A3A3A3A3E060046488
:10D17000047035050C8E828F83A3A3A3A3A3A3A35E
:10D18000A3A3A3E0F9120F8A780E1207FCAD0A8E52
:10D19000828F83A3A3A3A3A3A3A3A3A3E0FC8E8254
:10D1A0008F8312D2C612080F12D2B912D2CFE5085D
:10D1B00098E509995007E50CC3950B409675080052
:10D1C00075090085100CC3E508950CE5099400501D
:10D1D00043AA08AB09120F5A8A0C8B0DEA450D6061
:10D1E0002B780E1207FCEA240EF582EB129684FED1
:10D1F000EA240FF582EB128A00120F8AAD0AEEFCC8
:10D20000850C82850D8312D2C612080F12D2B98006
:10D21000B2750A00750C62900359E0600CF9121C9B
:10D220005CE9F87454C398F50C75F003E50C84F5CB
:10D230000B94204003750B1FAE0EAF0F751200E567
:10D240000C6006751220750C00E50BC3950A50059D
:10D25000850B0D8009850A0DE512D2E6F512EEFC6C
:10D26000EFFDAA12A90D120F2AE9F513E512A2E6A5
:10D27000402C150D750800750900800BEE2404FE86
:10D28000EF3400FF12D2B9850D10C3E5089510E503
:10D2900009940040E7E50DC50AC3950AF50AE9704F
:10D2A00006E512A2E65095E50E450F6007AA0EAB03
:10D2B0000F1213B6A91302BB7EE5082401F508E599
:10D2C000093400F509221293B1120F24740222903E
:10D2D00021BC12BD03C32274F2120363EAFEEBFF0A
:10D2E00089088C098D0A740E120A5512C2F77C0047
:10D2F0007D008C0B800EEAFCEBFDEA2404FAEB3493
:10D3000000FB050BE50BC3950A50228A828B83E054
:10D31000F47003A3E0F470188A828B83EEF0A3EF1D
:10D3200012A691A3A3E50912D019E508F0028661BF
:10D33000EC4D600C8C828D83C3E09EA3E09F50B6C1
:10D340008A828B8312D6ECEE98EF9950A9EAF8EB1B
:10D35000F988828983E0F47003A3E0F46011E82483
:10D3600004F8E93400F9050BE50BC3950A40E2E83F
:10D37000FCE9FDE824FCF8E934FFF988828983128E
:10D38000B0B88C828D8312D3B312D3ABA3A3E08C3D
:10D39000828D83A3A312DAF7E08C828D83A3A3A3EB
:10D3A000F0C3EA98EB9940C702D318F088828983CA
:10D3B00022A3A3E50CF0A3E50D2274F2120363741B
:10D3C000FD1208A389088A09ECFEEDFF750A0175B4
:10D3D000F003E9A42402C0E07401120A55D0E0125F
:10D3E000D4656077EA12D461EB12D6727408F074D7
:10D3F0001F55084509A3F012D64C750A0080398ED6
:10D40000828F83E088828983F0A3A882A9838E8299
:10D410008F8312BEBE8E828F83A3A3E05407C4FC09
:10D420008E828F83A3A3A3E054074C12BEC0EE24C8
:10D4300004FEEF3400FF050AE50AC3950840C08AE0
:10D44000828B83A3A374FCF0A374FFF0EA2413F58A
:10D4500082EB12C065120B16E9F50AA90A02865C76
:10D46000EE12D65F2212C0B2EA4B2274F1120363AD
:10D470008A0A8B0B7508007AFE7BFF7CFE7DFFE538
:10D480000A12861BE50B12D672A3E0F509741F552C
:10D4900009F50C12D64CE509A2E74017E50A241756
:10D4A000F582E50B129684FE75F003E50CA42402C8
:10D4B0006E60087901121B1202D649E50C600B88D8
:10D4C000828983E0FEA3E0FBEEFA750D00803988C7
:10D4D000828983E0FEA3E0FDEE2400E43DFFE82422
:10D4E000020808E912A4D1548870C8E05407F50E68
:10D4F000A3A882A983EEFC900361E06E7003A3E011
:10D500006F7003850E08050DE50DC3950C40C0E551
:10D5100008700BA909120F36E9700302D64912D61A
:10D520005612A0168A0C8B0DAE0CAF0DEE4F605349
:10D530008E828F83A3A3A3A3A3A3A3E4F09021D4FB
:10D5400093F88E828F83A3A3A3A3A3A3A3A3E0C373
:10D5500098401D12D688120212E88E828F83A3A3F0
:10D56000A3A3A3A3A3A3F0E508C39407500205084F
:10D570008E828F83A3A3A3A3A3A3A3A3A3E508F0F1
:10D5800002D6497CFF7DFF12D65612842812C2F7BC
:10D59000120F428A0C8B0DAE0CAF0DEE4F7049127C
:10D5A0000F488A0C8B0DAE0CAF0DEE4F700302D6F8
:10D5B000497C177D00790012131A12D6561284285E
:10D5C0001288C312BDD790036EE0F8A312D67DA3D4
:10D5D00012BDD7EE240F128425129F42120212129E
:10D5E000DE35EE240E12C0629021D4E493F8EE24CE
:10D5F0000D129681C398401212D68812021212DEC2
:10D6000035E508C3940750020508EE240E12842560
:10D61000E508F0EE240C12B65E2402FAEF3400FBAB
:10D62000120A6EE97023850A82850B83A3A3A3A344
:10D63000A3A3A3A3E06012E50A2415F582E50B126B
:10D640008A052402FAEF12D66702A0EDE824020848
:10D6500008E93400F922E50A12D65FE50B22EE2430
:10D660000BF58222FAE5093400FB121B2A2212D69E
:10D670005EEF12AA2712AF33888289832212BEB5C9
:10D68000A3A3A3A3A3A3A32212D68C2212D6947A77
:10D69000027B00229021D4E4932401F8E43400F9C1
:10D6A0002274F7120363E9FE74FE6A700374FF6B61
:10D6B00070047901803374605E646060F5EEA2E509
:10D6C000500E90036112D6ECEC98ED99401980E26F
:10D6D000A2E69003615008C3E09AA3E09B80EDC3EB
:10D6E000E09AA3E09B50DB790002C7F912AF33C385
:10D6F0002274F71203637E00800412DEE70E12D854
:10D700006A40F77E00EE12D71C12969688828983B3
:10D71000E4F00EEEC3940340EC02C7F975F003A4E5
:10D72000F8A9F074D628F8740339F988828983A39C
:10D730002274F71203637F0080010F9021DEE493CF
:10D74000F8EFC3985026EF12D9866A7003A3E06BF6
:10D7500070E812DE926C7003A3E06D600A74FF6CD7
:10D76000700374FF6D70D312D85380047A007B006D
:10D7700002C7F974F61203637CFF7DFF7AFE7BFF1C
:10D78000120F42EA4B7045750800803BE50875F0C2
:10D7900017A4F8A9F074B128F582740D39F583E067
:10D7A000600D74B028F582740D39F583E07016743D
:10D7B000A228FE740D39FF8E828F8312C2F7120CDD
:10D7C000B4EEFAEFFB050812D8D040C002BB95C0FA
:10D7D00082C0837A007B007D008014ED12D85D70DA
:10D7E00003A3E0F46008EA24010AEB3400FB0D9087
:10D7F00021DEE493F8EDC39840E102B77874F412A7
:10D8000003638A088B09ECFEEDFF800B120F60EEBC
:10D81000FCEFFDAA08AB09120F42EA4B70EE02A022
:10D820002F74F61203637D007E0080020D0E12D865
:10D830006A501912D85C7003A3E0F460F08D08EA16
:10D8400065087001EB70E512D85380047A007B0004
:10D8500002BB9574A228FA740D39FB22EE75F017FD
:10D86000A4F8A9F012D99164FE229021DEE493F885
:10D87000EEC3982274F7120363EAFEEBFFEE4F60EB
:10D880001012D89474FEF0A30412A510A3141296DB
:10D890009802C7F97C177D00790012131A8E828FC7
:10D8A000832274F7120363EAFEEBFF750800801809
:10D8B000E50875F017A4F8A9F012DEA67003A3E03E
:10D8C0006F600312DEEF050812D8D040E302C7F9FB
:10D8D0009021DEE493F8E508C3982274F412036300
:10D8E0008A088B09ECFEEDFF90036EE06E7003A3D7
:10D8F000E06F7019120ADA8A0A8B0BA80AA90BE8E2
:10D9000049600AE82408FAE93400FB8020EEFCEFC5
:10D91000FDAA08AB09120F428A088B09A808A909B9
:10D92000E8496005E8240D80DD7A007B0002A02F25
:10D9300074F41203638A0A8B0BECFEEDFF7508008A
:10D94000750900802EE50975F017A4F8A9F012DE1C
:10D95000DA601EE50912D986650A7004A3E0650B3A
:10D96000700375080AEEFCEFFD12DD7160034308D9
:10D97000A005099021DEE493F8E509C3985004E579
:10D980000860C20289F875F017A4F8A9F012D991BD
:10D990002212DD66E02274F61203637E007F0080AF
:10D9A00053EEF9120B04EAF8EBF9EA4B6043888274
:10D9B0008983A3A3A3A3E06401603688828983A33B
:10D9C000A3A3A3E064026029E82407F582E9129D7D
:10D9D000F774012AF09003B0E0C39A50148882894A
:10D9E00083A3A3A3A3A3A3A3A3A3A3E412DAEEA3F5
:10D9F000F012DA9312D2CFEE98EF9940A47E007F16
:10DA0000008055EEF8EFF9E875F017A4F8AAF07564
:10DA1000F017E9A42AF912D8647003A3E0F4603582
:10DA200012DA9C240CF582E912DACE740128F09007
:10DA300003B0E0C398501E12DA9C240FF582E9125D
:10DA4000DAC5E8240EF582E912DABA12A50BFAA3B8
:10DA5000E0FB120CB412DA939021DEE493F8C3EEEB
:10DA600098EF9400409D7E007F00EEF8EFF9E87596
:10DA7000F003A4F8AAF075F003E9A42AF912DADE9B
:10DA8000600214F012DA93C3EE9403EF940040DACC
:10DA900002BB95EE24010EEF3400FF22EEF8EFF901
:10DAA000E875F017A4F875F017E9A42AF974A2280C
:10DAB000F8740D39F9E822F582EF12AA27E422EE74
:10DAC0002411F582EF12AA27E4F022F582EB12DA94
:10DAD000D8F822240FF582EF3400F583E02212DA21
:10DAE000E3E02274D628F582740339F5832212DA32
:10DAF000F7A3A3A3A3A322F088828983A3A3A322CD
:10DB000074F21203638A088B09ECFEEDFF740E12A7
:10DB10000A5512CC05750C007C007D018010121393
:10DB200026E50CF5F0EA84ACF0750C007D00780079
:10DB30007900800312DCAA12DD06400302DBCCE888
:10DB4000FAE9FBEA75F017A4FA85F00D75F017EB0A
:10DB5000A4250D12DCE27003A3E0F460D712DCC050
:10DB600065087004A3E0650960CA12DCC06E70032A
:10DB7000A3E06F60BF12DCC0650A7004A3E0650B10
:10DB800060B2E8FAE9FBEA75F017A4FA75F017EB52
:10DB9000A4250DFB74B02AF582740D12DCA15094FB
:10DBA00074016D050C608DE50CC39C4087E875F031
:10DBB00017A4F8AAF075F017E9A42AF974A228F5B9
:10DBC00082740D39F58312C2F702DC9E7800790069
:10DBD000800312DCAA12DD13400302DC85E8FAE9B7
:10DBE000FBEA75F012A4FA85F00D12DCF264FE7007
:10DBF00003A3E0F460DC12DCE865087004A3E065D0
:10DC00000960CF12DCE86E7003A3E06F60C412DC21
:10DC1000E8650A7004A3E0650B60B7E8FAE9FBEA7F
:10DC200075F012A4FA75F012EBA4250DFB74E92A25
:10DC3000F582740B12DCA15099E8FAE9FBEA75F061
:10DC400012A4FA75F012EBA4250D12DCB364016086
:10DC500081E06402700302DBD274016D050C700375
:10DC600002DBD2E50CC39C500302DBD2E875F01254
:10DC7000A4F8AAF075F012E9A42AF974E028F58254
:10DC8000740B02DBC3E50C6011EC700E7401650CC3
:10DC9000600302DB1E7C0102DB297AFE7BFF028629
:10DCA000613BF583E014C3940622E8240108E934BB
:10DCB00000F922FB74E42AF582740B3BF583E02221
:10DCC000E8FAE9FBEA75F017A4FA75F017EBA4255A
:10DCD0000D12DCD522FB74A22AF582740D3BF5836C
:10DCE000E02212DCD564FE22E8FAE9FBEA75F012C4
:10DCF000A4FA75F012EBA4250DFB74E02AF58274EA
:10DD00000B3BF583E0229021DEE493FAC3E89AE925
:10DD10009400229021BCE493FA740193FBC3E89A27
:10DD2000E99B2274F51203638A088B09ECFEEDFF70
:10DD3000750A008002050A9021DEE493F8E50AC323
:10DD4000985021EEFCEFFDE50A75F017A4F8A9F054
:10DD500012DD7160E0E50A75F017A4F8A9F012DD94
:10DD60006612DD80802574A228F582740D39F58352
:10DD70002274A428FA740D39FB121B24E922A3A3F0
:10DD8000E508F0A3E509F02212080F7F030205CA97
:10DD9000E9F87907C3940D400479018019E8C39428
:10DDA0000740047903800FE8C394034004191980E5
:10DDB00005E8700279000207C174F01203638A0853
:10DDC0008B098C0A8D0B890C120F488A0E8B0FAEB3
:10DDD0000EAF0FEE4F605B12D89412DD808E828FF3
:10DDE00083A3A3A3A3A3A3A3A312CC0DE50C600A52
:10DDF000EE240F128425E50C8006EE240F12DE3E81
:10DE0000F09003EE12AAF6601A9003B5E064017078
:10DE100008EE240E12DAB78010EE240E1284257458
:10DE2000078006EE240E12DE3E129F4412021212EA
:10DE3000DE3502CB12EE240D12AA24E8F02212AA3B
:10DE40002474012274F51203638A088B09ECFEED39
:10DE5000FF750A00800F12DEA67003A3E06F600357
:10DE600012DEEF050A9021DEE493F8E50AC398502C
:10DE70001EE50A75F017A4F8A9F012DE9265087085
:10DE800004A3E0650970CF12DE9B12CE6380D4023A
:10DE9000DD8B12DE962212DE9BE02274AC28F58226
:10DEA000740D39F5832212DE966E2274F712036325
:10DEB000EAFEEBFF7508008019E50812D9866E703E
:10DEC00003A3E06F700A12DEDA7005E50812DEE8DF
:10DED000050812D8D040E202C7F974A428FA740DDC
:10DEE00039FB120A6EE922EE75F017A4F8A9F012B8
:10DEF000D853120F602274F71203637E008013124E
:10DF0000D85C7003A3E0F4600812DEDA700312DE5E
:10DF1000E70E12D86A40E802C7F9C082C0839003B6
:10DF2000F274AEF0A3740FF09003F474B4F0A37421
:10DF30000FF09003F674BAF0A3740F02A27274F794
:10DF4000120363EAF8EBF990033512DF85702B8832
:10DF5000828983A3A3A3A3A3A3A3A3A31206999037
:10DF6000033512DF7D120A3288828983A3E0F91219
:10DF70000BA6740212080F120B2802C7F912A4F89C
:10DF8000F5838A8222E012DF8DA3A3E022FAA3E0C8
:10DF9000F5838A82A3A3A3A322C082C0839003B87F
:10DFA00012E05CF09003B812AAF670057901120E27
:10DFB000E802B77874F612036374FC1208A3E9FE52
:10DFC0009021D9E493700874E16E600302E057EA8F
:10DFD0002408F8EB12B2B812E05C12E065700E9003
:10DFE00003B8E4F0A3F07901120EE8806A9011A35F
:10DFF000E06064FA9003B812D6ECEA98E4995057BE
:10E000007900120EE88A088B09AC08AD09ECF8ED2E
:10E01000F9E875F064A4F8AAF075F064E9A42AF9A7
:10E020009003B812C2F712021AE8941AE994004059
:10E0300026900A6112AAF6601E9003B812C1BF12A0
:10E04000BDD77402120A55ECF0A3ED12C264900A17
:10E050006112CBCE121CF4740402BB92E02401F0D6
:10E06000A3E034002212D3AB12AAFB4922C082C023
:10E070008374F81208A3851882851983AC82AD8356
:10E0800075838075822C740812073D851882851966
:10E0900083AC82AD8312C1B4640170047900800244
:10E0A0007901740802AB8674F412036374F81208E1
:10E0B000A37E008E089004C7E4F07F79750A087586
:10E0C0000B00780A1207FC7402120A55AC82AD8369
:10E0D0007A007B00EFF912EA0512080F8518828595
:10E0E0001983E0F47003A3E0F470139004C7E070A8
:10E0F00004EFF080197A01EFF91213C28010740452
:10E10000120A55E0F47003A3E0F46002EFFE0FEF93
:10E11000C3947F40A7EE9004C7601EE0600FF91221
:10E1200013CE7A007B00EEF91213D48013EEF912AD
:10E1300013CEEE9004C7F08007E06004F91213CE0E
:10E140007F79AC087A007B00EFF91213C88B0BEAD9
:10E15000450B60057508017F780FEFC3947F40E29F
:10E16000E508A2E050147F797C007A007B00EFF98B
:10E170001213C80FEFC3947F40EE9004C7E0704ABB
:10E180007F007A0012E1CF64F87004A3E0640770A6
:10E1900004EAFF802AEFC333F8E433F912E1DBC06D
:10E1A00082C08312E1CFF8A3E0F9D083D082C3E02C
:10E1B00098A3E0995002EAFF0AEAC3940640C574A6
:10E1C000792F9004C7F0F91213CE790102EA43EADD
:10E1D000C333F8E433F912E1DBE02274BB28F582A3
:10E1E000740439F5832274F712036374F81208A3D8
:10E1F000EAFF851882851983E4F0A3F0EF600874C4
:10E2000002120A55E480077402120A5574FF12E8DC
:10E21000647A007B001213F8740812080F7F010261
:10E2200005CA74EE12036374F81208A3890C8A0EEF
:10E230008B0F8C0D750A08750B007E007F0075082A
:10E240000875090078081207FC7402120A55AC829E
:10E25000AD83AA0AAB0BA90C12EA0512080F8518A8
:10E2600082851983E0F47003A3E0F4700302E3B045
:10E270007402120A5512E67640087508FC7509FF0B
:10E28000800D7402120A5512E67FF508E9F509744B
:10E29000F8C3950AF87407950BF9C3E89508E99552
:10E2A00009501AEE2400F8EF3408F9E8C3950AFE85
:10E2B000E9950BFF750A00750B0802E3B012EF69D0
:10E2C00012E3CBE849700302E386E50E450F604A8E
:10E2D000A80EE50F547FF9851882851983E06870D0
:10E2E00003A3E069600302E396E50F5480701374A2
:10E2F00006120A55E0F47003A3E0F4600302E3960B
:10E3000080117406120A55E0F47003A3E0F4700360
:10E3100002E396AA0AAB0B02E3C77402120A551273
:10E32000F3D2A90C12E64C7404120A55E06870038B
:10E33000A3E0697046E50D602E7406120A55E0F4FC
:10E340007003A3E0F4704F851882851983E0FAA367
:10E35000E04480FB1213DAEA4B603B7C019004C876
:10E36000E0F91213E6802F7406120A55E0F47003E8
:10E37000A3E0F460217AFF7BFF804C7C01AA0AAB0A
:10E380000BA90C1213E6E5082408F8E5093400F996
:10E39000EE28FEEF39FFE50A2508F50AE50B3509F9
:10E3A000F50BC3E50A94F8E50B9407500302E23E2F
:10E3B000E50C12E658E50AF0A3E50B12E3FEEEF0D9
:10E3C000A3EFF07A007B007408800E85188285190F
:10E3D00083E0F8A3E0F922740412080F7F0A020513
:10E3E000CA74F7120363E9FE121806EE12E65874B7
:10E3F00008F0A3E412E3FEE4F0A3F002E21DF074DF
:10E40000C928F582740339F5832274EE120363740C
:10E41000F71208A389088A0A8B0B7E007F00750C0F
:10E4200001750D00780C1207FC7402120A55AC82BB
:10E43000AD83EEFAEFFB9004C7E0F912EA0512088B
:10E440000F851882851983E0F4600812E66D790063
:10E4500002E641EE24010EEF3400FFC3940840BEF3
:10E460007E087F007401F09004C7E012E658E0F5E2
:10E470000CA3E0F50D750E08750F00780E1207FC61
:10E480007403120A55AC82AD83EEFAEFFBA90812B1
:10E49000EA0512080F7401120A55E0F47003A3E0B4
:10E4A000F4700302E6177403120A5512E676400868
:10E4B000750EFC750FFF800D7403120A5512E67F6E
:10E4C000F50EE9F50F74F8C39EF874079FF9C3E8D9
:10E4D000950EE9950F500302E61774F8C3950CF8F2
:10E4E0007407950DF9C3E8950EE9950F500B851843
:10E4F00082851983E4F002E620EE2408FEEF340062
:10E50000FF7401120A5512E3D1E849700302E603D1
:10E510007401120A55E0650A7004A3E0650B7003EC
:10E5200002E6037403120A5512F3AFEEFAEFFBA9E9
:10E530000812E646120A55E0687003A3E06960031A
:10E5400002E6037407120A55E0F47003A3E0F470C6
:10E550000B7C00EEFAEFFBA9081213E675090078B0
:10E5600009120800E4F510F51178101207FC740682
:10E57000120A5512F3AF7404120A5512E96490049A
:10E58000C7E0F9121410740312080FE9700302E4D3
:10E59000EEE50C2408F50CE50D3400F50D780E12AF
:10E5A00007FC780C1207FC9004C7E0FCEEFAEFFBC6
:10E5B000A90812140A740412080F7403120A5512DF
:10E5C000E69012E646120A55E0687003A3E069601F
:10E5D0000302E4EE7405120A5512E6901213EC8A57
:10E5E000108B11A810A9117405120A55E068700368
:10E5F000A3E069600302E4EE7401120A5512E6908A
:10E6000012141CEE250EFEEF350FFFC3EE94F8EF4B
:10E610009407500302E467851882851983E070052A
:10E6200012E66D8014E50A450B700E12E848A90841
:10E630001213CEE5089004C7F0851882851983E08F
:10E64000F9740902E3D912E64C7405221213F28A16
:10E65000108B11A810A9112212E65C22C333F8E432
:10E6600033F974BD28F582740339F583229004C709
:10E67000E0F91213CE22C3E094FCA3E094FF22122F
:10E68000E68322E02403F8A3E03400F9E854FC22F6
:10E6900012F3AFAA0CAB0D9004C7E0F92274F41288
:10E6A0000363EAFEEB800374804FFF7508797C00FA
:10E6B000EEFAEFFBA9081213C88B0BA90BEA49600D
:10E6C00008E5089004C8F080150508E508C3947FA4
:10E6D00040DCEF548060D09004C8E4F0FAFB02EA1A
:10E6E0004874EE12036374F61208A3890A8A0C8B2D
:10E6F0000D8C088D09741C120A5512EF7EC3EC9420
:10E70000F4ED94FF400E85188285198374FCF0A304
:10E7100074FF801CEC2403F8ED3400F9E854FC2469
:10E7200008F8E93400F9851882851983E8F0A3E92F
:10E73000F07F007C069004C7E004FEEEC3947F40A7
:10E74000027E799004C7E06E602B74872EC333F885
:10E75000E433F974AF28F582740439F58312E9645F
:10E76000E4C39AFA74089BFB12E1D62AFAA3E03BB1
:10E7700012E85350080E1CEC70C102E841EC700323
:10E7800002E841EE12EF88FA74089912E853400348
:10E7900002E81E7510088F1178101207FC7404121D
:10E7A0000A55AC82AD837A007B00EEF912EA0512BD
:10E7B000080F7406120A55E0F47003A3E0F4700B1E
:10E7C00012E85D7A04FBEEF91213FEAA0CAB0DEE13
:10E7D000F91213D4E9606AE50AF50B780B12080008
:10E7E000780E1207FCAC08AD09AA0CAB0D9004C75B
:10E7F000E0F9121410740312080FE960059004C7C1
:10E80000E0FFE50A700AEE850E82850F83F0803105
:10E8100012E848EEF91213CEEE9004C780EFE50A35
:10E82000F50B780B120800780E1207FCAC08AA0C46
:10E83000AB0DEEF9121410740312080FE96002EE2A
:10E84000FFEFF9740A02E3D97A019004C7E0F912E4
:10E8500013C222FB12E3CBC3EA98EB9922851882FC
:10E86000851983E4F0A312EFA12274F212036374FA
:10E87000F81208A389098C08EA24F8F50AEB34FF9A
:10E88000F50B750C08750D00780C1207FC7402125C
:10E890000A55AC82AD83AA0AAB0B12EA0512080F27
:10E8A000E50870237406120A55E4F0A3F07404120C
:10E8B0000A55AC82AD83E50A2404FAE50B3400FB6B
:10E8C000A9091213F880197402120A5512EF921254
:10E8D000E85DAA0AAB0BA9091213F8E50912E8EAE8
:10E8E000740812080F7F060205CAC333F8E433F92F
:10E8F00074C928F582740339F583E02EF0A3E03F54
:10E90000F02274F412036374FE1208A38518828542
:10E910001983ECF0A3EDF08908EAFEEBFFEE24FC8E
:10E92000FEEF34FFFF851882851983AC82AD83EE3C
:10E93000FAEFFB1213FE750A02750B00780A120734
:10E94000FC7402120A55AC82AD83EEFAEFFBA90803
:10E9500012EA0512080F85188285198312E964747A
:10E960000202EA45E0FAA3E0FB2274F012036374AA
:10E97000FC1208A3890C8A0A8B0BECFEEDFF7508CC
:10E9800000750900EE2403F50EEF3400F50F740254
:10E99000780E120A07AE0EAF0F12ED4C6049750EDD
:10E9A00004750F00780E1207FC7402120A55AC822F
:10E9B000AD83AA0AAB0BA90C12EA0512080FE50AEF
:10E9C0002404F50AE50B3400F50B7800880E12EBF1
:10E9D000F6E0FAE5082AF508E5093400F50908E843
:10E9E000C3940450B480E5AA08AB09740412080F5C
:10E9F0007F080205CAE5822510FCE5833400FDAAE4
:10EA00000CAB0DA90E1217FA74022274F4120363F0
:10EA1000E9FE75080175090078081207FC8A088B61
:10EA20000974027808120A078E0AF50B7409780A2D
:10EA3000120945E5082400FAE509350BFB12180018
:10EA400002E95F740812080F7F040205CA74F71206
:10EA5000036374FC1208A38C828D83E08518828581
:10EA60001983F08C828D83A3E0C0E07401120A55F3
:10EA7000D0E0F07402120A5574FFF07403120A55C4
:10EA800074FF12EF9D1213F8740402E21A74EE126E
:10EA9000036374FC1208A38909EAFEEBFF8C0C8D5A
:10EAA0000D7416120A5512EF76EE5403F508606ADB
:10EAB00074FC5EFE750E04750F00780E1207FC7470
:10EAC00002120A55AC82AD83EEFA12EA0512080F63
:10EAD000E50C450D6029850A82850B83E0C0E08541
:10EAE000080E12EBF6D0E012EC090508E50C24FF45
:10EAF000F50CE50D34FFF50DE508C3940440D18510
:10EB00001882851983AC82AD83EEFAEFFBA9091256
:10EB100013F8EE2404FEEF3400FFE50C5403F5086F
:10EB2000850C0E850D0F7402780E120A07850E0CE7
:10EB3000850F0DE50C450D604D780C1207FCAC0AF5
:10EB4000AD0B8E0E8F0F7402780E120A0785091016
:10EB5000F51174097810120945E50E2400FAE50F45
:10EB60003511FB121800740212080F7402780C128F
:10EB70000945A80CA90DEE28FEEF39FFE50A28F596
:10EB80000AE50B39F50BE5086069750E00750C0494
:10EB9000750D00780C1207FC7402120A55AC82AD98
:10EBA00083EEFAEFFBA90912EA0512080F8025850A
:10EBB0000A82850B83E0C0E0850E0C8518828519DA
:10EBC00083E582250CF582E5833400F583D0E012DD
:10EBD000EC09050E85080C74FF250CF5080470CFB0
:10EBE000851882851983AC82AD83EEFAEFFBA90903
:10EBF0001213F802E3D7851882851983E582250E62
:10EC0000F582E5833400F58322F0850A82850B8343
:10EC1000A385820A85830B2274EE12036374FC12AF
:10EC200008A3890E8A0C8B0D8C0B7416120A55E002
:10EC3000F508A3E0F5097418120A55E0FEA3E0FFF9
:10EC4000E5085403F50A6060F510C3E5089510F572
:10EC500008E5099400F50975100475110078101283
:10EC600007FC7402120A55AC82AD83AA08AB09A94D
:10EC70000B12EA0512080FEE4F602A75100178108A
:10EC80001207FC850A107402120A5512E9F51208DF
:10EC90000F12ED5B050AEE24FF1EEF34FFFFE50ABD
:10ECA000C3940440D212ED68EE5403F50A8E108F1F
:10ECB0001174027810120A07AE10AF118029751076
:10ECC0000475110078101207FC7402120A55AC8208
:10ECD000AD8312E9FF12080FE50C2404F50CE50DD5
:10ECE0003400F50D12ED6812ED4C70D2E50A605952
:10ECF0007E007510048E1178101207FC7402120A3F
:10ED000055AC82AD83AA08AB09A90B12EA0512081B
:10ED10000F801975100178101207FC8E1074021202
:10ED20000A5512E9F512080F12ED5B0EAF0A74FFD7
:10ED30002FF50A0470DD851882851983AC82AD83B6
:10ED4000AA08AB09A90B1213F802E3D7EEF8EFF902
:10ED5000E824FF1EE934FFFFE84922E50C2401F511
:10ED60000CE50D3400F50D22851882851983AC82DF
:10ED7000AD83AA08AB09A90B1213F8E5082404F522
:10ED800008E5093400F5092274EC12036374F812E3
:10ED900008A389088A108B11ECFEEDFF741C120A7F
:10EDA0005512EF7E741E120A55E0F50CE912E65872
:10EDB00012EF76750900851882851983EAF0A3EBB6
:10EDC000F07402120A55EEF0A3EF12EF9DAA0AABFF
:10EDD0000BA9081213F875120875130078121207A0
:10EDE000FC7402120A55AC82AD83AA0AAB0BA908C7
:10EDF00012EA0512080F851882851983E0651070E4
:10EE000004A3E06511600302EF127402120A55E0D8
:10EE10006E7003A3E06F600302EF12E50C70030253
:10EE2000EEF0850E82850F83EEF8EFF9E85403F5D6
:10EE30000CE58245837015E875F0FFA4F8AAF0751B
:10EE4000F0FFE9A42AF9E8FAE9FB80207A007B00C8
:10EE5000800AE0FCEA2CFAEB3400FBA3E8FCE9FDB5
:10EE6000EC24FF18ED34FFF9EC4D70E6E50C601E64
:10EE70007404C3950CF895E0F9E875F0FFA4F8ACBC
:10EE8000F075F0FFE9A42CF9EA28FAEB39FB7404D9
:10EE9000120A55EAF0A3EBF012EF69E50E450F6098
:10EEA00017780E1207FCEEFCEFFDAA0AAB0BA908BF
:10EEB000121404740212080FEEFCEFFDAA0AAB0B49
:10EEC00012F3C47404120A55E0687003A3E0697079
:10EED000227404120A5512F3FC7404120A55E068F5
:10EEE0007003A3E069700C85188285198312F3F50D
:10EEF0007509017402120A55C3E094F4A3E094FF6B
:10EF000040067EFC7FFF80437402120A5512EF9286
:10EF100080397402120A55C3E094F4A3E094FF40D0
:10EF2000067EFC7FFF80087402120A5512EF9212CF
:10EF3000EF86F8740899F9C3E89EE99F500812EF2C
:10EF400086FE740899FFE50812E8EAE508C333F87D
:10EF5000E433F974BD28F582740312E8F7A9097443
:10EF60000812080F7F0C0205CAE50A2408F50AE515
:10EF70000B3400F50B22E0F50AA3E0F50B22E0F5D7
:10EF80000EA3E0F50F22E50812E65C12E3D1E4C31C
:10EF9000982212E6832408FEE93400FF2212EFA132
:10EFA00022F0851882851983AC82AD8322C082C08D
:10EFB000837900E9C333FCE433FD743C2CF582749F
:10EFC000803DF583E06A7003A3E06B600709E9C345
:10EFD000940340DFD083D0820207C174F61203632A
:10EFE000E9FE8A088B09ECFAEDFB12F0CD500E1207
:10EFF000F0D6EE12F0E2E508F0A3E509F07F020298
:10F0000005CAC082C0831213BC80C974F2120363A4
:10F01000EAFEEBFF8C088D09740E120A5512EF768A
:10F02000794E1217CAE97004790A8037EEFAEFFBBD
:10F030001213DAEA4B6010EEFCEFFD9004C8E0F921
:10F0400012141C7900801C780A1207FCAC08AD0968
:10F05000EEFAEFFB79011213E0740212080FE96077
:10F06000C7790902E8E574F412036374F81208A37F
:10F07000EAFEEBFF12F0CD503F12F0D6E09004C84C
:10F0800012F0E212E964750A08750B00780A12079B
:10F09000FC7402120A55AC82AD83EA24F8FAEB3410
:10F0A000FFFB9004C8E0F912EA0512080F7402127F
:10F0B0000A5512E96402EA43EEFAEFFB1213DA8B07
:10F0C0000BA90BEA4970BF7A007B0080E812141686
:10F0D000E9F8C394032274C928F58274043400F556
:10F0E0008322F0E812F0E822C333F8E433F974CC59
:10F0F00028F582740439F5832274E812036374F5E9
:10F100001208A38A168B178C0C8D0D7423120A55C6
:10F11000E0F512A3E0F513751100794E1217CAE954
:10F120007005790A02F3A5E5124513700302F3A3F3
:10F13000AA16AB171213DA8A088B09A808A909883E
:10F140000A890B7401120A55E8F0A3E9F09004C88B
:10F15000E0F510E8450B7005790902F3A57508087C
:10F1600075090078081207FC7405120A55AC82ADC7
:10F1700083EA24F8FAE934FFFBA91012EA05120821
:10F180000F7405120A55E50C2512F8E50D3513F933
:10F19000C3E098A3E099408A12F3B5120A5512EF22
:10F1A0007EAE12AF137508008071751401751500DD
:10F1B00078141207FC7402120A55AC82AD83AA0AB5
:10F1C000AB0BA91012EA0512080F85188285198366
:10F1D000E0F8850E82850F83E0686026750801746B
:10F1E00007120A55C3E098F0A3E09400F0850E8260
:10F1F000850F83E0F87407120A55E028F0A3E03485
:10F2000000F0E50A2401F50AE50B3400F50B850E44
:10F2100082850F83A385820E85830F12ED4C708A41
:10F22000E508A2E0400302F3A3851882851983E470
:10F23000F085820885830978081207FC7407120A92
:10F240005512F3AFAA16AB1779001213E07402122D
:10F25000080FE9F508700302F34D7405120A551200
:10F26000E67640067EFC7FFF800B7405120A55127D
:10F27000E67FFEE9FF12F3DA7409120A55E0F47032
:10F2800003A3E0F4700A7C007401120A5512F3EA39
:10F29000780C1207FC780A1207FCAC087405120AF5
:10F2A0005512E964A91012140A740412080F12F31B
:10F2B000B5120A55120699AC12AD13AA0AAB0BA9E6
:10F2C00008121404740212080F7405120A55E0C3E0
:10F2D000950CF8A3E0950DF9E8C39512F50EE995A4
:10F2E00013F50F780E1207FCE50A2512F50AE50B57
:10F2F0003513F50B780A1207FCAC087405120A5591
:10F30000E0250CF8A3E0350DF9E82512FAE93513EC
:10F31000FBA91012140A740412080F12F3DA740510
:10F32000120A5512F3D212F3C47407120A55E06898
:10F330007003A3E06970167407120A5512F3FC7487
:10F3400007120A55E0687003A3E069600575110AA9
:10F3500080087403120A5512F3F585188285198303
:10F36000E060266510700B740A6511700512E66D79
:10F37000801712E84885188285198312E67085186F
:10F3800082851983E09004C7F0851882851983E08F
:10F390006510600F740A651160097C01EC120A5552
:10F3A00012F3EAA911740B12080F7F100205CAE0CC
:10F3B000FCA3E0FD22E50A250CF50AE50B350DF569
:10F3C0000B742522A9081213F28A0C8B0DA80CA924
:10F3D0000D2212F3AFAA0AAB0B22E50812E65CE09D
:10F3E000C39EF50AA3E09FF50B22E0FAA3E0FBA978
:10F3F000101213E62212F40B12141C2212F40B1238
:10F4000013EC8A0C8B0DA80CA90D22E0FCA3E0FDE7
:10F41000AA0AAB0BA9082274F0120363EAFEEBFF01
:10F420008C0A8D0B7410120A55E0F50CA3E0F50D53
:10F430007412120A55E0F508A3E0F50912F0CD5058
:10F44000278882AE82780C1207FCAC08AD09EE1258
:10F45000F0E8E0250AFAA3E0350BFB74C92EF5822B
:10F4600074043400F5838023EEFAEFFB1213DAEA1A
:10F470004B7004790A801E780C1207FCAC08AD09A9
:10F48000EA250AFAEB350BFB9004C8E0F912EA050D
:10F4900012080F790002E9F074F4120363EAFEEB3C
:10F4A000FF8C088D097A097B001213B0EA4B603596
:10F4B00090049E12FCEA8A828B8312FCD890049EF0
:10F4C000EAF0A3EB12F57CEEF0A3EF12F4E8E50806
:10F4D000F0A3E50912F4E8A3A3743212F4F6740160
:10F4E00012F4F6A3F002FEDB12F4EC22F08A828B17
:10F4F00083A3A3A3A32212F4ECA3A3A32274F61262
:10F500000363EAFEEBFF8E828F83E0F91212DE8B3B
:10F5100009EA45096004790280187C007D00EEFA52
:10F52000EFFB1212BA8B09EA4509700479108002C8
:10F53000790002FDD774F212036389088A098B0AE5
:10F540001212E48A0C8B0DAE0CAF0DEE4F60287AD0
:10F55000047B0012132CEA4B601D8A828B8374FD9E
:10F56000F0A3E50A12F57CE50812F57CA3E509F0A5
:10F570008E828F8312F97A7F060205CAF08A828B07
:10F5800083A3A32274E812036374FC1208A3740219
:10F59000120A55ECF0A3EDF07401120A55E9F08A55
:10F5A000108B11741C120A55E0F512A3E0F51374C8
:10F5B00021120A55780C1209F890049EE0F508A370
:10F5C000E0F509750AFE8A828B83E0540C640C70A6
:10F5D0001779FE12F786700302F75712F76170036E
:10F5E00002F75712F778803BA3A3E0F4700BE5080D
:10F5F0004509700302F757801D8A828B83A3A3E01D
:10F60000F91212E48A148B15A814A915E8FEE9FF73
:10F61000E849600F80CD850882850983A3A3E0FEB9
:10F62000A3E0FFEE4F700302F7578015A90A12F707
:10F6300086700302F75712F761700302F75712F74B
:10F64000787516FF7517FF85088285098312F79A6A
:10F650008E828F836028E0FA79028508828509838B
:10F66000A3A3A3A312FD24121CF4EA4B60278A82F1
:10F670008B83E0F516A3E0F5171213B6801712F787
:10F680009B60128E828F83A3A3A312FD24A3E0F5B7
:10F6900016A3E0F517851082851183A3A3A3A3A366
:10F6A000A3A3A3E065167004A3E0651760168E821D
:10F6B0008F83E07076851082851183A3A3A3A312A4
:10F6C000F79A7067E5102402F514E5113400F5157A
:10F6D000851482F583E0851882851983F08E828FE8
:10F6E0008312F76F780C1207F47424120A55E0F5B0
:10F6F0000B780B1208007423120A5512069978121F
:10F700001207FC740B120A55120699740C120A5552
:10F71000E0F9EEFCEFFDAA10AB111212D2740B123D
:10F72000080F85188285198312F76F85108285115D
:10F7300083E0540C640C700302F62CA3A3E0F47075
:10F7400016850882850983E0F508A3E0F509E50838
:10F750004509600302F616740412080F7F100205B3
:10F76000CA1212E48A088B09AE08AF09EE4F22E0F4
:10F77000851482851583F0228E828F83E0F9121220
:10F78000DE8A088B0922A3A3A3A3E0FAA3E0FB125D
:10F790001BBAE9F50A74FE650A22A3A3A3A3E0F845
:10F7A000A3E0F9E8492274E81203638A088B098C04
:10F7B000128D138917741C120A55E0F50AA3E0F59F
:10F7C0000B741E120A55E0F516741F120A55780CB8
:10F7D0001209F8EA240EF582EB12F95C12FCDEEA5B
:10F7E0002410F582EB12F95CE02424FA7B0012135A
:10F7F0002C8A148B15AE14AF15EE4F700302F9531B
:10F800008E828F83741A12FCC912F96A12FCD88591
:10F810000882850983A3A312F96AA3A312FCD874F2
:10F8200018120A5512FCF0EE2406FAEF3400FB120F
:10F830001302850882850983A3A3A3E0C0E0EE2418
:10F840000F12F959D0E0F0851282851383E0C0E0F1
:10F85000EE241412F959D0E0F0E508240CF582E505
:10F860000912F95CE0C0E0EE241512F959D0E0F07D
:10F87000850A82850B83E0C0E0EE241612F959D088
:10F88000E012F961E0C0E0EE241712F959D0E0125D
:10F89000F961A3E0C0E0EE241812F959D0E0F0EECF
:10F8A000241912F959E516F0EE241A12F959780CB8
:10F8B000120A16EE241E12F959E51712FCC9A3A369
:10F8C000A3A3A3A312FCE6EE241212FCD1741A1215
:10F8D0000A5512FCEAEE241012FCD1EE241F12F994
:10F8E00059E4F0E5082410F582E50912F95CE0F826
:10F8F00012F956E8F0A3E4F0E86041EE2422F8EFB4
:10F900003400F9E8FAE9FBEE24240808EF3400F9A2
:10F910008A828B8312FCD8851008851109750A002C
:10F9200078081207F812F95612FCF08A828B8312BB
:10F93000FD4712130E740312080F800AEE242212E0
:10F94000F959E4F0A3F0EEFAEFFB851282851383F8
:10F9500012F97A02F75CEE2420F582EF3400F58389
:10F9600022F0850A82850B83A322A3A3A3A3E0F838
:10F97000A3E0F98E828F83A3A322A3E0F8A3E0F58E
:10F98000838882E0F91213382274EA12036374E266
:10F990001208A3EAFEEBFF8C088D09890A74341261
:10F9A0000A5512FCDE7436120A55E0F50EA3E0F596
:10F9B0000F7438120A55E0F514A3E0F515743A12E5
:10F9C0000A55E0F50CA3E0F50D743C120A55E0F57C
:10F9D0000BEC45097005790202FCBF8E828F83A370
:10F9E000A3A3A3A3A3A3A3E060ECE9A2E3503B8EEF
:10F9F000828F83A3A3A3A3A3A3A3A3E0640270D6CF
:10FA0000120E108A128B13A812A9138E828F83E014
:10FA1000687003A3E06960127C03790112FD431250
:10FA20000C96E9600579CD02FCBF8E828F83A3A37B
:10FA3000A3A3A3A3A3A3E0640260118E828F83A378
:10FA4000A3A3A3A3A3A3A3E0640F702212FD4312F8
:10FA50000E82E98E828F83A3A3A3A3A3A3A3A36093
:10FA600005740FF0803CE0640F703702F9D68E8287
:10FA70008F83A3A3A3A3A3A3A3A3E0640360238E04
:10FA8000828F83A3A3A3A3A3A3A3A3E06401601213
:10FA90008E828F83A3A3A3A3A3A3A3A3E0600302E7
:10FAA000F9D6EE2408F8EF12FE82C0E0740A120ABA
:10FAB00055D0E012FE8B7012EEFCEFFD7402120ABC
:10FAC00055AA82AB83121B2A800F8E828F8312FC71
:10FAD000EA7402120A5512FCD87411120A55E4F0A5
:10FAE000A3F090049E12F79E604B88828983A3A3A3
:10FAF00012FD47E5086A7003E5096B888289837007
:10FB0000E412FCE6E8FCE9FDEC4D602985088285FD
:10FB10000983E0FA79028C828D83121CF4EA4B602F
:10FB2000368A828B8312FCEA7411120A5512FCD8B1
:10FB30001213B6802285088285098312F79B60170D
:10FB4000850882850983A3A3A312FD2412FCE9740E
:10FB500011120A5512FCD87417120A55E4F0A3F0DA
:10FB6000E50AA2E4501A740A120A55E0640F601004
:10FB7000E06401600B7417120A557404F0A3E4F0FA
:10FB8000E50AA2E750097417120A55E04410F0E59F
:10FB90000AA2E650127417120A55E04401F07401EB
:10FBA000120A55740180067401120A55E4F0E50A40
:10FBB000A2E250097417120A55E04440F0851882F9
:10FBC000851983E4F0850C82850D83E0C0E074190B
:10FBD000120A55D0E012FCC9E0C0E0740B120A55BD
:10FBE000D0E0F08E828F83A3A3A3A3A3A3A3A3A398
:10FBF000E0C0E0740C120A55D0E0F0740F120A5500
:10FC0000E510F0A3E511F07413120A55E50EF0A308
:10FC1000E50FF07415120A55E514F0A3E515F09000
:10FC20001170E0C0E0741A120A55D0E0F0741B1293
:10FC30000A55E50BF0851882851983AA82AB8312D9
:10FC400012F0E9C3950EE4950F502090031412F7BB
:10FC50009E60147402120A55AA82AB839003151297
:10FC6000FD25121CF480107E02800E7402120A55CB
:10FC7000AA82AB83121CBCE9FE740A120A55E06426
:10FC800002702E120E108A0E8B0FA80EA90F74028E
:10FC9000120A55E0687003A3E0697015EEFB850C4D
:10FCA00082850D83E0FA850882850983E0F91212C6
:10FCB000C6EE7009850C82850D83E004F0EEF974C0
:10FCC0001E12080F7F0E0205CAF08508828509837F
:10FCD00022F582EF3400F583E8F0A3E9F022E0F5A5
:10FCE00010A3E0F51122A3A3A3A3E0F8A3E0F92257
:10FCF000E0FCA3E0FD22C082C08390049E80048AC1
:10FD0000828B8312FD47EA4B600B8A828B8312FD44
:10FD100020E06970EAD083D0820207C18C828D8393
:10FD2000A3A3E0F8A3E0F58388822274F6120363AC
:10FD300012FDDC6007A3A312FD4780047A007B005C
:10FD400002FDD78E828F83E0FAA3E0FB2274F412C7
:10FD50000363EAFEEBFF89081212DE8A0A8B0BAC02
:10FD60000AAD0B7900EC4D603E8C828D83A3A3A37A
:10FD7000A312FD47EA4B601CAA08098C828D83A35D
:10FD8000A312FD20121CF48E828F83EAF0A3EBF005
:10FD90007901801B12FD1CA3A3A312FD478E828F45
:10FDA00083EAF0A3EB80078E828F83E4F0A3F00256
:10FDB000FEDB74F71203638A828B83E064017004B4
:10FDC0007E0880027E00A3AA82AB83121CB6E9C320
:10FDD0009EF97F010205CA7F020205CA1212DE8A5D
:10FDE000828B83E582458322C082C08390049E1269
:10FDF000FCEA88828983790080080912FD478A829B
:10FE00008B83E582458370F202FD15C082C083902A
:10FE1000049E801A12FD1CE0F8E96003E8600BE81C
:10FE20008A828B83F0A3AA82AB838C828D8312FC9F
:10FE3000F0EC4D70DF02FD1574F7120363EAFEEB80
:10FE4000FFEC2408F8ED12FE828E828F83A3A3A319
:10FE5000A3A3A3A3A312FE8B7005121B2A800E8CF2
:10FE6000828D8312FCEA8E828F8312FCD88E828F61
:10FE700083A3A3A3A3A3A3A3A3A3A3E4F0A3F00238
:10FE8000FDD23400F988828983E022F08882898358
:10FE9000E064032274F4120363EAFEEBFF1212DE45
:10FEA0008A088B09A808A909E849700D8E828F83FA
:10FEB0007432F0A37401F08022E82406F508E934D6
:10FEC00000F509750A0078081207F87C027D00EE3B
:10FED000FAEFFB12130E740312080F7F040205CA17
:10FEE000C082C08312FF356004790080358A828B1E
:10FEF00083A3A3A3A3A3A3A3A3E060ED64028A82C8
:10FF00008B83700E12FF297003A3E06970DB790107
:10FF10008010A3A3A3A3A3A3A3A3E0640370CA12A6
:10FF20001B24D083D0820207C1E0F8A3E0F98C82C1
:10FF30008D83E068228A828B83A3A3A3A3A3A3A3B8
:10FF4000A3E0F88C828D83A3A3A3A3A3A3A3A3E020
:10FF50006822C082C0838C828D83A3A3A3A3A3A3A2
:10FF6000A3A3E0F88A828B83A3A3A3A3A3A3A3A341
:10FF7000F07403687005121B2A80128C828D83E056
:10FF8000F8A3E0F98A828B83E8F0A3E9F002FF226C
:10FF900074F6120363750808EAFEEBFF8E828F8306
:10FFA000A3AA82AB83ECF8EDF988828983A3AC82A3
:10FFB000AD838E828F83E0FE88828983E06E600449
:10FFC000790080081508E50870CE79017F020205E6
:10FFD000CA74F51203638C088D09750A007808123B
:10FFE00007F87C087D0012130E740312080F7F03BC
:03FFF0000205CA3D
:020000040001F9
:100000008882898312839A22129FB4F9EA2290048B
:1000100002129FB4FB12103822E0F508E4F509F54E
:100020000AF50B227401F0900B88E0640F2274092A
:1000300012080F7F040205CAEE2412FAEF3400FB07
:100040001211D6E92212080F7F060205CA7905129D
:1000500011E2740422A3A3E024F5C394122212181F
:10006000A28A0C8B0D8C0E8D0F221212B4900BA84D
:1000700012A8507A147B0022C082C083900402121E
:100080009D546009900402129FAF1213B69003FFB3
:1000900012953D7408F0A3E4F0A3F090046EF09084
:1000A0000404F07C0BFDF97A057B0412131A7C0B17
:1000B0007D0079007A107B0412131A0294AA74F15D
:1000C00012036374F71208A3EAFEEBFF128CCB74E1
:1000D000051297497403F0EE24020A0AEF34001265
:1000E000817F2421FCEF3400FD8C828D83E08882A7
:1000F000898312818A600BEE241F128CCE74FFF06C
:10010000A3F0EE241FEF34001C1CFD8C828D83A312
:10011000E0C0E0129407D0E012818A8882898312BD
:100120009ACF7403F0EE2417F508EF12B130AC0843
:10013000FD851882851983AA82AB83121B2A740855
:10014000120A557403F0EE242212B1021207F87C51
:100150000B7D00AA08AB0912AD0C12080F900B9D85
:100160001206997402120A55AC82AD8312A4F112E0
:10017000080FE97007EEFAEFFB1210CE02B178FB20
:10018000128196E8F0A3E9F0EE22F0128196E8F0F1
:10019000A312B4E6E0221282638A828B832274F077
:1001A000120363EAFEEBFF8C088D09890A741012B2
:1001B0000A5512B1357412120A5512B564EE2402B2
:1001C0000A0AEF3400FB128263850F0DE50D888269
:1001D000898312828DE50E12828DE50A12827F904C
:1001E0000BA212827A900BA112827AED12827BEC22
:1001F00088828983F0E8FC8A828B83E0C39C8E82AC
:100200008F83A3A3A3A312A93F12A0798508828597
:100210000983A3A3A3A3A3A3A3A3E064037005126C
:1002200082718004128CCBE41297497409F0750C2A
:1002300005750D04750E00780C1207F8129E7E12DB
:10024000080F750CFF750DFF780C1207FCAC08AD9C
:100250000912A4F112080FE97007EEFAEFFB121071
:10026000CE80388A828B83E024FFF8A3E034FFF944
:1002700022EE240E12AAA6740122E088828983123B
:10028000828322F0E824FF18E934FFF922128283E6
:1002900088828983221287D312080F7F080205CA39
:1002A00074F0120363EAFEEBFF890B8C0E8D0F7561
:1002B0000A00A2AFE433F50CC2AF90041B803512E4
:1002C000837E502D12838B6403702612A3C785088A
:1002D00082850983A3A3E02405FCA3E03400FDEE9E
:1002E000FAEFFB121B2A12A3D07410250AF50A1587
:1002F0000B12936012B033E50B6006E508450970F8
:10030000BEE50CA2E092AFA2AFE433F50CC2AF9011
:10031000041B80222402F8E50912B184FAE9FB8A61
:10032000828B8312AA9712A40112940712A40105CA
:100330000A150B129360129371602512838B64026D
:1003400070F112837EE50840CB12918BE509128390
:100350007850E0850E82850F837401F0E50B70D331
:10036000E50CA2E092AF8E828F83E50AF0EE24FFC7
:10037000FAEF34FFFB02829B12875CA2E522E508BC
:1003800012A3E9E50912875CA2E6228508828509A5
:1003900083A3A312940F12839A22A3E01313543F52
:1003A00054032274ED12036374F61208A389128AAF
:1003B000108B0F851882851983E4F0900421E0C327
:1003C000940840057511078003E0F511E5113333FA
:1003D0003354F8900B87F8E0282433F50A129DC6B1
:1003E0007003028517EA250AF8EB3400F9EA2402C3
:1003F000F50AEB3400F50B850A82F58312A079909B
:100400000B87E0FCFAC3E49AFA95E0FBE82AFEE9E0
:100410003BFF900B8512A3EE750E00780C1207F8C7
:100420007D00EEFAEFFB12AD0C12080F85188285E5
:100430001983AC82AD83A911EE24FFFAEF34FFFBE0
:10044000120FE48A0C8B0DAE0CAF0D8E828F83E4FD
:1004500012A40BE50FC454F0F990046FE0C43333D9
:1004600054C0F8900B81E0A2E0E4331313484944F0
:100470000F12A407E510C454F045128E828F83F04A
:10048000EEF8850A82850B83E0C39885088285098A
:1004900083A3A3A3A3F0850A82850B83EEF0A3EFC9
:1004A000F0E508240E128525E508240D1285257433
:1004B00009120A55E4F0750C10750D04780C12073A
:1004C000F87C0B7D00E5082417FAE509129E8712D7
:1004D000080F851882851983E0600EE508240EF563
:1004E00082E509128B7ED2E3F0E4F50AF50B780A77
:1004F0001207FC7403120A55AE82AF831211C4EEC8
:10050000FCEFFDAA08AB0912A4F712080FE9AA082C
:10051000AB0960071213327A007B00740A12080FCD
:100520007F0B0205CAF582E50912AAA9E4F022743C
:10053000F31203638A0A8B0BA2AFE433F50CC2AF4C
:1005400075080075090090041B8026128762501EF2
:10055000850A82850B83A3A312B564129FA9121189
:10056000CAE9600A128752C2E6F08E088F09128724
:10057000421289A070D5E5084509600612863FD26F
:10058000E6F0E50CA2E092AF7F050205CA74F01216
:100590000363EAFEEBFF8C0C8D0D750E00A2AFE439
:1005A00033F50FC2AF75080075090090041B802455
:1005B000850A08850B0912863FD2E4F0E5081291FE
:1005C0008BE509128B7ED2E7F0E50A24FBF582E584
:1005D0000B12B16612B0EAE50A450B604BE50A1250
:1005E000A3E9E50B128B7EA2E750DE850A82850B1C
:1005F00083A3A3120699AC0CAD0DEEFAEFFB12111A
:10060000D0740212080FE960C0E508450960A1E551
:1006100008240DF582E50912899A700C85088285F7
:10062000098312A9CDD2E4F0E50FA2E092AFE5086C
:10063000450960061210C8750E01A90E02829BE5DD
:100640000812A3E9E50912875C2274F212036374AD
:10065000FE1208A3750C00750D008518828519839C
:10066000E4F0A3F0A2AF33F50AC2AF90041B12B0BE
:10067000F2802FEE24FBF582EF34FF12973712073A
:10068000FC12873412080FEEFCEFFD8518828519E5
:1006900083AA82AB8312134AAE08AF09900421E00B
:1006A00014F0EE4F60251287625017EE240B12876C
:1006B0004C24FFF0A3E034FFF088828983129D541C
:1006C00060B18E0C8F0D12874280A3E50AA2E092E2
:1006D000AF900421E0602C900B88E0640F600690DE
:1006E000046EE0701E7AF97B031212B490805B12E4
:1006F00006957AF97B031287D312080F800574F0F0
:1007000012941C851882851983AA82AB8312135018
:100710008A088B09AE08AF09EE4F6013120FF01272
:100720008752A2E28E828F83A350D374E980D17462
:1007300002028045EEFCEFFD7A1B7B04121C8074E4
:100740000222EE24FBF582EF12B16622F8EF12B11D
:10075000232212875622EE2410F582EF3400F5830F
:10076000E022128756A2E72274F7120363EAFEEB37
:10077000FF120FF090115A12940B121CF4E964014D
:10078000900BA4700AE02401F8A3E034008004E098
:10079000F8A3E0F9EE240B128CCE12A0799004217C
:1007A000E0701F900B88E0640F70177AF97B0312DA
:1007B00012B490805B1206957AF97B031287D312EC
:1007C000080FE5A8F8C2AF900421E004F0E8A2E722
:1007D00002A03B1212A874042274F7120363EAFE0B
:1007E000EBFF12880FF0120FF0EEFCEFFD7A1B7B8F
:1007F00004121356E5A8F8C2AF900421129043905A
:100800000B88E0640F7005790812117C02990512BB
:100810008756C2E42274F712036374EA1208A3EA4B
:10082000FEEBFF900B81E06035851882851983749B
:1008300001F0120A55E41288A5120A55AA82AB8368
:10084000121B2A8E828F8312A9CDC0E0740A120A6D
:1008500055D0E012A72C740B120A55129A987416F0
:10086000028D60C082C083120FD80294AA74F7125E
:10087000036374EB1208A3EAFEEBFF851882851967
:100880008374061288A5120A55AA82AB83121B2A0A
:10089000EE2407FCEF3400FD740A120A55129A98F0
:1008A0007415028D60F0EE2412FCEF3400FD74022A
:1008B0002274F712036374F71208A3EAFEEBFFEE4B
:1008C0002421128B7B604112A4FD85188285198337
:1008D000AA82AB83121B2A7408120A557403F09083
:1008E0000B9D120699EE241F128CCE120699900BC6
:1008F000B0E0F97404120A55AC82AD83EEFAEFFB56
:10090000120FDE740412080F7409028D6074F21263
:1009100003638A088B09750A00750B00750CE7A242
:10092000AFE433F50DC2AF90041B80078E0A8F0B26
:100930001287421289A0602B12876250EF128994AD
:1009400070EAEE242E12898C8A828B83A3A3E0683E
:1009500070DA780A1207FC12873412080F9004210B
:10096000E014F0E50DA2E092AFEE4F6013EEFAEF67
:10097000FB120FF079F0EEFAEFFB121182750C000A
:10098000A90CAA08AB09121182028048F582EF1265
:10099000875CF822EE240DF582EF12875C64012259
:1009A000E0FEA3E0FFEE4F2274F412036374F7122B
:1009B00008A3EAFEEBFF121032E9F508704AEE24B4
:1009C0000E128B7B60427A00790912107AEA4B6032
:1009D000377408120A55128A181206997508FF759D
:1009E00009FF78081207FC8E828F83A3A3A3A3A319
:1009F000A3A3A3E0F97404120A55AC82AD83120FCD
:100A0000DE740412080F800D8E828F83A3E5081216
:100A10008BDD12103E02802E740212B15174FFF071
:100A2000A312AD252274F1120363EAFEEBFF7508F1
:100A3000008E828F83A3A3A3A3A3A3128055400398
:100A40007508E88E828F83A3A3A3A3A3A3A3A3A364
:100A5000A3E0C3941040057508E880138E828F834D
:100A6000A3A3A3A3A3A3A3A3A3A3E0640F600B90DA
:100A7000044BE0540870037508E8EE240B12898CCF
:100A80008E828F83A3A3A3A3A3A3A3A3A3A3E0C343
:100A900098500DEE240B128B7B640F60037508E8F1
:100AA000900BA1E0F47003A3E0F470037508EC7AF6
:100AB000237B001213B090040212B18E9004021234
:100AC0009D5460288E828F83A3A3A982AA83890C58
:100AD0008A0D750E00780C1207F87C237D009004B7
:100AE00002129FAF12AD0C12080F800375081AA9ED
:100AF0000802B17D74F5120363EAFEEBFF8E828F6C
:100B000083A3A3A3A3A3A3A3A3E0900B8812AD2B5D
:100B1000900BA3F0EE240B128B7B900B8312AD2174
:100B2000A3A3A3A3E090046FF0F91219A490046F9B
:100B3000E0600CEE2404129723EE2406128B8290C0
:100B4000046E128024600474018001E4900404F0B7
:100B5000EE240D12AD151207F87C0B7D007A057B93
:100B60000412AD0C12080FEE24181299501207F857
:100B70007C0B7D007A107B0402959CF582EF128736
:100B80005C22FAEF3400FB79E112198C2274F7121F
:100B90000363EAFEEBFF8E828F83A3E07003128073
:100BA0000E8E828F83742C12A8CB02990574F712D3
:100BB0000363EAFEEBFF900402129D546010900460
:100BC00002129FAF900402E4F0A3F01213B68E82DB
:100BD0008F837408128BDD121B96029905F0EEFAD2
:100BE000EFFB2274F612036390046EE06010900431
:100BF00004E0700A128C01EA4B60031210CE02A9C5
:100C0000F4900B83E0FB900BA3E0FA900B88E0F9E3
:100C1000120FEA2274F512036374EF1208A3EAFEBE
:100C2000EBFF8E828F83A3A3A3A3A3A3E0A2E24042
:100C300003028CC6EE242AF582EF340012B562EE70
:100C40002412FAEF3400FB120FF6E9707990804617
:100C5000E064017031EE241A1297317029851882F0
:100C60008519837410F0EE241212B0DF7402120A98
:100C700055128183242A12B0DF7404120A55E8F059
:100C8000A312B0CE804012AD121207F87C0B7D008B
:100C90007409120A5512AD0812080F1211C4E9FAAC
:100CA0007406120A5585820885830978081207FCA4
:100CB000EE242A128CCE1206997B3012A6D079012E
:100CC00012804F12080F741102959FEE240EF582C8
:100CD000EF12AAA922C082C08390046FE0600312C1
:100CE00012360294AAC082C08390046674B8F0A33E
:100CF0007421F0A37435F0A37421F0A374ACF0A3B5
:100D00007421F09011667446F0A3741FF0900450A3
:100D100074D2F0A3740FF09011507402F0A3741009
:100D2000F09011527408F0A37410F090044BE0445A
:100D3000028002F0A3F00294AAC082C083128D4503
:100D40007903029B24EAFCEBFDEA2413F582EB1203
:100D5000875CFA22C082C083128D457905029B24EC
:100D600012080F029905C082C083790802AB6DC0DA
:100D700082C08374FE1208A380077A1B7B04128D45
:100D8000AD90041B129D5470F190041D129D54608F
:100D9000097A1D7B04128DAD80EF90041BE4F0A353
:100DA000F0900421F0A3F0A3F07402801612135007
:100DB000851882851983EAF0A3EB12B0431211B8AB
:100DC00022741112080F0294AA74F6120363E9FF49
:100DD0008F087484129E737421129E78FE8E08FA16
:100DE0007B0012132CEA4B6017EA2508F8EB34005D
:100DF000F98A828B8312A939A3A3A3A3E4F08022EA
:100E00007A027B0012132CEA4B60138F0874631272
:100E10009E737421129190F0A3741A1291A57A0016
:100E20007B0002A9F4E9FDEAFC74062DFAECA2E0CD
:100E3000501EEA75F00A84A8F0E86014740A2AC308
:100E400098FAE8C394054004740A2AFA740B2AFA43
:100E5000EDC394134004781480027806E82A24092C
:100E6000F8E43400F97A0A7B00120212E8F902076A
:100E7000C1C082C08390044BE05402600A121B9CE4
:100E8000E960047901800279000294AAC082C083DB
:100E900090044BE054026014900421E0700A129D0B
:100EA000516009128EB150047901800279000294D8
:100EB000AA900424E02410129380A2E722C082C0EA
:100EC00083908044E0F8900423E0C3985005121307
:100ED0002C80047A007B000294AAC082C083121185
:100EE000B879000294AAC082C08374FE1208A38558
:100EF000188285198312904C600D14606524FE7071
:100F000003028F86029010900B88E0640F60181225
:100F1000118EE97012851882851983129FAF901186
:100F20005412940B121CF4900BB0E0C0E0851882B0
:100F3000851983129AADD0E0129032F81290207485
:100F400014129032FCA3E0FD7A1D7B0412134AE5D3
:100F5000A8F8C2AF900423129043792012117C02AA
:100F60008DA9121188E98518828519836011129460
:100F70000B740D129032FAA3E0FB121B9680E01264
:100F8000940B741580BB1293867003029010851821
:100F90008285198312A9CAC0E0129025D0E0129070
:100FA000322402F81292772401FAA3E03400FB887D
:100FB00082898312904C14C394095020129386FAAC
:100FC000851882851983A312B288A3A3A3E0F874BD
:100FD000A228F5827421129E786A600F129025E093
:100FE0006408702C12938664087025851882851910
:100FF00083E0F812938C14129050240AC0E08518F4
:1010000082851983129020D0E012905004028F4103
:10101000851882851983AA82AB831211B8028F5F6B
:10102000A31294162285188285198312B295A3A360
:10103000A3221290362212B151E022E5A8F8C2AFE5
:10104000900422E004F0E8A2E792AF22EAF0A3EBDA
:10105000129036F8129391A3E022C082C0839004CC
:1010600026129D546008129021121CF4800279000F
:101070000294AA74F7120363EAFEEBFFEE240D124A
:101080008274F0EE242F128B7BC0E0128CCBD0E068
:10109000F0EE2430128B7BC0E0EE2412128CCED006
:1010A000E012A700C0E0EE2413128CCED0E0F0EEE8
:1010B000242B128CCE120699EE2422FCEF3400FD74
:1010C000EE242D128B7BF912A4F712080FE970079A
:1010D000EEFAEFFB1210CE029905C082C083121106
:1010E0008EE960047920800279010294AAC082C04E
:1010F00083EA12A3E0E0D2E0028D35C082C0831201
:10110000A3D912899A701112919A400C8A828B830A
:10111000A3E0F91211828069129184128B7EA2E6FB
:1011200050128A828B83A3E0F990115612940B120D
:101130001CF4804D12A3D912899A700D12919A5005
:10114000088A828B83743080358A828B83A3E06423
:101150001B8A828B83700474228023A3E0700F1299
:10116000A3D912898F745828F5827421800D12A397
:10117000D912898F746328F582742112919012918B
:10118000A50294AAEA12918BEB22EE240FF582229B
:1011900012AAA9E4938A828B8322EA12918BEB1222
:1011A000875CA2E322F0900446E0F912133822741F
:1011B000F7120363E9FE129D51602EEE702E90042B
:1011C0002412AA97E4F0900424129FAF1210BC904E
:1011D0000424E0240E128EB7500312AB5C9004245A
:1011E000E4F0A3F0791012117C029905741B6E7063
:1011F0001012927B640570C690042412AA97EE80A8
:10120000C474E96E7050900424E02411F8129277AF
:1012100060E6900424E0240E181818129277A2E2D7
:10122000900424E0400C241112927414F0121AD08D
:1012300080B7240F129276C2E7F012927B6403709B
:101240000C900424E02410129274D2E2F0129285E1
:10125000121CF40291CF741C6E709D900424129F96
:10126000AF90115C12940B121CF4900424E4F0A3D0
:10127000F00291E908080812938122900424E024E6
:101280000D12938022900424129FB4FB90115212ED
:10129000940F2274F4120363750A00750B00A2AF59
:1012A000E433FEC2AF129D516008EEA2E092AF029D
:1012B000935890115A12940B121CF4E94410F890B0
:1012C000041B800985080A85090B1293601293712B
:1012D00060D812863F586870EB780A1207FCAC0899
:1012E000AD0912873812080F900424E508F0A3E531
:1012F00009F0128EB14064900422E014F0EEA2E0F6
:1013000092AF900424E0240E181812B182FEE9FF77
:101310008E828F83E0FA900424E0F812938CF91205
:101320001080E990041FF0A3E412A856E0A2E75051
:1013300018900424E0241212936C1219C89004240B
:10134000E0241312936C1219BC900424129379A216
:10135000E1B3E433F9121AB8028033900421809A81
:10136000E50824FBF582E50912B16622129380F9A3
:101370002212B037E508450922E0240F129380229B
:10138000F812B142E022851882851983129391E008
:1013900022129415A3A3A3A32274F7120363EAFEF7
:1013A000EBFF1211B212918AEF12919F400A12893B
:1013B0009470059080428003908043E0F9EEFCEF4A
:1013C000FD7A1B7B04121362E9602FEEFAEFFB90AB
:1013D000115812940B121CF4EE240EF582EF1294A5
:1013E00094400812903B1210C88019EEFAEFFB905F
:1013F000115012940B121CF4800A8E828F83A374F6
:10140000F112941C0299058A828B8312940F221286
:10141000941322E0F8A3E0F583888222128BDD1278
:1014200010BC22C082C0831210C80294AAC082C01D
:1014300083790090044BE05402700712948E50029E
:1014400079E890044BE05460700FEA242FF582EBAA
:10145000128B7EA2E1500279E88A828B83A3A3A338
:10146000A3E0C39475400279E8EA242DF582EB12DB
:101470008B7E7012EA242AF582EB128B7E7007793C
:10148000F51211828024E970F81210AA80F6EA247D
:101490002FF582EB12875CA2E222C082C0838A828F
:1014A0008B83740DF0121B968000D083D0820207CC
:1014B000C1C082C0838A828B83E4F0A3F012948E31
:1014C000908042E0F8400F900422E0C398400F79EA
:1014D000F112118280D4900421E0C39850F1129D42
:1014E000D480F174F6120363E9FE244AFAE434006E
:1014F000FB12132CEA4B601DEE8A828B83A3A3A3FD
:10150000A3F0EA244AF8EB3400F98A828B83A3A380
:1015100012A07980047A007B0002A9F4C082C08303
:10152000900442E4F0900445F090042E12953D742E
:1015300002F090043712953D7401028D35747CF0F1
:10154000A37411F0A32274F512036374F11208A3BB
:101550008518828519837402F07401120A55E9F026
:1015600060047AFF7BFF7402120A5512B18E75086F
:101570003A750904750A0078081207F87C0B7D009B
:101580007407120A5512AD0812080F8518828519C2
:1015900083AA82AB83121B96740F800312AD0C12C8
:1015A000080F7F030205CA74F712036374FE120862
:1015B000A3851882851983740AF07401120A5512E2
:1015C000B0CE7402028D6074F012036312AE8A1200
:1015D00009F87808790C12027378081207F47A3146
:1015E0007B0402829574F412036374CB1208A390F7
:1015F0000B88E0640F600D851882851983742E12A4
:101600009FC980227A287B0412806A12021A8808F5
:101610008909E4F50AF50B78081207F47A287B04A7
:101620001287D312080F743502803074F1120363ED
:1016300074F71208A3EAFEEBFF780012972E6007FA
:10164000E06403600278E8EE2417128CCE12805713
:101650005022E87021EE2417128B82EE242212977A
:101660002312972E7022EE241912B0DF900B9712DE
:10167000A079802678E8E88E828F83A312A856741A
:1016800017F012119402B178900B9774FEF0A30436
:1016900012973F7A8E7B0B121B2AEE2425F508EF5A
:1016A000340085080CF50D750E00780C1207F87CD7
:1016B0000B7D007A3A7B0412AD0C12080F12827176
:1016C000129749740212973F851882851983AA825E
:1016D000AB83121B1EEE2422F582EF3400129737E3
:1016E0001207F8129E7E12080FEE2402F8EF12B1D4
:1016F00084FAE912817F242412A50678081207FCD7
:101700007402120A55AC82AD8379831A1A12A4F5B9
:1017100012080FE96003029685EEFAEFFB1210CE75
:10172000029685FAEF3400FB795012198C22EE24D0
:1017300021128759640222F58312B037780C22F007
:10174000EE2419FCEF3400FD22F0EE240D12AAA6BF
:101750002274F612036374F71208A3900445E07034
:10176000387401F0F9121A82851882851983AA82C9
:10177000AB831211BE75083A75090478081207FC8C
:10178000900B9D1206997B017404120A55AC82AD30
:10179000837A0312804D12080F740902A9F174F7BD
:1017A00012036312997C7004A374EBF0900445E07B
:1017B000A2E25003C2E2F0E0A2E1500512998D804E
:1017C000098E828F83742A12A8CB02990574F412B1
:1017D000036374FE1208A312988CEE2402F8EF340F
:1017E00000F9129AB9851882851983129AD3E0F507
:1017F0000B7012851882851983AA82AB83795312E4
:10180000198C12B02512AD121207F87C0B7D007AEC
:101810003A7B0412AD0C12080F85188285198312C9
:101820009FAFA90B1210F8900445E0A2E1500A8E78
:10183000828F83A3E0F91210FE900445E4F0740255
:1018400002803074F7120363EAFEEBFF8E828F830F
:10185000A374EBF0900445E0A2E1500579EB12107F
:10186000FEEEFAEFFB12112E02990574F7120363D4
:1018700012988C900442E4F0900445F07AFF7BFFCC
:101880008E828F83A3E0F91210F88079EAFEEBFFD5
:101890007901121A887A287B041212B47A317B04F7
:1018A0001212B42274F7120363EAFEEBFF1211283E
:1018B000804C74F71203631299E5A3A3A3E06003BD
:1018C000E4800274EB1298F15003C2E2F0E0A2E16E
:1018D000500512998D8011A2E0500D8E828F837475
:1018E0002AF0A374EB12A8CBEEFAEFFB1210E08003
:1018F000148E828F83A3F0900445E0A2E222EEFAD8
:10190000EFFB12122A7F010205CA74F6120363EA82
:10191000FEEBFF900445E0D2E1F07901121A82EE6D
:10192000240D1299501207FCEE240B128CCE1206D5
:1019300099EE2402EF3400FF0E0E7401C0E0121184
:10194000C4E9FAD0E0FBEEFCEFFD12804D02A9F1F4
:10195000F508EF12B13078082274F7120363129978
:101960007C7004A374EBF0900445E0A2E25003C243
:10197000E2F0E0A2E1500312998D8089EAFEEBFFCC
:101980007901121A888E828F83E0642022C2E112CC
:10199000A710E0F91210FE2274F7120363EAFEEBBF
:1019A000FF7901121A887A287B0412B315E06003CC
:1019B000E4800274EB1298F15003C2E2F0E0A2E17D
:1019C000500312998D0298E874F71203631299E597
:1019D00074EB1298F65003C2E2F0E0A2E150031259
:1019E000998D029905EAFEEBFF7901121A888E8221
:1019F0008F83A32274F7120363129A0A0298FE746B
:101A0000F7120363129A0A029905EAFEEBFF7A289D
:101A10007B041212B4EEFAEFFB1211522274F71289
:101A2000036374EF1208A3EAFEEBFF12A6D07A8ECE
:101A30007B0B121B18E9605B85188285198374097A
:101A4000F07401120A5574EF12B159129AB9F87470
:101A500002120A55E8129AD3A3A3E0C0E07404125C
:101A60000A55D0E0129ACFE0640870168E828F83F8
:101A7000A3A3129AADA3E0C0E07405120A55D0E00A
:101A800080067405120A55E412A72C7406120A5532
:101A9000129A987411028D60AA82AB831211F48598
:101AA0001882851983AA82AB83121B9622129AB1DF
:101AB0002212B299A3A3A3A322E8FAE9FB8A828B9C
:101AC0008312A85088828983E0FCA3E0F9EC2212FB
:101AD000A72122F0A3E9F08A828B8312B29522C05B
:101AE00082C0831212360294AAC082C0839004621C
:101AF00074EDF0A37420F0A37499F0A37421F09016
:101B00001160740AF0A37420F0A37482F0A3741E11
:101B1000F090044E74F2F0A37410F090044BE04483
:101B200001028D351211A00294AA74F61203637497
:101B3000FE1208A3900447129D5460077A477B0465
:101B40001211B890044DE4F09004E5129D54602CFD
:101B5000800D851882851983AA82AB831211B890F3
:101B60000446E0F912133E8A088B09A808A90985E2
:101B7000188285198312A079E84970D602A9EF74FA
:101B8000F6120363E9FA7B00900446E0F912136849
:101B900002A9F474F712036374F01208A3EAFEEBCF
:101BA000FF89088E828F83E0F8744D28F5827421B6
:101BB000129E78C0E07401120A55D0E0F0640B70F8
:101BC0000D8E828F83A3E9F0121218029C8BE070B5
:101BD00003029C8B640C6003029C777404120A5508
:101BE000EEF0A3EF12A6F8C0E07403120A55D0E09D
:101BF000129ACFA3120A327406120A55120A3E8EA6
:101C0000828F83A3A3A3A3A3A3A3A3A312B0E67469
:101C10000A120A55128183240E128B7BA2E450090A
:101C2000851882851983E48012EE241112898C9024
:101C30000BAAE0C398851882851983F0E0C0E07490
:101C40000C120A55D0E0F0EE2414128B7BC0E07425
:101C50000D120A55D0E0F0EE2415128B7BC0E07413
:101C60000E120A55D0E0F0EE2416128B7BC0E07401
